:020000040800F2
:1080000070E20020A1810008A981000805AA0008EB
:10801000AD810008AF810008B181000800000000B8
:10802000000000000000000000000000B381000814
:10803000B581000800000000B7810008B981000880
:10804000BB810008BB810008BB810008BB81000820
:10805000BB810008BB810008BB810008BB81000810
:10806000BB810008BB810008BB810008BB81000800
:10807000BB810008BB810008379900083F990008C0
:10808000BB81000847990008BB810008BB8100083C
:10809000BB810008BB810008BB810008BB810008D0
:1080A000BB810008BB810008BB810008BB810008C0
:1080B000C5920208BB810008BB810008BB81000893
:1080C000BB810008BB810008BB810008BB810008A0
:1080D000BB810008E3A00208EBA00208F3A002089D
:1080E000999D0008BB810008BB810008BB81000886
:1080F000BB810008BB810008BB8100084F990008C4
:10810000BB810008BB810008BB810008BB8100085F
:10811000D3A00208DBA00208BB810008BB810008D5
:10812000BB810008BB810008BB810008BB8100083F
:10813000BB810008BB810008BB810008BB8100082F
:10814000BB810008BB810008BB810008BB8100081F
:10815000BB810008579900085F990008FBA002083E
:10816000BB810008BB810008BB810008BB810008FF
:10817000BB810008BB810008BB810008BB810008EF
:10818000BB810008BB810008DFF810D000F058FC6C
:108190000048004741BF0208AFF3008070E20020B2
:1081A0000648804706480047FEE7FEE7FEE7FEE791
:1081B000FEE7FEE7FEE7FEE7FEE7FEE75D92020868
:1081C000898100082DE9F0410024061B254671F144
:1081D000000605DA01240027D0EB070067EB010158
:1081E000161E73F1000605DA0027D2EB07020125FF
:1081F00067EB030300F0C1FA86460E4617469C461D
:10820000AC4204D00025D0EB050E65EB010624B18D
:108210000020D2EB000760EB030C704631463A4673
:108220006346BDE8F081202A06DBCB17203A41FAED
:1082300002F043EAE07306E041FA02F3D040C2F1F3
:108240002002914008431946704740EA01039B070A
:1082500003D009E008C9121F08C0042AFAD203E0BB
:1082600011F8013B00F8013B521EF9D27047421E43
:1082700012F8013F002BFBD111F8013B02F8013B42
:10828000002BF9D17047421C10F8011B0029FBD1CB
:10829000801A704730B505460020034600E05B1C9D
:1082A000934205D2EC5CC85C201A01D1002CF6D1B7
:1082B00030BD2DE9FE4F804681EA0300C00F0C4619
:1082C000009021F0004123F00045B8EB0200A941E5
:1082D00005D24046214690461C460B46024623F0F6
:1082E0000040104347D0270DC7F30A00C3F30A51DB
:1082F0000290401A019040286BDAC3F3130040F457
:10830000801B0098924620B10023D2EB030A63EB56
:108310000B0B01985946C0F14002504600F05EFA3E
:1083200006460D4650465946019AFFF77CFF10EB72
:1083300008006141002487EA115284EAE7731A4376
:1083400040D0009A62B3019A012A4FEA075215DC25
:10835000001B61EB02014FF0004202EA0752CDE937
:108360000042001C41F5801132462B4600F0EAFA2B
:1083700003B0BDE8F08F40462146F9E7001B61EBF2
:108380000201001C41F5801300185B412018A2F582
:10839000001747EB030140EAD570B6196D4111E0B3
:1083A0006D084FEA360645EAC0754FEA0752001BD2
:1083B00061EB0201001C41F5801149084FEA3000D1
:1083C0000019514132462B4603B0BDE8F04F00F092
:1083D000AABA0098012240000023D0EB020263EB0E
:1083E000E073009821464FEAE074B8EB000061EBBF
:1083F0000401E9E783F000435BE781F0004158E7BF
:108400002DE9FE4F81EA030404F0004421F000410D
:1084100000944FF0000B23F0004350EA01045ED0BB
:1084200052EA03045BD0C3F30A54C1F30A552C4447
:10843000A4F2F3340194A0FB0254C1F3130141F4FC
:108440008011C3F3130343F4801301FB024400FBC8
:10845000034E840A970A44EA815447EA8357A4FBEF
:10846000076802958D0A05FB07854FEA932C04FBEC
:108470000C542705029D4FEA065847EA1637B5EB1C
:1084800008056EEB070C870E920E47EA811742EA49
:108490008312A7FB0201B6EB0B0164EB00042B0D6A
:1084A00043EA0C335E1844EB1C50DA465146E7FBB6
:1084B0000201C5F313044FEA0B3343EA14534FEAA6
:1084C0000432019C43EA0603A4F10C040294009CCC
:1084D000CDE900B400F036FA03B0BDE8F08F00201B
:1084E0000146F9E72DE9F04D81EA030404F0004B61
:1084F00021F0004514464FF0000A23F0004150EAF5
:10850000050220D054EA01021DD0C5F30A570246E5
:10851000C5F31303C1F31300C1F30A5640F48015E9
:1085200043F48013A7EB0608101BD64608F2FD386B
:1085300073EB050002D308F1010801E092185B41DA
:10854000B8F1000F03DA00200146BDE8F08D0020ED
:108550004FF48011064684460EE0171B73EB0507A7
:1085600005D3121B63EB050306434CEA010C4908D3
:108570004FEA300092185B4150EA0107EDD152EA10
:10858000030012D082EA040083EA0501084305D003
:10859000101BAB4106D20122002306E000224FF05F
:1085A000004302E06FF0010253101AEB06004CEB9F
:1085B000085110EB0A0041EB0B01BDE8F04D00F053
:1085C000B2B9F0B4CA17CB0F50405140C61841F1B0
:1085D00000054FEAC372314628004FF0960303D0DE
:1085E000B623F0BC00F071B930460021F9E70EB5B2
:1085F000C10F80EAE0700844CA07002140F233430B
:108600008DE80E000A460B4600F09CF903B000BD51
:108610000EB540F2334102910021CDE900110A4626
:108620000B4600F08FF903B000BD3EB5CA17CB0F63
:10863000002450405140C0186141DA0740F23343F2
:108640000094CDE901232246234600F07BF903B0D4
:1086500030BD10B500F0004420F00040C20DC0F362
:10866000160040F400007F2A02DA0020014610BD07
:108670000021962A03DCC2F19602D04002E0963A2D
:1086800000F0ACF8002CF2D00023D0EB030063EB39
:10869000010110BD70B5C1F30A5201F0004500247C
:1086A000C1F3130140F2FF3341F480119A4201DA21
:1086B000002070BD40F233439A42A2F2334203DC01
:1086C000524200F09AF800E090402C43F1D0404232
:1086D00070BD70B5C1F30A5201F000450024C1F32A
:1086E000130140F2FF3341F480119A4202DA002074
:1086F000014670BD40F233439A42A2F2334203DC9A
:10870000524200F07AF801E000F068F82C43F0D013
:108710000023D0EB030063EB010170BD00F00042C9
:1087200030F000400AD0C10D01F56071C0F31600B1
:1087300042EA0151C2084007114370470020014638
:10874000704701F0004330B421F0004150EA0102CB
:1087500006D00A0DA2F56072C1F31301002A02DCF3
:1087600030BC00207047440F44EAC104C100E01847
:1087700030BC00EBC25000F09FB82DE9F05F054619
:10878000002092469B4688460646814640241BE0D0
:10879000284641464746224600F02FF853465A469F
:1087A000C01A914110D311461846224600F016F81F
:1087B0002D1A67EB01084F4622460120002100F0E8
:1087C0000DF817EB00094E41201EA4F10104DFDC77
:1087D000484631462A464346BDE8F09F202A04DB3E
:1087E000203A00FA02F1002070479140C2F12003C4
:1087F00020FA03F3194390407047202A04DB203A03
:1088000021FA02F00021704721FA02F3D040C2F1B0
:108810002002914008431946704700000FB400231E
:1088200000B589B00CA900910B996FF00042CB60A4
:108830001E4B06931E4B07930423CDE901321D4ABC
:10884000089202466B46002000F0A6F909B05DF8D8
:1088500014FB70B586B006464FF0FF300091CDE9AD
:108860000101002015460C4604903246694604A8D2
:10887000FFF7D4FF02460498211825B108B1084635
:1088800000E020462860049800280DD0002A02DD70
:108890000098884208D0081B0094CDE901043246B4
:1088A000694604A8FFF7BAFF06B070BDD18D000875
:1088B000EF8D0008658A00080029A8BF7047401C9A
:1088C000490008BF20F00100704710B4B0FA80FCE6
:1088D00000FA0CF050EA010404BF10BC704749B123
:1088E000CCF1200421FA04F411FA0CF118BF012193
:1088F00021430843A3EB0C01CB1D4FEA00614FEA73
:10890000102042BF002010BC704700EBC350104441
:108910000029A4BF10BC7047401C490008BF20F0CC
:10892000010010BC704710B5141E73F1000408DA82
:10893000401C41F1000192185B411A4301D120F023
:10894000010010BD2DE9F04D92469B4611B1B1FAE0
:1089500081F202E0B0FA80F220329046FFF73EFF4B
:1089600004460F4640EA0A0041EA0B0153465A46C4
:10897000084313D0114653EA010019D0C8F1400250
:108980005046FFF73AFF05460E46504659464246C6
:10899000FFF724FF084305D0012004E020463946B4
:1089A000BDE8F08D0020054346EAE0762C433743CE
:1089B0000A986305E40AA0EB08000022FD0A44EAD5
:1089C00047540A3002D500200146E9E70105101995
:1089D0006941DDE9084500196941BDE8F04DA2E7AC
:1089E00070B521F0004303430CD0C1F30A550024B5
:1089F000D5EB040564EB0403D617AD1AB34102DBD3
:108A00000020014670BD201841EB025170BD0000EE
:108A100030B5041E71F1000404DB4FF00044404205
:108A200064EB0101141E73F1000405DB1C464FF0DA
:108A30000043524263EB0403994208BF904230BDA9
:108A4000064C074D06E0E06840F0010394E807009B
:108A500098471034AC42F6D3FFF79AFBD84403088A
:108A6000F8440308C0B24FF4F05100F03BBA0000E4
:108A70002DE9FF4F087883B09946FF2805D0491C9F
:108A80002D2804D00024002008E000200BE0012461
:108A9000F9E700EB800003EB4000491C0B78FF2B4B
:108AA000F7D104B1404200230293147819461D46C1
:108AB0002D2C01D02B2C04D1521C2D2C13D0002492
:108AC0000294AA461478FF2C0FD00A25A3FB057840
:108AD00001FB05814FF0000C03FB0C11521CE31944
:108AE0004AEB0101EEE70124EAE7814453EA010081
:108AF00002D019F5C87F06DA03980021C0E90011F9
:108B000007B0BDE8F08F0025AE4E2F46DFF8B882E3
:108B1000184600F0FBF9CDE90001B9F1000002DAD6
:108B2000C9F1000400E004460023A74A1AEB030B36
:108B300042EB045A12E0E00707D02A463346384693
:108B40004146FFF75DFC074688462A4633461046F5
:108B50001946FFF755FC05460E466410002CEAD175
:108B6000DDE90001B9F1000F5A46534606DAFFF776
:108B7000B9FC3A464346FFF7B5FC05E0FFF740FC79
:108B80003A464346FFF73CFC029A0AB181F00041A5
:108B9000039AC2E90001B3E72DE9FF4F1F468DB0EC
:108BA000D7E901464FF0FF382E2045464FF0000927
:108BB0000B90B9696D1C0E988847396A82468847C0
:108BC0000028F6D1BAF1FF3F0AD024F4D064002E79
:108BD00011DDBAF12B0F08D0BAF12D0F0BD102E045
:108BE000404611B08DE744F48064B9696D1C0E985D
:108BF00088478246761E6946600501D52D2000E033
:108C00002B208DF8000001F1010B0DF1200809E087
:108C1000B9696D1C0E98884782460F9844F4007419
:108C2000761E0560002E02DDBAF1300FF0D00B99F0
:108C30008A453ED144F0800406E00F99681CA9F1F2
:108C4000010944F400740860B9696D1C761E0E9821
:108C5000884782463028F0D02BE00B998A4505D111
:108C6000200603D444F08004761E18E0504622F01B
:108C700081FD08B30DF11301761E44F400748B4599
:108C800008D2AAF130000BF8010B200607D5A9F194
:108C9000010003E0200602D409F101008146A0058D
:108CA00002D50F99681C0860B9696D1C0E98884739
:108CB0008246002ED1DC53E0002E51DDBAF1650F63
:108CC00002D0BAF1450F4BD1A00549D5B9696D1C49
:108CD00024F44074761E0E9888478246002E0CDDE0
:108CE0002B2804D0BAF12D0F07D144F48074B96950
:108CF0006D1C0E9888478246761EE00501D52D2111
:108D000000E02B2108F8011BCDF82C8021E00DF1AB
:108D10002901761E44F4007488450CD2AAF1300073
:108D200010F0FF0088F8000002D10B99884509D99E
:108D300008F1010806E0E00501D5244801E042F20F
:108D40000F708146B9696D1C0E98884782460F984E
:108D50000560002E04DD504622F00CFD0028D6D11F
:108D6000F9690E988847FF208BF8000088F800000A
:108D70000020069007904B466A4608A906A8FFF710
:108D800077FEA00502D46FF001002AE714F0240F4B
:108D90000AD0E00714D1DDE906123868031D3B60F4
:108DA0000068C0E900120BE0DDE90601FFF7C9FC2D
:108DB0000146E00704D13868021D3A60006801608E
:108DC00028460EE7000014400000F03FF1D8FFFFF6
:108DD000426842B1016811F8013B23B1521EC0E95B
:108DE0000012184670470121C160881E7047426812
:108DF0005AB1C368016843B983688B4205D0491EE4
:108E0000521CC0E90012002070474FF0FF3070473D
:108E10002DE9F04D00231A461B1A8A4103DB00207E
:108E20000146BDE8F08DC1F30A52C1F3130141F4CC
:108E300080154FF0000BD10702D100186D41521E72
:108E40000027044640F2FF11384601EB620A3E4615
:108E50008046024600204FF48011FFF7CEFCC21975
:108E60007141BB1846EB0100B4EB030C75EB000C31
:108E700004D3E41A65EB000517460E46241908F1E1
:108E800001006D4180463428E3DDF91946EB060008
:108E9000091BA84103D24FF0FF32134601E0002224
:108EA00013461BEB070046EB0A51BDE8F04DFFF7F8
:108EB0003ABD000030B5041E71F1000404DB4FF030
:108EC0000044404264EB0101141E73F1000405DB11
:108ED0001C464FF00043524263EB04038B4208BF31
:108EE000824230BD7F2801D9002208E0064A02EB09
:108EF0005002C007127800D1120902F00F020120BF
:108F00009040084070470000984403080EB540F2B6
:108F1000334202920022CDE900221346FFF712FDF0
:108F200003B000BD70B58C1810F8015B15F0070395
:108F300001D110F8013B2A1106D110F8012B03E0F2
:108F400010F8016B01F8016B5B1EF9D12B0705D4FA
:108F50000023521E0DD401F8013BFAE710F8013B43
:108F6000CB1A921C03E013F8015B01F8015B521E5F
:108F7000F9D5A142D8D3002070BD10B502461078B3
:108F800003E012F8014B2318D8B20B1EA1F1010423
:108F9000A1B2F6D110BD000070B5ADF5287D044634
:108FA0000D460020A790A690002604EB44004549FA
:108FB00001EBC000408AA84203DC00200DF5287DAB
:108FC00070BD0020A69077E004EB44003D4B03EB1E
:108FD000C000028A04EB440003EBC00080892844EF
:108FE00081B2394800F010F90020A79011E004EB9D
:108FF0004400344901EBC0004068BDF89C12405C5D
:1090000001A9BDF89C228854BDF89C02401C80B286
:10901000A79004EB44002B4901EBC000008ABDF887
:109020009C128842E3DC04EB4400264A02EBC000B9
:10903000008A401E81B201A8FFF79FFF23490870F4
:1090400004EB44001F4901EBC000008A401E01A947
:10905000085C1E490978884226D10020A79016E0B6
:1090600004EB4400174901EBC0004068BDF89C12B6
:10907000405C04EB4401134A02EBC1018968BDF86E
:109080009C228854BDF89C02401C80B2A79004EB3F
:1090900044000C4901EBC000008A401EBDF89C1240
:1090A0008842DDDC012089E7642022F0A1FDBDF8C3
:1090B0009802401C80B2A690BDF89802062883DB77
:1090C00000207BE7001D0308D89B0020310A002008
:1090D0002DE9F043ADF5257D04460E460025002719
:1090E000A846A94604EB4400324901EBC000408A7F
:1090F000B04204DC00200DF5257DBDE8F08300259D
:1091000018E004EB44002B4901EBC0008068405D8F
:1091100004EB4401274A02EBC1014968485504EBBE
:109120004400114601EBC0004068405D0DF80500A9
:10913000681C85B204EB44001E4901EBC000008AA4
:10914000401EA842DDDC04EB44000A4602EBC000EE
:10915000008A401E81B26846FFF70FFF04EB44010E
:10916000144A02EBC101098A491E0DF801000027CB
:109170001BE004EB44000F4B03EBC000028A04EB3E
:10918000440003EBC0008089304481B2684600F09F
:109190004FF931462046FFF7FFFE012800D1AAE72C
:1091A000642022F025FD781C87B2062FE1DB002029
:1091B000A1E70000001D030808B5002000901DF085
:1091C00035FB0F49087000F09BF80D480078242803
:1091D00004D0272807D028280FD109E0002109480A
:1091E00080F8151E09E00121064880F8151E04E0EC
:1091F0000221044880F8151E00BF00BF08BD000012
:109200002C0A0020BC2200202DE9F04106460D4624
:1092100017460024012022F0A3FA002028490880E4
:109220000DE01DF0E5FA00F0800000B10BE0012038
:1092300022F0DEFC22480088401C2149088020489A
:109240000088C828EDDB00BF1D480088C82832DA36
:1092500010211C4801F0CAFB08211A4801F0C8FB84
:10926000E82000F031F8C5F3871000F02DF8A906CA
:10927000080E00F029F8002000F026F8002404E091
:10928000002000F021F8601C84B2042CF8DB0024DC
:1092900005E0FF2000F018F83055601C84B2BC4295
:1092A000F7DB1021074801F0A3FB002022F058FA59
:1092B0000120BDE8F081002022F052FA0020F8E7FA
:1092C0002E0A00200000024010B5044600BF022113
:1092D0000A481DF0BBFB0028F9D0214607481DF0C5
:1092E000C1FB00BF012105481DF0B0FB0028F9D0EB
:1092F00002481DF0B4FBC0B210BD000000300140B8
:1093000010B5012022F02CFA00201E4908800DE043
:109310001DF06EFA00F0800000B10BE0012022F099
:1093200067FC18480088401C1649088015480088CA
:10933000C828EDDB00BF13480088C8281CDA1021BC
:10934000114801F053FB08210F4801F051FB3D206B
:10935000FFF7BAFF2A20FFF7B7FF8020FFF7B4FF1F
:10936000A720FFF7B1FF1021074801F041FB0020C3
:1093700022F0F6F9012010BD002022F0F1F90020C2
:10938000F9E700002E0A00200000024070B50546F3
:109390000E460024012022F0E3F900202249088033
:1093A0000DE01DF025FA00F0800000B10BE0012077
:1093B00022F01EFC1C480088401C1B4908801A48EB
:1093C0000088C828EDDB00BF17480088C82825DAC8
:1093D0001021164801F00AFB0821144801F008FB8F
:1093E0008420FFF771FF0020FFF76EFF0020FFF7DA
:1093F0006BFF0020FFF768FF002404E0285DFFF703
:1094000063FF601C84B2B442F8DB1021074801F00E
:10941000EFFA002022F0A4F9012070BD002022F014
:109420009FF90020F9E700002E0A0020000002400A
:1094300070B506460C461546012022F091F92946E2
:109440003046FFF7A3FF08B9002070BD00201F4978
:1094500008800DE01DF0CCF900F0800000B10BE0B9
:10946000012022F0C5FB19480088401C17490880DC
:1094700016480088C828EDDB00BF14480088C828BB
:109480001EDA1021124801F0B1FA0821104801F04B
:10949000AFFA8320FFF718FFC4F38710FFF714FF1C
:1094A000A106080EFFF710FF0020FFF70DFF1021A7
:1094B000074801F09DFA002022F052F90120C4E78C
:1094C000002022F04DF90020BFE700002E0A002006
:1094D0000000024030B502460020002304E012F8EC
:1094E000014B60405C1CE3B28B42F8DB30BD0000F6
:1094F00010B50446392022F0C1FDE0B222F0DEFDB5
:10950000C4F3072022F0DAFDC4F3074022F0D6FDB1
:10951000200E22F0D3FD4FF48051034801F068FA89
:1095200020F02EFF10BD0000000402402DE9F041A4
:1095300007460E4614463A2022F0A0FDF0B222F073
:10954000BDFD301222F0BAFD4FF480510F4801F0FA
:109550004FFA19E020F014FF05461D2D11D13846B1
:1095600000F0ACF805463B2022F088FD4FF4805116
:10957000064801F03DFA2F4434B120882844208069
:1095800002E02846BDE8F081E4E700000004024064
:109590002DE9F04107460E4614463C2022F06EFDB0
:1095A000F0B222F08BFD301222F088FD4FF4805192
:1095B000104801F01DFA0CB10020208019E020F0C5
:1095C000DFFE05461E2D11D1384600F02BF9054669
:1095D0003D2022F053FD4FF48051064801F008FA77
:1095E0002F4434B120882844208002E02846BDE87A
:1095F000F081E4E70004024010B51CF0F1FF08B16F
:1096000000F02EF8302000F0A9F810BD10B5044687
:109610002146362000F08EF810BD10B5044614B176
:10962000204600F0ABF8342000F098F810BD10B5DB
:109630000446204600F0A2F820785C2802D020786A
:109640002F2803D10021642000F008F9322000F017
:1096500085F810BD10B5682000F04CF810BD000072
:1096600010B5222022F00AFD22F0FDFC04464FF442
:109670008051024801F0BCF9204610BD00040240B0
:109680002DE9F04122F0EFFC044622F0ECFC054607
:1096900022F0E9FC064622F0E6FC07464FF4805132
:1096A000054801F0A5F944EA052040EA064040EAF1
:1096B0000760BDE8F08100000004024070B5044678
:1096C000272022F0DBFC22F0CEFC0646054646B100
:1096D00000BF22F0C8FC2070641C701EC0B2061EC1
:1096E000F7D14FF48051024801F082F9284670BD4D
:1096F0000004024010B504460C2022F0BFFC2046B6
:1097000022F0DCFCFFF7BCFF10BD000070B5044682
:109710000A2022F0B3FC204622F0D0FC22F0A3FC69
:1097200005464FF48051024801F062F9284670BDA9
:109730000004024070B505460C46284622F09EFC07
:10974000204622F0BBFC4FF48051034801F050F951
:1097500020F016FE70BD00000004024010B5044663
:10976000204622F08BFC4FF48051034801F040F971
:1097700020F006FE10BD0000000402402DE9F0417B
:109780000646012022F07AFC22F06DFC43282BDAF9
:109790002B20FFF7BBFF102826DA2F2022F06EFCCB
:1097A000002022F08BFC3220FFF7D8FF0446142C57
:1097B0001AD1CF20FFF7AAFF0446ACB14C20FFF727
:1097C00099FF00EB042739464C2000F047F8502061
:1097D000FFF790FF00EB04273946502000F03EF8D9
:1097E0000021702000F03AF82F2022F047FC357855
:1097F000284622F063FC09E0761C35785C2D01D008
:109800002F2D00D10025284622F058FC002DF3D141
:109810004FF48051024801F0EBF8BDE8F081000000
:109820000004024070B504462D2022F027FC22F0EF
:109830001AFC0646054646B100BF207822F03EFCE1
:10984000641C701EC0B2061EF7D14FF4805102484E
:1098500001F0CEF8284670BD0004024070B5054600
:109860000C460D2022F00AFC284622F027FCE0B22C
:1098700022F024FCC4F3072022F020FCC4F30740AC
:1098800022F01CFC200E22F019FC4FF480510248FB
:1098900001F0AEF870BD00000004024070B5024651
:1098A0000C46FF25FF2309E012F8010B80EA0501B1
:1098B0000648405C80EA03050548435C201EA4F18D
:1098C0000106B4B2F0D145EA032070BD641A030862
:1098D000641B03082DE9F04103460C4600200146B5
:1098E000024606E013F8010B411842F10002601E27
:1098F00084B2002CF6DC080C40EA024C100C8DB24D
:109900001CEB050140F10002080C40EA024041183E
:109910006FEA010080B2BDE8F08130B50246002058
:10992000002305E012F8015B2C18E0B25C1CE3B2E6
:109930008B42F7DB30BD10B513F050FD10BD10B5F4
:1099400013F0EAFC10BD10B513F0B6FC10BD10B555
:1099500013F012FD10BD10B515F066FC10BD10B56A
:109960001CF034FA10BD00000246094B9A4201D2A5
:10997000084801E00648103801F000531BB1064BBF
:109980000B40C36002E0044B0B4083607047000053
:1099900010640240006002407D0F7D0F21B102681B
:1099A00042F00102026003E0026822F0010202605C
:1099B00070470000016821F0010101600021016091
:1099C00041608160C1600161212141614A49884251
:1099D00004D13D21484A103A91608CE04649183143
:1099E000884205D14FF47461434A103A916082E095
:1099F00041493031884205D14FF474113E4A103A42
:109A0000916078E03C494831884205D14FF074615B
:109A1000394A103A91606EE037496031884204D18A
:109A20003649354A103AD16065E033497831884289
:109A300004D13349304A103AD1605CE02E4990316C
:109A4000884204D12F492C4A103AD16053E02A4968
:109A5000A831884205D14FF03D51274A103AD160D4
:109A600049E02949884204D13D21274A083A11603A
:109A700041E025491831884205D14FF47461224AEA
:109A8000083A116037E020493031884205D14FF45F
:109A900074111D4A083A11602DE01B494831884273
:109AA00005D14FF07461184A083A116023E0164955
:109AB0006031884204D11149134A121F11601AE023
:109AC00011497831884204D10D490F4A121F1160A3
:109AD00011E00D499031884204D10A490A4A121F07
:109AE000116008E00849A831884204D14FF03D5187
:109AF000054A121F11607047106002403D000020AF
:109B0000400F002000003D201064024010B501F01D
:109B100080034BB122B1436943F08003436103E00A
:109B2000436923F08003436180290BD02AB1036885
:109B300001F01E042343036004E0036801F01E04E7
:109B4000A343036010BD000010B500220268134B50
:109B50001A40CC680B6823434C6923438C69234328
:109B6000CC6923430C6A23434C6A23438C6A234306
:109B70004C6B23438C6B23431A430260426922F0EF
:109B80000702D1E90B3423431A4342610B69436056
:109B90004B6883608B68C36010BD00003F801CF081
:109BA0001CB50024012120201CF026FD302000904F
:109BB00001208DF8040000208DF8060003208DF8A8
:109BC000050000208DF807006946164800F09AFE4F
:109BD0003021144800F00CFF0021134880F8401792
:109BE00000F5E860817001214170C1704FF4FA7195
:109BF000816000F01BF80C48007E592810DD2420FD
:109C0000094918314871082008713020C8701420A3
:109C100088702020487000210348017600F048F841
:109C20001CBD000000140240BC3200201CB522F014
:109C3000E7F8D02022F0B0F822F016F9002022F048
:109C4000ABF822F011F922F0DBF8D12022F0A4F8D1
:109C500022F00AF900240EE0062C05DA012022F099
:109C60006BF80DF8040004E0002022F065F80DF810
:109C70000400601CC4B2072CEEDB22F0DBF89DF878
:109C800006000A4948719DF8050008719DF8040016
:109C9000C8709DF8020088709DF8010048709DF81A
:109CA00000100248183801761CBD0000D432002094
:109CB0001CB500241D48007E8DF800001B4818309C
:109CC00040788DF801001948183080788DF802002E
:109CD00001208DF8030015481830C0788DF8040075
:109CE0001248183000798DF8050010481830407976
:109CF0008DF8060022F084F8D02022F04DF822F0F2
:109D0000B3F8002022F048F822F0AEF800BF07E0D8
:109D10001DF8040022F040F822F0A6F8601CC4B23E
:109D2000072CF5DB22F086F81CBD0000BC320020B9
:109D300070B502460C460025002309E012F8010B1D
:109D400080EA05010648405C80EA03050548435C5B
:109D5000201EA4F10106B4B2F0D145EA032070BD83
:109D6000641A0308641B030810B504460B4600215F
:109D7000072A00DD072244EA042001462BB901FA34
:109D800002F081B20912084610BD012B02D1114127
:109D9000C8B2F9E700BFF7E7704710B504460B46B5
:109DA0000021072A00DD072244EA0420014613B9F6
:109DB0001141C8B210BD012B05D101FA02F081B2E8
:109DC00009120846F6E700BFF4E70000F0B5ADF26F
:109DD0001C5D04460D460020CDF81805CDF814058D
:109DE000002604EB4400584901EBC000408AA84219
:109DF00003DC00200DF21C5DF0BD0020CDF8140541
:109E00009AE051480122C168504800F097FA4E4844
:109E1000406800788DF800009DF8000038287DD15A
:109E200004EB4400484B03EBC000C06804EB440360
:109E3000454F07EBC3031B8A03FB050104EB4400FA
:109E40003B4603EBC000028A404800F077FA00204E
:109E5000CDF8180512E004EB44003B4901EBC000CB
:109E60004068BDF81815405CBDF818250DF80200D3
:109E7000BDF81805401C80B2CDF8180504EB44006D
:109E8000314901EBC000008ABDF818158842E2DCB8
:109E900004EB44002C4A02EBC000008A401E81B251
:109EA000684600F011FB064604EB4400264901EB2E
:109EB000C000008A401E1DF80000B04233D10020CF
:109EC000CDF8180520E004EB44001F4901EBC00069
:109ED0004068BDF81815415C04EB44001A4A02EBD7
:109EE000C0008068BDF81825024404EB4400164BFE
:109EF00003EBC000008A401E68431154BDF81805EA
:109F0000401C80B2CDF8180504EB44000E4901EB6B
:109F1000C000008A401EBDF8181500E003E088422A
:109F2000D1DC012066E7642021F062FEBDF8140553
:109F3000401C80B2CDF81405BDF814050628FFF6C4
:109F400060AF002056E7000094CB02081C6E002092
:109F50002DE9F041ADF5A36D04460E46002500271E
:109F6000A8460020009004EB4400474901EBC000E4
:109F7000408AB04204DC00200DF5A36DBDE8F081FD
:109F800000210846FFF722FF01287AD1002520E0B2
:109F900004EB44003C4901EBC0008068411904EB2C
:109FA0004400394A02EBC000008A401E7043085C3E
:109FB00004EB440102EBC1014968485504EB44003D
:109FC000114601EBC0004068405D01A94855681C7E
:109FD00085B204EB44002C4901EBC000008AA84282
:109FE000D6DC00274BE004EB4400274B03EBC0001A
:109FF000C06804EB4403DFF890C00CEBC3031B8A7A
:10A0000003FB060104EB4400634603EBC000008A37
:10A01000401E82B21D4800F013FA04EB44001A4AB5
:10A0200002EBC000008A401E81B201A800F04CFA89
:10A03000009004EB4400144A02EBC000C06804EB3B
:10A040004402114B03EBC202128A104404EB440297
:10A0500003EBC202128A02FB0600411E012268467F
:10A0600000F0EEF931462046FFF7B0FE012801D19D
:10A0700082E706E0642021F0BBFD781C87B2062F42
:10A08000B1DB002078E7000094CB02081C6E0020B2
:10A0900070B5ADF5A36D0025002400200090464961
:10A0A000088080E000256FE0002414E0424800882A
:10A0B00000EB4000414951F83000005D3E490988FD
:10A0C00001EB41013D4A02EBC1014968085501A974
:10A0D0000855601C84B23848008800EB40003749BE
:10A0E00001EBC000008A401EA042DFDC324800883D
:10A0F00000EB40000A4602EBC000008A401E81B21D
:10A1000001A800F0E1F900902B48008800EB400026
:10A110002A4B03EBC000C068274B1B8803EB4303AB
:10A12000264E06EBC3031B8A03FB05012248008869
:10A1300000EB4000334603EBC000008A401E82B2B1
:10A140001F4800F07DF91C48008800EB40003246B3
:10A1500002EBC000C068184A128802EB4202334684
:10A1600003EBC202128A1044134A128802EB420225
:10A1700003EBC202128A02FB0500411E012268465F
:10A1800000F05EF9681C85B20B48008800EB4000C7
:10A190000A4901EBC000408AA84285DC06480088D5
:10A1A000401C05490880044800880D28FFF67AAF56
:10A1B0000DF5A36D70BD00001000002094CB0208C7
:10A1C0001C6E00201CB5012108461CF015FA012068
:10A1D0008DF8040002208DF8050000208DF806009F
:10A1E00001208DF80700182000906946144800F0FF
:10A1F00089FB05221146124800F0CCFB05220621FE
:10A200000F4800F0C7FB052207210D4800F0C2FBF4
:10A21000A020009002208DF8040003208DF8050096
:10A2200000208DF806008DF807006946044800F00C
:10A2300069FB402000906946014800F063FB1CBDAB
:10A24000000002402DE9F84300240027A04600202A
:10A2500000900025FFF7B6FF00F0C2F800BF00E055
:10A260006D1C30488542FBD36E4608212E4800F015
:10A27000BDFB10212C4800F0BBFB062000F094F839
:10A280000821294800F0B4FB0821274800F0AEFB64
:10A290001021254800F0ACFB012000F085F80020DB
:10A2A00000F082F80821204800F0A2FB1F48D0F8F7
:10A2B0002C11B0F83021B0F8320102FB0010B0F5DB
:10A2C000003F02D900BE00BFFEE71948006808B988
:10A2D000FFF7DEFE00201749088017E0002406E0A3
:10A2E000144908782146FFF771FD601C84B21148BB
:10A2F000008800EB40000D4901EBC000408AA042FD
:10A30000EEDC0C480088401C0A4908800948008897
:10A310000D28E3DB0848D0F8140207490871BDE8AE
:10A32000F8830000FFFF0F000000024094CB0208FA
:10A330001C02434210000020BC1200202DE9F04115
:10A3400005460C4616460027012021F006FA082192
:10A35000144800F04BFB1021124800F049FB032089
:10A3600000F022F8C4F3074000F01EF8C4F3072001
:10A3700000F01AF8E0B200F017F800BF06E0002085
:10A3800000F012F828706D1C781C87B2B742F6DB1B
:10A390000821044800F02CFB002021F0DEF9BDE884
:10A3A000F08100000000024010B5044600BF022109
:10A3B0000A481CF04BFB0028F9D0214607481CF046
:10A3C00051FB00BF012105481CF040FB0028F9D0DB
:10A3D00002481CF044FBC0B210BD00000030014038
:10A3E00000B585B0012108031CF056F913481CF094
:10A3F00001FB0020ADF80000ADF80400ADF8060048
:10A40000ADF808004FF40070ADF80A000820ADF870
:10A410000C000020ADF80E000720ADF810004FF43E
:10A420008270ADF80200694604481CF01DFB012152
:10A4300002481CF0D3FA05B000BD00000030014016
:10A440002DE9F04105460C4616460027012021F073
:10A4500084F908211B4800F0C9FA1021194800F0BE
:10A46000C7FA0620FFF7A0FF0821164800F0C0FA3F
:10A470000821144800F0BAFA1021124800F0B8FA86
:10A480000220FFF791FFC4F30740FFF78DFFC4F3ED
:10A490000720FFF789FFE0B2FFF786FF00BF05E066
:10A4A0002878FFF781FF6D1C781C87B2B742F7DB75
:10A4B0000821044800F09CFA002021F04EF9BDE884
:10A4C000F08100000000024010B50246107803E061
:10A4D00012F8014B2318D8B20B1EA1F10104A1B24E
:10A4E000F6D110BD2C48807C012854D100212A4887
:10A4F00081742A480078C0B901202849087028488A
:10A500000068C0002749D1F8301240EA810025498F
:10A51000D1F82C1240EA41002249D1F82812084310
:10A520000F2181432048017017E000201B4908706B
:10A530001B480068C0001B49D1F8301240EA810076
:10A540001849D1F82C1240EA41001649D1F82812D6
:10A5500008430F21814315480170134800781349BF
:10A560000978884217D110480078114908700846C8
:10A5700000781049097888420DD00D4800780649C6
:10A5800088730B4800780B4908700948007810B1AF
:10A590000120014948737047BC120020DE0A0020E8
:10A5A0003402424200004242DF0A0020E00A00205A
:10A5B000E10A0020DD0A002010B5ADF57C7D002405
:10A5C0007CA00068FB9000200090FFF715F814288D
:10A5D0007CD17948FFF72BF8784908700846007855
:10A5E000142874D1FFF736F80021754A03C2BDF86C
:10A5F0000000FEF77DFF6A464FF4FA7101A8FEF7EE
:10A6000095FF70A101A821F0D5FC7049088008468B
:10A61000008810B300BF04E000216D480155601CA4
:10A6200084B2282CF8DB01A9684A1288881869A12D
:10A6300021F0C0FC68490880002409E063480088D4
:10A64000C01C204401A9095C61480155601C84B20A
:10A6500061480088001FA042F0DC60A101A821F041
:10A66000A9FC5A4908800846008820B3002405E068
:10A670000021574828300155601C84B2282CF7DB94
:10A6800001A9524A1288881852A121F093FC52491C
:10A69000088000240AE04D4800880830204401A9C1
:10A6A000095C4B4828300155601C84B24A48008838
:10A6B0000938A042EFDC4CA101A821F07BFC434902
:10A6C00008800846008830B3002407E06BE05BE0B8
:10A6D00000213F4850300155601C84B2142CF7DB38
:10A6E00001A93A4A128888183AA121F063FC3A4934
:10A6F000088000240AE0354800880C30204401A975
:10A70000095C334850300155601C84B232480088DF
:10A710000D38A042EFDC38A101A821F04BFC2B49F9
:10A7200008800846008820B3002405E0002028495E
:10A7300046390855601C84B2322CF7DB01A9234A44
:10A740001288881823A121F035FC234908800024B1
:10A750000AE01E480088801D204401A9085C1C49AD
:10A7600046390855601C84B21B480088C01FA042AF
:10A77000EFDC00210320FFF7EBFB0120FEF746FF93
:10A7800001200DF57C7D10BD0C480078422803D1D6
:10A790000948FEF742FF0BE00120FEF737FF0020DB
:10A7A0000649087004E000211548C17521F092FBAC
:10A7B00000BFE6E70D0A0000480A0020380A002022
:10A7C000400A002041504E3D000000005E0A00207B
:10A7D000CC3A00203B0000005C0A00205749464963
:10A7E0004E414D453D0000005749464950415353A5
:10A7F000574F52443D0000005345525645523D00CC
:10A80000BC32002010B504463548844208D10121ED
:10A8100008461BF001FF002101201BF0FDFE5EE059
:10A820003048844208D1012102201BF0F5FE0021AE
:10A8300002201BF0F1FE52E02B48844208D1012196
:10A8400004201BF0E9FE002104201BF0E5FE46E099
:10A850002648844208D1012108201BF0DDFE00219A
:10A8600008201BF0D9FE3AE02148844208D101219A
:10A8700010201BF0D1FE002110201BF0CDFE2EE099
:10A880001C48844208D1012120201BF0C5FE002174
:10A8900020201BF0C1FE22E01748844208D101218C
:10A8A00040201BF0B9FE002140201BF0B5FE16E051
:10A8B0001248844208D1012180201BF0ADFE002106
:10A8C00080201BF0A9FE0AE00D48844207D1012137
:10A8D00080151BF0A1FE0021A0151BF09DFE10BDF0
:10A8E000000002400004024000080240000C024048
:10A8F000001002400014024000180240001C0240F8
:10A9000000200240F0B50A4600210023002400BFC9
:10A910003DE0012505FA01F3156805EA03049C42B0
:10A9200034D105684F000326BE40B5430560157954
:10A930004E00B5400668354305601579012D02D0FB
:10A940001579022D16D185684F000326BE40B54308
:10A95000856055794E00B540866835438560456809
:10A9600001268E40B5434560456896798E40B6B263
:10A9700035434560C5684F000326BE40B543C560FA
:10A98000D5794E00B540C6683543C560491C1029CD
:10A99000BFD3F0BDF0B5002300244D07ED0E02FA41
:10A9A00005F3CE1000F1200555F826504E07F70E9E
:10A9B0000F26BE40B543CF1000F1200646F82750C1
:10A9C000CE1000F1200555F8265045EA0304CE10BC
:10A9D00000F1200545F82640F0BD0246002013692D
:10A9E0000B400BB1012000E000207047418370470D
:10A9F000018370470249887B0021014A91737047A7
:10AA0000BC1200200E48006800F0010000B100BE3A
:10AA1000012080F3138800BF00BFBFF34F8F0848A9
:10AA2000E438006800F4E06006490843001D04496A
:10AA3000E4390860BFF34F8F00BF00BFFEE700009E
:10AA4000F0ED00E00000FA054AF6AA20014908608E
:10AA500070470000003000400021017041707047D5
:10AA600030B502460024002305E012F8015B2819E6
:10AA7000C4B2581CC3B28B42F7DB6042C0B230BDD7
:10AA800010B5002421F026FA642021F0B1F810BDA1
:10AA90002DE9F043ADF2DC7D80460E461446994622
:10AAA0000025002783A00068CDF8D807002001907A
:10AAB000042C7CDC80480079302101EB101004EB81
:10AAC000C40101EB04117D4A114408717A480079F0
:10AAD00000F00F00303004EBC40101EB041111440D
:10AAE00048717548C078302101EB101004EBC401A7
:10AAF00001EB0411114488716F48C07800F00F0019
:10AB0000303004EBC40101EB04111144C871FEF7AD
:10AB100073FD14287ED16A480078142809D004EB0C
:10AB2000C40101EB0411654A8818FEF780FD6449F1
:10AB300008706348007814286DD1B6F57A7F01DD7E
:10AB40004FF47A76FEF786FD00215E4A03C25D4827
:10AB50000068FEF7CDFC5848C078302101EB10109A
:10AB60008DF808005448C07800F00F0030308DF8A0
:10AB700009005148807801EB10108DF80A004E480A
:10AB8000807800F00F0030308DF80B004A48407894
:10AB900001EB10108DF80C004748407800F00F00D2
:10ABA00030308DF80D0044481838007E00E07CE01D
:10ABB00001EB10108DF80E003F481838007E00F0B1
:10ABC0000F0030308DF80F00B9F1000F03D1542081
:10ABD0008DF8100005E0B9F1010F02D152208DF877
:10ABE00010003A208DF8110000252CE0284605EBD6
:10ABF000D071491018F801100F110A2097FBF0F0DE
:10AC0000C0EBC00107F130000844C1B202AA05F14F
:10AC10000A0001E043E02EE01154284605EBD07114
:10AC2000491018F8011001F00F070A2097FBF0F007
:10AC3000C0EBC00107F130000844C1B205F10B00C0
:10AC40001154A81C85B2B5EB460FCFDB0A2000EBF0
:10AC5000460081B201AA02A8FEF79AFC01AA0221CD
:10AC60000DF5FB60FEF794FC0120FEF7CFFC002001
:10AC70001349087019E012480078422808D104EB03
:10AC8000C40101EB04110D4A8818FEF7C6FC0CE064
:10AC90000120FEF7BBFC00200949087005E00021F7
:10ACA00005481838C17521F015F90DF2DC7DBDE8B5
:10ACB000F08300000D0A0000D4320020600A00205A
:10ACC000380A0020400A002070B5B8B00021379142
:10ACD00036913591349133913291319130910022F6
:10ACE0002E922F922C922D922B912A91299128917C
:10ACF00027912691259124912391159114911391D7
:10AD00001291119110910F919FEDFE0A8DED0E0A97
:10AD1000FDA006C8CDE90C12FDA006C8CDE90A12B7
:10AD2000BAE0FD48807858B30020FB498870FB48A2
:10AD3000B0F80C0BFA490968C1F57A7188421FD145
:10AD4000F7480068C0F57A7081B2F448A0F8041B97
:10AD50000021F348001FFEF721FEF249F048001FD2
:10AD6000FEF702FE0120F04908704FF47A70EC49BA
:10AD70008C39C1F88C000121E948001FFEF70EFE56
:10AD8000E548807B50B30021E3488173E748408861
:10AD9000E3498C39496CC1F57A7188421ED1E0488B
:10ADA0008C38406CC0F57A70E04908394880002141
:10ADB000DB484C38FEF7F2FDDD49D9484C38FEF748
:10ADC000D3FD0120DB4908704FF47A70D4498C39E7
:10ADD00048640121D2484C38FEF7E0FDCE48807E21
:10ADE00050B30021CC488176D0488088CC498C393A
:10ADF0004969C1F57A7188421ED1C9488C384069C9
:10AE0000C0F57A70C949083988800021C4487C3867
:10AE1000FEF7C4FDC849C2487C38FEF7A5FD0120F5
:10AE2000C64908704FF47A70BD498C3948610121D8
:10AE3000BB487C38FEF7B2FDB74890F8260058B3FF
:10AE40000021B54880F82610B848C088B4498C392C
:10AE5000C96AC1F57A7188421ED1B1488C38C06A7E
:10AE6000C0F57A70B1490839C8800021AC4864380F
:10AE7000FEF794FDB249AA486438FEF775FD01203B
:10AE8000B04908704FF47A70A5498C39C862012125
:10AE9000A3486438FEF782FD9F488178807B014497
:10AEA0009D48807E01449C4890F826000844002874
:10AEB0007FF437AF0BF08EBB9B48007828B10020A1
:10AEC0009949087000212B9119E09A48007828B11F
:10AED00000209849087001212B9110E097480078D4
:10AEE00028B100209549087002212B9107E0954870
:10AEF000007820B100209349087003212B919DF820
:10AF0000AC1001EB4100C0EBC1108F4911F83000CB
:10AF1000C12836D19DF8AC1001EB4100C0EBC11047
:10AF2000894901EBC000807808282AD101217B489B
:10AF300080F85C1B9DF8AC0030B101280AD00228D3
:10AF40000ED0032818D111E04FF480417F48FFF75D
:10AF50004DFD11E04FF400517C48FFF747FD0BE039
:10AF60004FF480517948FFF741FD05E04FF400614F
:10AF70007648FFF73BFD00BF00BF00207449086022
:10AF800098E765480C389DF8AC1010F811000121C5
:10AF9000B1EBD01F4BF08C816E48C07DB8B16349D6
:10AFA00008399DF8AC0031F8101009919DF8AC00FB
:10AFB00000EB4001C1EBC010634901EBC00101236C
:10AFC00008919DF8AC20DDE90801FFF761FD9DF8CF
:10AFD000AC0000EB400101EB00105F4901EB0010F9
:10AFE00081792A919DF8A80009288BF01F81DFE85C
:10AFF00010F0765009008C145C23E92F1A322336A6
:10B000008D41794C9DF8AC1001EB4100C0EBC110B3
:10B010004D4901EBC000417808460991002112F02A
:10B0200069F8C1B22691002134911CE09DF8AC1062
:10B0300001EB410000EB0110474901EB00113031F9
:10B04000BDF8D00001EB001041789DF898008142D6
:10B0500004D1BDF8D000C1B2269112E0BDF8D000F5
:10B06000401C81B234919DF8AC1001EB410000EB23
:10B070000110394901EB0010C179BDF8D0008142BF
:10B08000D4DC00BF9DF8AC0000EB4001C1EBC01068
:10B090002D4901EBC000807800F0F000A0280DD110
:10B0A0009DF8AC0000EB4001C1EBC011264800EB5D
:10B0B000C100807800F00F0127910AE09DF8AC00F4
:10B0C00000EB4001C1EBC0101F4901EBC0008178CB
:10B0D0002791BDF89C0008B9102127919DF8AC106C
:10B0E00001EB4100C0EBC110174901EBC001BDF8F5
:10B0F0009C00401C095C2491BDF89C00401C81B25E
:10B1000009912BE00000000001693230313030003D
:10B110000169323045303000D43E0020BC6200204E
:10B120008C6002400088002012000020C86D0020C2
:10B130000080201013000020208000101400002048
:10B140000088001015000020347C00200018024008
:10B1500088024242BC320020004100209DF8AC1021
:10B1600001EB4100C0EBC110FE4901EBC0010891A9
:10B17000DDE9080112F04EFC35909DF8AC0000EBC3
:10B180004001C1EBC010F74901EBC001BDF89C00C4
:10B19000801C095CBDF8D400814242F0B4839DF864
:10B1A000AC0000EB4001C1EBC010EE4901EBC00068
:10B1B0004078002842F3A7839DF8AC0000EB4001E3
:10B1C000C1EBC010E74901EBC001BDF89C00C01CF9
:10B1D0000A5C9DF8AC0000EB8000E34901EB4021E4
:10B1E000C0319DF8980000EB800303EB401001EBA9
:10B1F000800080F83C200021DC4A9DF8AC0002EB86
:10B2000000129DF898001154D948007F012840D1C0
:10B210009DF8AC0000EB400101EB0010D54901EBBB
:10B22000001030309DF8981000EB0110801C099040
:10B23000007820F08000803009990870BDF89000F7
:10B24000B62814D0C52819D0D52802D0D9281CD1A9
:10B2500006E0BDF89C00032801DA0020249017E0E6
:10B26000BDF89C00032801DA0021249110E0BDF80C
:10B270009C00032801DA0020249009E0BDF89C001E
:10B28000032801DA0021249102E00021249100BF6B
:10B2900000BF9DF8AC1001EB410000EB0110B54977
:10B2A00001EB001030309DF8981000EB0110801C6D
:10B2B0000990007820F04000403009990870BDF8EE
:10B2C0009000C52801F02B8417DCB5287ED00DDC5A
:10B2D000112802F0B381122802F0F281132802F043
:10B2E0007B82B22842F00E8301F0E7BBB6286ED015
:10B2F000B9286DD0C328F5D1FDE3D92869D007DC82
:10B30000CA2867D0CE2802F0B480D528EAD109E057
:10B31000E12802F0C180E52802F0D180E728E1D1E0
:10B3200002F06BB99DF8AC1001EB4100C0EBC1100D
:10B330008C4901EBC000C1788F4880F80E1E9DF843
:10B34000AC0000EB8000884901EB4021C0319DF842
:10B35000980000EB800202EB401011F820109DF8DD
:10B36000AC0000EB8000804A02EB40200079814273
:10B370007EDA9DF8AC1001EB410000EB01107D4935
:10B3800001EB001030309DF8981000EB0110801C8C
:10B390000990794890F80E0E0121A1EBD01009997F
:10B3A000097860F3000109980170734890F80E0E57
:10B3B000C0F34010F0BB9DF8AC0000EB400101EB86
:10B3C00000106C4901EB0010303004E0FEE3FEE3B6
:10B3D000FEE3FEE3FEE39DF8981000EB0110807899
:10B3E000C0F3401030B39DF8AC0000EB400101EB1E
:10B3F0000010604901EB001030309DF8981000EB10
:10B400000110801C0990007820F00200801C09992E
:10B4100008709DF8AC0000EB8000114601EB402065
:10B42000C0309DF8981001EB810202EB411100EB56
:10B43000810000E00CE018300990007820F0020054
:10B44000801C099908709DF8AC100220FEF780FD61
:10B4500000219DF8AC0000EB8000434A02EB402045
:10B46000C17002229DF8AC0000EB80003E4900E074
:10B470001DE001EB4021C0319DF8980000EB8003F6
:10B4800003EB401001F82020B6229DF8AC0000EB41
:10B490008000354901EB4020C0309DF8981001EB49
:10B4A000810303EB411100EB81004271FEE332485E
:10B4B00090F80E0EC0F3C00090B9E5229DF8AC00E4
:10B4C00000EB8000284901EB4020C0309DF8981027
:10B4D00001EB810303EB411100EB81004271E5E3D5
:10B4E0009DF8AC1001EB410000EB0110214901EB8C
:10B4F000001030309DF8981000EB0110801C09906E
:10B500001D4890F80E1E0120A0EBD11009990A7871
:10B5100060F300020A709DF8AC0000EB400101EB03
:10B520000010144901EB001030309DF8981000EB2A
:10B530000110801C0990104890F80E0E42090998DD
:10B54000007862F34100099908709DF8AC1001EB96
:10B55000410000EB0110074901EB001030309DF86D
:10B5600098100BE0347C0020C0450020343F0020C0
:10B57000BC12002000410020BC22002000EB011082
:10B580008078C0F340029DF8AC0000EB8000FE49DB
:10B5900001EB4020C0309DF8981001EB810303EBD4
:10B5A000411100EB8100007EC0F34000824277D061
:10B5B0009DF8AC0000EB8000F34901EB4020C03067
:10B5C0009DF8981001EB810202EB411100EB810024
:10B5D000183009909DF8AC0000EB400101EB001021
:10B5E000EA4901EB001030309DF8981000EB011093
:10B5F000807842080998007862F341000999087040
:10B600009DF8AC0000EB400101EB0010DF4901EBBD
:10B61000001030309DF8981000EB01108078C0F3D6
:10B620004000E0B3D9229DF8AC0000EB8000D64981
:10B6300001EB4020C0309DF8981001EB810303EB33
:10B64000411100EB81004271D14890F88C0800282C
:10B650007BD19DF8AC0000EB8000CB4901EB402092
:10B66000C0309DF8981001EB810202EB411100EB14
:10B67000810090F87D00002867D011239DF8AC0070
:10B6800000EB8000C04901EB4021C0319DF89800DB
:10B6900000EB800202EB401001EB800001E055E07E
:10B6A00043E190F87E0000EB8000B74901EB4021B8
:10B6B000C0319DF8AC0000EB8000B34A02EB4022A1
:10B6C000C0329DF8980000EB800404EB401002EBC0
:10B6D000800090F87F0000EB800202EB401001EB4D
:10B6E000800080F87630F3239DF8AC0000EB8000FA
:10B6F000A54901EB4021C0319DF8980000EB800284
:10B7000002EB401001EB800090F87E0000EB80001F
:10B710009D4901EB4021C0319DF8AC0000EB800059
:10B72000994A02EB4020C0309DF8982002EB820439
:10B7300004EB421200EB820090F87F0000EB8002E5
:10B7400002EB401001EB80004371E9E001229DF81B
:10B75000AC0000EB80008C4901EB4021C0319DF82A
:10B76000980000EB800303EB401001EB8000427374
:10B77000D9229DF8AC0000EB8000834901EB402109
:10B78000C0319DF8980000EB800303EB401001EB03
:10B790008000427101229DF8AC0000EB80007A49E4
:10B7A00001EB4020C0309DF8981001EB810303EBC2
:10B7B000411100EB810080F83E20754890F88C081C
:10B7C000E8BB9DF8AC0000EB80006F4901EB402026
:10B7D000C0309DF8981001EB810202EB411100EBA3
:10B7E000810090F87D0050B39DF8AC0000EB800024
:10B7F000654901EB4021C0319DF8980000EB8002C3
:10B8000002EB401001EB800090F87E1001EB41004C
:10B8100000EB01105D4901EB001130319DF8AC00E7
:10B8200000EB8000584A02EB4022C0329DF898009D
:10B8300000EB800303EB401002EB800000E06FE0C0
:10B8400090F87F0001EB0010801C0990007820F038
:10B8500004020998027000239DF8AC0000EB800000
:10B86000494901EB4020C0309DF8981001EB81025E
:10B8700002EB411100EB810090F87E0000EB8000AC
:10B88000414901EB4020C0309DF8AC1001EB810133
:10B890003D4A02EB4122C0329DF8981001EB810431
:10B8A00004EB411102EB810191F87F1001EB810261
:10B8B00002EB411100EB810080F87630F3239DF814
:10B8C000AC0000EB8000304901EB4020C0309DF817
:10B8D000981001EB810202EB411100EB810090F81E
:10B8E0007E0000EB8000284901EB4020C0309DF82D
:10B8F000AC1001EB8101244A02EB4121C0319DF8DB
:10B90000982002EB820404EB421201EB820191F8D1
:10B910007F1001EB810202EB411100EB81004371CA
:10B920009DF8AC100220FEF713FB9DF8AC0000EB75
:10B93000400101EB0010154901EB001130319DF879
:10B94000980001EB0010807800F001029DF8AC0037
:10B9500000EB80000C4901EB4020C0309DF89810AE
:10B9600001EB810303EB411100EB8100007E00F04D
:10B97000010082427DD09DF8AC0000EB80000249BE
:10B9800001EB4020C03005E0C04500200041002010
:10B99000BC3200209DF8981001EB810202EB4111AE
:10B9A00000EB8100183009909DF8AC0000EB4001DD
:10B9B00001EB0010FE4901EB001030309DF89810AB
:10B9C00000EB0110807809990A7860F300020A7090
:10B9D0009DF8AC0000EB400101EB0010F44901EBD5
:10B9E000001030309DF8981000EB0110807800F0C6
:10B9F0000100E8BB9DF8AC0000EB400101EB00103A
:10BA0000EB4901EB001030309DF8981000EB01106D
:10BA10008078C0F3401068B39DF8AC0000EB800064
:10BA2000E44901EB4020C0309DF8981001EB810201
:10BA300002EB411100EB810090F83E00D0B99DF877
:10BA4000AC0000EB8000DB4901EB4020C0309DF8EA
:10BA5000981001EB810202EB411100EB8100407B69
:10BA600040B99DF8AC0000EB400101EB001002E092
:10BA70005BE02EE240E0CE4901EB001030309DF853
:10BA8000981000EB01108078C0F34000A0BB0122A9
:10BA90009DF8AC0000EB8000C64901EB4021C031AD
:10BAA0009DF8980000EB800303EB401001EB800051
:10BAB0004273D9229DF8AC0000EB8000BD4901EB38
:10BAC0004021C0319DF8980000EB800303EB40104B
:10BAD00001EB8000427101229DF8AC0000EB800078
:10BAE000B44901EB4020C0309DF8981001EB810370
:10BAF00003EB411101E0FCE303E000EB810080F87F
:10BB00003E2000229DF8AC0000EB8000A94901EB2B
:10BB10004020C0309DF8981001EB810303EB4111E8
:10BB200000EB810080F83D20CEE19DF8AC0000EBF9
:10BB30008000A04901EB4020C0309DF8981001EB37
:10BB4000810202EB411100EB810090F83E0098B9B0
:10BB500001229DF8AC0000EB8000964901EB4020EB
:10BB6000C0309DF8981001EB810303EB411100EB0D
:10BB7000810080F83D2027E000229DF8AC0000EB1A
:10BB800080008C4901EB4021C0319DF8980000EB0A
:10BB9000800303EB401001EB800080F83D209DF80E
:10BBA000AC1001EB410000EB0110814901EB0011E9
:10BBB00030319DF8980001EB0010801C099000784E
:10BBC00020F00102099802707B4804E0EFE3EFE304
:10BBD000EFE30EE3EEE390F88C0880B19DF8AC1033
:10BBE00001EB410000EB0110714901EB0010303016
:10BBF0009DF8981000EB0110807A022894D16F48CC
:10BC0000407F012890D16D48D0F814026B49C98B50
:10BC1000884289D29DF8AC0000EB8000654901EBB9
:10BC20004020C0309DF8981001EB810202EB4111D9
:10BC300000EB810090F83D00012838D19DF8AC0060
:10BC400000EB80005B4901EB4020C0309DF898106C
:10BC500001EB810202EB411100EB810090F87D00C5
:10BC600028BB9DF8AC0000EB400101EB00105049EF
:10BC700001EB001130319DF8980001EB00100178C4
:10BC80009DF8AC0000EB80004A4A02EB4020417076
:10BC9000C3229DF8AC0000EB8000464901EB402137
:10BCA000C0319DF8980000EB800301E07EE15CE08C
:10BCB00003EB401001EB8000427100229DF8AC00C4
:10BCC00000EB400101EB0010394901EB001130316C
:10BCD0009DF8980001EB001042609DF8AC10022026
:10BCE000FEF736F90021379119E000229DF8AC00EB
:10BCF00000EB80002F4901EB4021C0319DF89800F6
:10BD000000EB800303EB401001EB80013F31BDF8F5
:10BD1000DC000A54BDF8DC00401C81B23791BDF84C
:10BD2000DC000A28E1DB0020379019E000229DF8B2
:10BD3000AC0000EB80001F4901EB4021C0319DF8B1
:10BD4000980000EB800303EB401001EB80015B31B6
:10BD5000BDF8DC000A54BDF8DC00401C81B237910C
:10BD6000BDF8DC000F28E1DBAEE09DF8AC0000EB95
:10BD70008000104901EB4020C0309DF8981001EB85
:10BD8000810202EB411100EB810090F83D00012897
:10BD90007ED19DF8AC0000EB8000064901EB40210C
:10BDA000C0319DF8980000EB800202EB401007E0E4
:10BDB00000410020C0450020BC320020BC12002001
:10BDC00001EB800090F87E0000EB8000FE4901EB63
:10BDD0004021C0319DF8AC0000EB8000FA4A02EB34
:10BDE0004020C0309DF8982002EB820303EB421202
:10BDF00000EB820090F87F0000EB800202EB401025
:10BE000001EB800090F8760003285DD100239DF8B7
:10BE1000AC0000EB8000EC4901EB4021C0319DF803
:10BE2000980000EB800202EB401001EB800090F8DC
:10BE30007E0000EB8000E44901EB4021C0319DF819
:10BE4000AC0000EB8000E04A02EB4022C0329DF8DB
:10BE5000980000EB800404EB401002EB800090F8A7
:10BE60007F0000EB800202EB401001EB800080F8C5
:10BE700076309DF8AC0000EB400101EB0010D34997
:10BE800001EB001130319DF8980001EB001000E04B
:10BE90001AE001789DF8AC0000EB8000CA4A02EB82
:10BEA00040204170C3229DF8AC0000EB8000C649E1
:10BEB00001EB4020C0309DF8981001EB810303EBAB
:10BEC000411100EB810042719DF8AC100220FEF799
:10BED0003FF89DF8AC0000EB400101EB0010BB49BE
:10BEE00001EB001030309DF8981000EB01108078C5
:10BEF000C0F3400088B1D9229DF8AC0000EB80006F
:10BF0000B14901EB4020C0309DF8981001EB81034E
:10BF100003EB411100EB810042719DF8AC0000EB96
:10BF20008000A94901EB4020C0309DF8981001EB3A
:10BF3000810202EB411100EB81008078B22835D1FB
:10BF40009DF8AC0000EB400101EB00109F4901EBB4
:10BF5000001030309DF8981000EB01108078C0F38D
:10BF6000400018BB9DF8AC0000EB400101EB001055
:10BF7000964901EB001030309DF8981000EB01104D
:10BF80008078C0F3401088B9E5229DF8AC0000EB42
:10BF900080008D4901EB4020C0309DF8981001EBE6
:10BFA000810303EB411100EB810042719DF8AC006D
:10BFB00000EB400101EB0010844901EB0010303030
:10BFC0009DF8981000EB011080780121B1EBD01F93
:10BFD00075D19DF8AC0000EB400101EB00107B49EE
:10BFE00001EB001030309DF8981000EB01108078C4
:10BFF00000F00100002862D19DF8AC0000EB800049
:10C00000714901EB4020C0309DF8981001EB81028E
:10C0100002EB411100EB810090F83E0000284ED168
:10C020009DF8AC0000EB400101EB0010674901EB0B
:10C03000001030309DF8981000EB01108078C0F3AC
:10C04000C000E0BB9DF8AC0000EB400101EB00102C
:10C050005E4901EB001030309DF8981000EB0110A4
:10C06000407A00F0010050B39DF8AC0000EB800076
:10C07000554901EB4020C0309DF8981001EB81023A
:10C0800002EB411100EB810090F88E0000F00100FE
:10C09000A8B99DF8AC0000EB80004B4901EB4020B3
:10C0A000C0309DF8981001EB810202EB411100EBCA
:10C0B000810090F8800010B1002037902AE096E0CF
:10C0C0009DF8AC0000EB80003F4901EB4021C031FE
:10C0D0009DF8980000EB800202EB401001EB80001D
:10C0E00000F18101BDF8DC000A5C9DF8AC0000EBBA
:10C0F000400101EB0010354901EB00100E30BDF896
:10C10000DC10405C824200D008E0BDF8DC00401C3E
:10C1100081B23791BDF8DC000628D1DB00BFBDF845
:10C12000DC00062863D1379029E09DF8AC0000EBD5
:10C130008000254901EB4021C0319DF8980000EBBB
:10C14000800202EB401001EB800000F18101BDF89C
:10C15000DC000A5C9DF8AC0000EB400101EB001034
:10C160001A4901EB00100E30BDF8DC10405C824231
:10C1700000D008E0BDF8DC00401C81B23791BDF86A
:10C18000DC000A28D1DB00BFBDF8DC000A282ED075
:10C190009DF8AC0000EB80000B4901EB4020C03063
:10C1A0009DF8981001EB810202EB411100EB810038
:10C1B0008E300990007820F00100401C0999087029
:10C1C00012229DF8AC0003E0C04500200041002091
:10C1D00000EB8000FE4901EB4020C0309DF8981034
:10C1E00001EB810303EB411100EB8100427101F08F
:10C1F00089BB9DF8AC1001EB410000EB0110F54943
:10C2000001EB0010007BD0BBBDF89C00082800D0DB
:10C21000EDE70020379028E09DF8AC1001EB4100DD
:10C22000C0EBC110EC4901EBC001BDF8DC00C01C43
:10C23000085C00F00F00092800DD1AE09DF8AC1042
:10C2400001EB4100C0EBC110E34901EBC001BDF8B7
:10C25000DC00C01C085C00F0F000902800DD08E065
:10C26000BDF8DC00401C81B23791BDF8DC00062827
:10C27000D2DB00BFBDF8DC00062801DAB7E76AE0D0
:10C280009DF8AC1001EB4100C0EBC110D24901EBAD
:10C29000C000C07801049DF8AC0000EB4002C2EB86
:10C2A000C010CD4A02EBC000007941EA00219DF8A0
:10C2B000AC0000EB4002C2EBC010C74A02EBC0006A
:10C2C000407901439DF8AC0000EB8000C04A02EBCE
:10C2D0004022C0329DF8980000EB800303EB401031
:10C2E00002EB8000C0F81A109DF8AC1001EB410081
:10C2F00000E0A2E1C0EBC110B74901EBC0008079BA
:10C3000001049DF8AC0000EB4002C2EBC010B24A41
:10C3100002EBC000C07941EA00219DF8AC0000EBBF
:10C320004002C2EBC010AC4A02EBC000007A0143ED
:10C330009DF8AC0000EB8000A54A02EB4020C03025
:10C340009DF8982002EB820303EB421200EB82007F
:10C35000C0F81E10BEE0BDF89C000A2800D046E7D9
:10C36000002037902CE09DF8AC1001EB4100C0EBB1
:10C37000C110994901EBC001BDF8DC00C01C085C8C
:10C3800000F00F00092800DD1EE09DF8AC1001EB65
:10C390004100C0EBC110904901EBC001BDF8DC00C9
:10C3A000C01C085C00F0F000902804DD0CE08AE17D
:10C3B0005DE2F2E174E1BDF8DC00401C81B237912E
:10C3C000BDF8DC000828CEDB00BFBDF8DC00082883
:10C3D00000DA0CE79DF8AC1001EB4100C0EBC11096
:10C3E0007D4901EBC000C07801069DF8AC0000EB70
:10C3F0004002C2EBC010784A02EBC000007941EA6B
:10C4000000419DF8AC0000EB4002C2EBC010724A44
:10C4100002EBC000407941EA00219DF8AC0000EB3E
:10C420004002C2EBC0106C4A02EBC00080790143AD
:10C430009DF8AC0000EB8000654A02EB4022C03260
:10C440009DF8980000EB800303EB401002EB8000A6
:10C45000C0F81A109DF8AC1001EB4100C0EBC11000
:10C460005D4901EBC000C07901069DF8AC0000EB0E
:10C470004002C2EBC010584A02EBC000007A41EA09
:10C4800000419DF8AC0000EB4002C2EBC010524AE4
:10C4900002EBC000407A41EA00219DF8AC0000EBBD
:10C4A0004002C2EBC0104C4A02EBC000807A01434C
:10C4B0009DF8AC0000EB8000454A02EB4020C03004
:10C4C0009DF8982002EB820303EB421200EB8200FE
:10C4D000C0F81E109DF8AC0000EB80003C4901EB59
:10C4E0004021C0319DF8980000EB800202EB401023
:10C4F00011F820109DF8AC0000EB8000344A02EBEC
:10C500004020007981422BDA00219DF8AC0000EB3D
:10C51000800002EB4020C17004229DF8AC0000EBCB
:10C5200080002B4901EB4021C0319DF8980000EBC1
:10C53000800303EB401001F82020C5229DF8AC00D9
:10C5400000EB8000224901EB4020C0309DF898109C
:10C5500001EB810303EB411100EB810042716BE0C1
:10C560009DF8AC0000EB400101EB0010194901EB14
:10C57000001030309DF8981000EB01108078C0F367
:10C58000400090B1D5229DF8AC0000EB800010492E
:10C5900001EB4020C0309DF8981001EB810303EBC4
:10C5A000411100EB8100427146E09DF8AC0000EBC8
:10C5B0008000074901EB4020C0309DF8981001EB46
:10C5C000810202EB411100EB8100807B012805E034
:10C5D000C045002000410020347C00202CD10022E6
:10C5E0009DF8AC0000EB8000F74901EB4021C03121
:10C5F0009DF8980000EB800303EB401001EB8000F6
:10C600008273B6229DF8AC0000EB8000EE4901EB8E
:10C610004021C0319DF8980000EB800303EB4010EF
:10C6200001EB8000427100219DF8AC0000EB80001E
:10C63000E54A02EB4020C170D9E5D5229DF8AC0057
:10C6400000EB8000E04901EB4021C0319DF89800EB
:10C6500000EB800303EB401001EB800042710121ED
:10C660009DF8AC0000EB8000D74A02EB4020C1707F
:10C670009DF8AC0000EB400101EB0010A2F59861C1
:10C6800001EB001130319DF8980001EB0010801C87
:10C690000990007820F02000203009990870A6E564
:10C6A000D5229DF8AC0000EB8000C74901EB40208B
:10C6B000C0309DF8981001EB810303EB411100EBB2
:10C6C0008100427193E59DF8AC0000EB8000BE490B
:10C6D00001EB4020C030BDF8D01001EB810202EB2D
:10C6E000411100EB8100807901283AD100229DF8A8
:10C6F000AC0000EB8000B44901EB4021C031BDF833
:10C70000D00000EB800303EB401001EB800082714E
:10C71000D5229DF8AC0000EB8000AB4901EB402135
:10C72000C0319DF8980000EB800303EB401001EB53
:10C73000800042719DF8AC1001EB410000EB01104C
:10C74000A24901EB001130319DF8980001EB001077
:10C75000801C0990007820F00400001D09990870E1
:10C760001AE0C3229DF8AC0000EB8000964901EB73
:10C770004021C0319DF8980000EB800303EB40108E
:10C7800001EB8000427100219DF8AC0000EB8000BD
:10C790008D4A02EB4020C17029E59DF8AC0000EB0A
:10C7A0008000894901EB4020C030BDF8D01001EB7A
:10C7B000810202EB411100EB8100807901283AD11E
:10C7C00000229DF8AC0000EB80007F4901EB402186
:10C7D000C031BDF8D00000EB800303EB401001EB4B
:10C7E00080008271D5229DF8AC0000EB8000764974
:10C7F00001EB4021C0319DF8980000EB800303EB72
:10C80000401001EB800042719DF8AC1001EB41003B
:10C8100000EB01106D4901EB001130319DF89800DB
:10C8200001EB0010801C0990007820F00400001D2E
:10C83000099908701AE0C3229DF8AC0000EB800053
:10C84000614901EB4021C0319DF8980000EB800365
:10C8500003EB401001EB8000427100219DF8AC0019
:10C8600000EB8000584A02EB4020C170BFE49DF805
:10C87000AC1001EB410000EB0110544901EB00103A
:10C88000007B38BB9DF8AC1001EB4100C0EBC11040
:10C890004F4901EBC00001799DF8AC0000EB40026C
:10C8A000C2EBC0104A4A02EBC000C07841EA002245
:10C8B0009DF8AC0000EB8000434901EB4020C03004
:10C8C0009DF8981001EB810303EB411100EB81000F
:10C8D000426332E09DF8AC1001EB4100C0EBC110A7
:10C8E0003B4901EBC000C07801049DF8AC0000EBAF
:10C8F0004002C2EBC010364A02EBC000007941EAA8
:10C9000000219DF8AC0000EB4002C2EBC010304AA1
:10C9100002EBC000407901439DF8AC0000EB8000C1
:10C92000294A02EB4020C0309DF8982002EB820398
:10C9300003EB421200EB820041639DF8AC0000EB78
:10C940008000214901EB4021C0319DF8980000EBA7
:10C95000800202EB401011F820109DF8AC0000EBB3
:10C960008000194A02EB40200079814232DA00212E
:10C970009DF8AC0000EB800002EB4020C170032268
:10C980009DF8AC0000EB80000F4901EB4021C03165
:10C990009DF8980000EB800303EB401001F8202085
:10C9A000D9229DF8AC0000EB8000074901EB402044
:10C9B000C0309DF8981001EB810303EB411100EBAF
:10C9C0008100427178E00000C04500200041002055
:10C9D000347C00209DF8AC0000EB8000FE4901EBA8
:10C9E0004020C030BDF8D01001EB810202EB4111B4
:10C9F00000EB81008079012843D100229DF8AC0032
:10CA000000EB8000F44901EB4021C031BDF8D000BB
:10CA100000EB800303EB401001EB80008271D92210
:10CA20009DF8AC0000EB8000EB4901EB4021C031E8
:10CA30009DF8980000EB800303EB401001EB8000B1
:10CA400042719DF8AC1001EB410000EB0110E3498D
:10CA500001EB001130319DF8980001EB0010801CB3
:10CA60000990007820F00400001D09990870012049
:10CA70009DF8AC1001EB8101D74A02EB4121C8704F
:10CA80001AE0C5229DF8AC0000EB8000D24901EB12
:10CA90004021C0319DF8980000EB800303EB40106B
:10CAA00001EB8000427100219DF8AC0000EB80009A
:10CAB000C94A02EB4020C17051E400219DF8AC004E
:10CAC00000EB8000C44A02EB4020C1709DF8AC002E
:10CAD00000EB400101EB0010C04901EB00113031C7
:10CAE0009DF8980001EB0010801C0990007820F060
:10CAF0000400001D09990870D5229DF8AC0000EBD8
:10CB00008000B54901EB4020C0309DF8981001EB42
:10CB1000810303EB411100EB810042711FE49DF89A
:10CB2000AC0000EB400101EB0010AC4901EB001040
:10CB3000007BD0BBBDF89C000C2800D00FE4002087
:10CB4000379028E09DF8AC0000EB4001C1EBC0102D
:10CB5000A34901EBC001BDF8DC00C01C085C00F07B
:10CB60000F00092800DD1AE09DF8AC0000EB400141
:10CB7000C1EBC0119A4800EBC101BDF8DC00C01C3C
:10CB8000085C00F0F000902800DD08E0BDF8DC0053
:10CB9000401C81B23791BDF8DC000A28D2DB00BF0F
:10CBA000BDF8DC000A2801DA13E47CE000202C90B8
:10CBB0002D90002137911EE0DDE92C10000240EAA3
:10CBC00011620902CDE92C129DF8AC0000EB400186
:10CBD000C1EBC011824800EBC101BDF8DC00C01CF4
:10CBE000085CDDE92C241043CDE92C04BDF8DC0001
:10CBF000401C80B23790BDF8DC000528DCDB9DF8D6
:10CC0000AC00DDE92C1200EB8000734B03EB4023FA
:10CC1000C0339DF8980000EB800404EB401003EB58
:10CC2000800040F8221F426000222C922D920021A9
:10CC300037911EE0DDE92C10000240EA1162090282
:10CC4000CDE92C129DF8AC0000EB4001C1EBC01007
:10CC5000634901EBC001BDF8DC000830085CDDE988
:10CC60002C241043CDE92C04BDF8DC00401C80B21C
:10CC70003790BDF8DC000528DCDB9DF8AC00DDE971
:10CC80002C1200EB8000544B03EB4020C0309DF889
:10CC9000983003EB830404EB431300EB8300223052
:10CCA0008160C260BEE0BDF89C000E2800D0C3E4E5
:10CCB0000020379028E09DF8AC0000EB4001C1EB6C
:10CCC000C010474901EBC001BDF8DC00C01C085C86
:10CCD00000F00F00092800DD1AE09DF8AC1001EB10
:10CCE0004100C0EBC1103E4901EBC001BDF8DC00C2
:10CCF000C01C085C00F0F000902800DD08E0BDF8E2
:10CD0000DC00401C81B23791BDF8DC000C28D2DB7E
:10CD100000BFBDF8DC000C2800DA8DE400202C9068
:10CD20002D90002137911EE0DDE92C10000240EA31
:10CD300011620902CDE92C129DF8AC1001EB410003
:10CD4000C0EBC110264901EBC001BDF8DC00C01CDE
:10CD5000085CDDE92C341843CDE92C04BDF8DC0077
:10CD6000401C80B23790BDF8DC000628DCDB9DF863
:10CD7000AC00DDE92C1200EB8000174B03EB4023E5
:10CD8000C0339DF8980000EB800404EB401003EBE7
:10CD9000800040F8221F426000222C922D92002138
:10CDA000379126E0DDE92C10000240EA1162090209
:10CDB000CDE92C129DF8AC1001EB4100C0EBC11085
:10CDC000074901EBC001BDF8DC000930085CDDE972
:10CDD0002C34184306E00000C0450020004100202C
:10CDE000347C0020CDE92C04BDF8DC00401C80B26E
:10CDF0003790BDF8DC000628D4DB9DF8AC00DDE9F7
:10CE00002C1200EB8000FE4B03EB4020C0309DF85D
:10CE1000983003EB830404EB431300EB83002230D0
:10CE20008160C2609DF8AC0000EB8000F44901EB2A
:10CE30004021C0319DF8980000EB800202EB4010C9
:10CE400011F820109DF8AC0000EB8000EC4A02EBDA
:10CE50004020007981427CD1EA4890F88C0888B162
:10CE60009DF8AC1001EB410000EB0110A2F59861B8
:10CE700001EB001030309DF8981000EB0110807A23
:10CE8000022867D1E048D0F814020521B0FBF1F286
:10CE900001FB120101EBC10000EB0111DA48203067
:10CEA00000EB81000021C0F81D10D748D0F8140213
:10CEB0000521B0FBF1F201FB120101EBC10000EB17
:10CEC0000111D148203000EB81000D3009909DF810
:10CED000AC0000EB8000CA4901EB4021C0319DF855
:10CEE000980000EB800202EB401001EB8000223042
:10CEF0001022014608900998FBF7A7F9C248D0F81C
:10CF000014020521B0FBF1F201FB120101EBC1009B
:10CF100000EB0111BC48203000EB81029DF8AC0011
:10CF200000EB8000B64901EB4021C0319DF898002C
:10CF300000EB800303EB401001EB800050F81A1F58
:10CF400042F8011F40685060AF48D0F81402052134
:10CF500001E02FE201E1B0FBF1F201FB120000EB76
:10CF6000C00101EB0013A84920319DF8AC0000EB93
:10CF7000400202EB0010A54A02EB001230329DF88D
:10CF8000980002EB0010007801F823009E48D0F8CA
:10CF900014020521B0FBF1F201FB120000EBC0010D
:10CFA00001EB00119848203000EB8101954882691F
:10CFB00041F8212F808B88809348D0F814020521F6
:10CFC000B0FBF1F201FB120000EBC00101EB00111C
:10CFD0008D48203000EB81029DF8AC0000EB800012
:10CFE000874901EB4021C0319DF8980000EB800398
:10CFF00003EB401001EB8000406BC2F8090082484F
:10D00000D0F814020521B0FBF1F201FB120000EB95
:10D01000C00101EB00117C48203000EB81029DF83B
:10D02000AC0000EB400101EB0010784901EB00116E
:10D0300030319DF8980001EB00104068C2F82700DD
:10D04000002137914CE07048D0F814020521B0FB64
:10D05000F1F201FB120000EBC00101EB00116A4884
:10D06000203000EB81012B31BDF8DC409DF8AC0095
:10D0700000EB8000624A02EB4022C0329DF898002B
:10D0800000EB800303EB401002EB800090F87E0081
:10D0900000EB80005A4A02EB4022C0329DF8AC00FF
:10D0A00000EB8000564B03EB4023C0339DF8980003
:10D0B00000EB800505EB401003EB800090F87F004B
:10D0C00000EB800303EB401002EB80023F32BDF81F
:10D0D000DC00105C0855BDF8DC00401C81B23791C3
:10D0E000BDF8DC000A28AEDB4748D0F81402052161
:10D0F000B0FBF1F080B2014609900220FBF7E8FF97
:10D1000000210620FCF724FF3F48D0F814023E49D6
:10D11000C98B884206D23C48D0F81402401C3A49D8
:10D12000C1F8140200210520FCF712FF9DF8AC00A5
:10D1300000EB400101EB0010344901EB00103030EE
:10D140009DF8981000EB0110801C0990007820F0E9
:10D150000400001D0999087015E09DF8AC0000EB73
:10D16000400101EB0010294901EB001030309DF81F
:10D17000981000EB0110801C0990007820F0080046
:10D180000830099908709DF8AC0000EB400101EBF4
:10D1900000101E4901EB001030309DF8981000EB94
:10D1A0000110801C0990007820F02002099802707C
:10D1B0009DF8AC100220FCF7CBFE9DF8AC009DF86A
:10D1C000981001EB0010C217CDE92C0200222C9818
:10D1D00000EBC00101EB00110D4800EB8100C0F82D
:10D1E0001D209DF8AC0000EB8000054901EB4020BC
:10D1F000C0309DF8981001EB810202EB411109E06B
:10D20000C0450020BC320020BC120020004100209C
:10D21000E014002000EB8100223009902C9800EBF4
:10D22000C00101EB0011FE4800EB81010D3110221D
:10D230000891DDE90801FBF708F89DF8AC0000EB68
:10D240008000F84901EB4021C0319DF8980000EBC7
:10D25000800202EB401001EB80012C9800EBC00231
:10D2600002EB0012EE4800EB820051F81A2F40F852
:10D27000012F496841609DF8AC0000EB400101EBD3
:10D280000010E94901EB001130319DF8980001EBE5
:10D29000001001782C9800EBC00202EB0012E0486D
:10D2A00000F822102C9800EBC00101EB0011DC48C3
:10D2B00000EB8101DD48826941F8212F808B888055
:10D2C0009DF8AC0000EB8000D64901EB4021C03155
:10D2D0009DF8980000EB800202EB401001EB80000B
:10D2E000416B2C9800EBC00202EB0012CC4800EB23
:10D2F0008200C0F809109DF8AC0000EB400101EB82
:10D300000010C94901EB001130319DF8980001EB84
:10D31000001041682C9800EBC00202EB0012C048DC
:10D3200000EB8200C0F827100021379124E09DF81F
:10D33000AC0000EB8000BB4901EB4021C0319DF8FF
:10D34000980000EB800202EB401001EB80013F31BE
:10D35000BDF8DC000A5C2C9800EBC00101EB001169
:10D36000AF4800EB81012B31BDF8DC000A54BDF859
:10D37000DC00401C81B23791BDF8DC000A28D6DB06
:10D380002C9881B208200991FCF7E2FD00229DF85B
:10D39000AC0000EB8000A34901EB4020C0309DF8B9
:10D3A000981001EB810303EB411100EB810080F841
:10D3B0003E204BE09DF8AC0000EB400101EB00107B
:10D3C000994901EB001030309DF8981000EB0110E6
:10D3D000801C0990007820F00400001D0999087055
:10D3E0009DF8AC0000EB400101EB00108E4901EB11
:10D3F000001030309DF8981000EB0110801C09904F
:10D40000007820F0800080300999087001209DF894
:10D41000AC1001EB8101834A02EB4121C8709DF8F9
:10D42000AC0000EB8000114601EB402002799DF832
:10D43000AC0000EB800001EB4020C0309DF898105C
:10D4400001EB810303EB411100F82120D5229DF867
:10D45000AC0000EB8000734901EB4020C0309DF828
:10D46000981001EB810303EB411100EB8100427145
:10D4700048E2D5229DF8AC0000EB8000694901EB41
:10D480004020C0309DF8981001EB810303EB41115F
:10D4900000EB8100427135E2D5229DF8AC0000EB33
:10D4A0008000604901EB4020C0309DF8981001EBEE
:10D4B000810303EB411100EB8100427122E2012163
:10D4C0005A4880F8B0179DF8AC0000EB8000554931
:10D4D00001EB4021C0319DF8980000EB800202EB87
:10D4E000401011F820109DF8AC0000EB80004D4A70
:10D4F00002EB4020007981422BDA00219DF8AC003C
:10D5000000EB800002EB4020C17001229DF8AC00CE
:10D5100000EB8000434901EB4021C0319DF89800A9
:10D5200000EB800303EB401001F8202011229DF84E
:10D53000AC0000EB80003B4901EB4020C0309DF87F
:10D54000981001EB810303EB411100EB8100427164
:10D5500052E09DF8AC0000EB8000324901EB402026
:10D56000C0309DF8981001EB810202EB411100EBF5
:10D5700081008078B2282DD100219DF8AC0000EB0D
:10D580008000284A02EB4020C170B2229DF8AC0016
:10D5900000EB8000234901EB4021C0319DF8980049
:10D5A00000EB800303EB401001EB8000427100228E
:10D5B0009DF8AC0000EB80001A4901EB4020C03020
:10D5C0009DF8981001EB810303EB411100EB810002
:10D5D000827011E0D5229DF8AC0000EB800011496B
:10D5E00001EB4020C0309DF8981001EB810303EB64
:10D5F000411100EB8100427184E100210B4880F869
:10D60000B017D5229DF8AC0000EB8000054901EB76
:10D610004020C0309DF8981001EB810308E0000025
:10D62000E0140020C045002000410020BC32002052
:10D6300003EB411100EB8100427163E101229DF88F
:10D64000AC0000EB8000FE4901EB4021C0319DF8A9
:10D65000980000EB800303EB401001EB800080F8A2
:10D6600080200021379126E09DF8AC1001EB4100AD
:10D67000C0EBC110F34901EBC001BDF8DC00C01CD8
:10D680000A5C9DF8AC0000EB8000ED4901EB402105
:10D69000C0319DF8980000EB800303EB401001EBD4
:10D6A000800000F18101BDF8DC000A54BDF8DC0007
:10D6B000401C81B23791BDF8DC000A28D4DB21E19F
:10D6C0009DF8AC1001EB4100C0EBC110DD4901EB4E
:10D6D000C000C07801049DF8AC0000EB4002C2EB32
:10D6E000C010D84A02EBC000007941EA00209DF842
:10D6F000AC1001EB4102C2EBC111D24A02EBC101F5
:10D7000049790843B0F5E13F65D19DF8AC1001EBD4
:10D71000410000EB0110CC4901EB001030309DF8C6
:10D72000981000EB0110801C0990007820F0040292
:10D730000998027000229DF8AC0000EB8000C049FF
:10D7400001EB4020C0309DF8981001EB810303EB02
:10D75000411100EB8100A0F88C2013229DF8AC0051
:10D7600000EB8000B64901EB4020C0309DF89810D6
:10D7700001EB810303EB411100EB810042719DF845
:10D78000AC1001EB410000EB0110AF4901EB0010C0
:10D79000407903464FF480524FF4E13109909DF8EF
:10D7A000AC0010F049F99DF8AC0000EB8000A449F2
:10D7B00001EB4021C0319DF8980000EB800202EBA4
:10D7C000401001EB80008E300990007820F00800B6
:10D7D00008300999087095E09DF8AC1001EB410004
:10D7E000C0EBC110974901EBC00001799DF8AC0076
:10D7F00000EB4002C2EBC010924A02EBC000C078BE
:10D8000041EA00229DF8AC0000EB80008C4901EB5E
:10D810004021C0319DF8980000EB800303EB4010DD
:10D8200001EB8000A0F88C209DF8AC0000EB80009C
:10D83000834901EB4021C0319DF8980000EB800244
:10D8400002EB401001EB8000B0F88C109DF8AC00AA
:10D8500000EB400202EB00107B4A02EB0010408B11
:10D8600081424EDBE5229DF8AC0000EB800074495C
:10D8700001EB4021C0319DF8980000EB800303EBE1
:10D88000401001EB8000427100229DF8AC0000EBDB
:10D8900080006B4901EB4021C0319DF8980000EBFE
:10D8A000800303EB401001F820209DF8AC1001EB41
:10D8B000410000EB0110644901EB001130319DF88B
:10D8C000980001EB0010801C0990007820F0800285
:10D8D000099802709DF8AC0000EB8000584901EBFC
:10D8E0004020C0309DF8981001EB810202EB4111FD
:10D8F00000EB81008E300990007820F00102099839
:10D90000027000BF00BF08F091BC9DF8AC1001EBA5
:10D910004100C0EBC1104B4911F83000042801D17F
:10D9200024900BE09DF8AC1001EB4100C0EBC1105E
:10D93000444911F83000152800D124909DF8AC100E
:10D9400001EB4100C0EBC1103E4901EBC000417842
:10D950009DF8AC0000EB4002C2EBC010394A12F84F
:10D96000300041EA002041F23001884202D1A62075
:10D9700024903DE09DF8AC1001EB4100C0EBC110DC
:10D98000304901EBC00041789DF8AC0000EB40024B
:10D99000C2EBC0102B4A12F8300041EA002041F2DD
:10D9A0003101884202D1A720249021E09DF8AC10DB
:10D9B00001EB4100C0EBC110224911F830000228F0
:10D9C00016D19DF8AC1001EB4100C0EBC1101D4910
:10D9D00001EBC00001799DF8AC0000EB4002C2EB06
:10D9E000C010184A02EBC000C07841EA002124911F
:10D9F0009DF8AC0000EB8000114901EB40208178DC
:10DA000026910021114A9DF8AC0002EB00129DF80E
:10DA1000980011540E48007F012820D19DF8AC10C9
:10DA200001EB410000EB0110074901EB0010303021
:10DA30009DF8981000EB0110801C0990007809E017
:10DA4000C0450020347C002000410020343F0020ED
:10DA5000BC12002020F080008030099908709DF8E9
:10DA6000AC1001EB410000EB0110FE4901EB00108E
:10DA700030309DF8981000EB0110801C0990007860
:10DA800020F04000403009990870BDF8901043F232
:10DA90003002881A91427DD009DC04297BD01529F7
:10DAA0007AD0A6290DD0A72941F0FC852CE1B0F54C
:10DAB000C06F72D0A0F2016000286FD00428F3D1AB
:10DAC000FEE300219DF8AC0000EB8000E64A02EB8B
:10DAD0004020C1709DF8AC0000EB8000114601EBC6
:10DAE0004020C0309DF8981001EB810202EB4111FB
:10DAF00010F82100032823DC04229DF8AC0000EB81
:10DB00008000D94901EB4021C0319DF8980000EB1D
:10DB1000800303EB401001F82020A8229DF8AC0000
:10DB200000EB8000D04901EB4020C0309DF89810F8
:10DB300001EB810303EB411100EB81004271E1E055
:10DB40009DF8AC0000EB8000C74901EB4020C030DD
:10DB50009DF8981001EB810202EB411110F82100B1
:10DB6000082829DC09229DF8AC0000EB8000BE49A2
:10DB700001EB4021C0319DF8980000EB800303EBDE
:10DB8000401001F82020A9229DF8AC0000EB800095
:10DB9000B54904E06AE1DBE1FDE3FDE3FDE301EB10
:10DBA0004021C0319DF8980000EB800303EB40104A
:10DBB00001EB80004271A5E09DF8AC0000EB800015
:10DBC000A94901EB4020C0309DF8981001EB81027B
:10DBD00002EB411110F821000D2823DC0E229DF8E4
:10DBE000AC0000EB8000A04901EB4021C0319DF862
:10DBF000980000EB800303EB401001F82020A222E4
:10DC00009DF8AC0000EB8000974901EB4020C0304C
:10DC10009DF8981001EB810303EB411100EB8100AB
:10DC200042716FE09DF8AC0000EB80008E4901EB83
:10DC30004020C0309DF8981001EB810202EB4111A9
:10DC400000EB81004079A52815D19DF8AC0000EBD0
:10DC5000400101EB0010834901EB001030309DF8CA
:10DC6000981000EB0110801C0990007820F004004F
:10DC7000001D099908709DF8AC0000EB80007A49FE
:10DC800001EB4020C0309DF8981001EB810202EBBF
:10DC9000411100EB81008078A12833D09DF8AC00C1
:10DCA00000EB8000704901EB4021C0319DF89800E5
:10DCB00000EB800202EB401001EB800082789DF8BF
:10DCC000AC0000EB8000684901EB4021C0319DF8B9
:10DCD000980000EB800303EB401001EB80004271E1
:10DCE000A1229DF8AC0000EB80005F4901EB4020D1
:10DCF000C0309DF8981001EB810303EB411100EB5C
:10DD00008100827001F0CEBC00219DF8AC0000EBD8
:10DD10008000554A02EB4020C1709DF8AC0000EB3A
:10DD20008000114601EB4020C0309DF8981001EBB7
:10DD3000810202EB411110F8210005281ADC0021B4
:10DD40009DF8AC0000EB8000474A02EB4020C17018
:10DD500006229DF8AC0000EB8000434901EB402017
:10DD6000C0309DF8981001EB810303EB411100F8DE
:10DD7000212022E09DF8AC0000EB80003A4901EB45
:10DD80004020C0309DF8981001EB810202EB411158
:10DD900010F82100092810DC0A229DF8AC0000EBE5
:10DDA0008000314901EB4020C0309DF8981001EB14
:10DDB000810303EB411100F821209DF8AC0000EB3A
:10DDC0008000294901EB4020C0309DF8981001EBFC
:10DDD000810202EB411100EB81004079A4282DD192
:10DDE0009DF8AC0000EB400101EB00101D4901EB78
:10DDF000001030309DF8981000EB0110801C099045
:10DE0000007820F0200020300999087000229DF849
:10DE1000AC0000EB8000144901EB4020C0309DF8BD
:10DE2000981001EB810303EB411100EB810080F8B6
:10DE30003D209DF8AC100220FCF78AF8A1229DF845
:10DE4000AC0000EB8000084901EB4020C0309DF899
:10DE5000981001EB810303EB411100EB810042714B
:10DE600050E7000000410020C0450020002037900E
:10DE700015E09DF8AC0000EB4001C1EBC010FE497D
:10DE800001EBC001BDF8DC00C01C095C16AABDF89E
:10DE9000DC001154BDF8DC00401C81B23791BDF8A4
:10DEA000DC000628E5DB062116A81DF0E5FE0021B2
:10DEB000CDE92E01DDE92E21100A40EA016080182B
:10DEC00041EB21214FF480724FF00003CDE90801AE
:10DED000FAF778F99DF8AC0000EB8000E74901EB18
:10DEE0004020C0309DF8981001EB810303EB4111F5
:10DEF00000EB8100027100209DF8AC1001EB810164
:10DF0000DE4A02EB4121C87001229DF8AC0000EB13
:10DF10008000DA4901EB4020C0309DF8981001EBF9
:10DF2000810303EB411100F82120A7229DF8AC00EA
:10DF300000EB8000D14901EB4020C0309DF89810E3
:10DF400001EB810303EB411100EB81004271D9E643
:10DF50009DF8AC0000EB8000C84901EB4020C030C8
:10DF60009DF8981001EB810202EB411110F821009D
:10DF700006282BDC00219DF8AC0000EB8000BF4A96
:10DF800002EB4020C17007229DF8AC0000EB80003E
:10DF9000BA4901EB4021C0319DF8980000EB8003A5
:10DFA00003EB401001F82020A7229DF8AC0000EB05
:10DFB0008000B24901EB4020C0309DF8981001EB81
:10DFC000810303EB411100EB810042719DF8AC002D
:10DFD00000EB8000A94901EB4020C0309DF898106B
:10DFE00001EB810202EB411110F8210001282CDC29
:10DFF00000219DF8AC0000EB8000A04A02EB40201D
:10E00000C17002229DF8AC0000EB80009B4901EB3F
:10E010004021C0319DF8980000EB800303EB4010D5
:10E0200001F82020A3229DF8AC0000EB800093496A
:10E0300001EB4021C0319DF8980000EB800303EB19
:10E04000401001EB800042710AE29DF8AC0000EB49
:10E0500080008A4901EB4020C0309DF8981001EB08
:10E06000810202EB411110F8210007282CDC00216D
:10E070009DF8AC0000EB8000804A02EB4020C170AC
:10E0800008229DF8AC0000EB80007C4901EB4021A8
:10E09000C0319DF8980000EB800303EB401001F8BD
:10E0A0002020A3229DF8AC0000EB8000734901EB17
:10E0B0004020C0309DF8981001EB810303EB411123
:10E0C00000EB81004271CBE19DF8AC0000EB8000D9
:10E0D0006A4901EB4020C0309DF8981001EB8102A5
:10E0E00002EB411110F821000B282CDC00219DF8D7
:10E0F000AC0000EB8000614A02EB4020C1700C22B2
:10E100009DF8AC0000EB80005C4901EB4021C03180
:10E110009DF8980000EB800303EB401001F82020ED
:10E12000A1229DF8AC0000EB8000544901EB402097
:10E13000C0309DF8981001EB810303EB411100EB17
:10E14000810042718CE19DF8AC0000EB80004B49EE
:10E1500001EB4020C0309DF8981001EB810202EBEA
:10E16000411110F821000C282CDC00219DF8AC0096
:10E1700000EB8000414A02EB4020C1700D229DF867
:10E18000AC0000EB80003D4901EB4021C0319DF81F
:10E19000980000EB800303EB401001F82020A3223D
:10E1A0009DF8AC0000EB8000344901EB4020C0300A
:10E1B0009DF8981001EB810303EB411100EB810006
:10E1C00042714DE19DF8AC0000EB80002B4901EB62
:10E1D0004020C0309DF8981001EB810202EB411104
:10E1E00010F821000E286CDC0F229DF8AC0000EB2B
:10E1F0008000224901EB4021C0319DF8980000EBDE
:10E20000800303EB401001F82020A1229DF8AC0010
:10E2100000EB8000194901EB4021C0319DF89800C6
:10E2200000EB800303EB401001EB800042719DF88E
:10E23000AC0000EB8000114901EB4021C0319DF89A
:10E24000980000EB800303EB401001EB800082702C
:10E250009DF8AC1001EB410000EB0110084901EB07
:10E26000001130319DF8980001EB0010801C0990DE
:10E27000007820F0800005E0347C0020C0450020BC
:10E28000004100208030099908709DF8AC0000EB37
:10E29000400101EB0010FC4901EB001030309DF80B
:10E2A000981000EB0110801C0990007820F0040009
:10E2B000001D099908709DF8AC0000EB400101E0D9
:10E2C000E9E352E001EB0010EF4901EB00103030C0
:10E2D0009DF8981000EB01108078C0F34010E8B36F
:10E2E0009DF8AC0000EB400101EB0010E64901EBAA
:10E2F000001030309DF8981000EB0110801C099040
:10E30000007820F02002099802709DF8AC0000EB24
:10E31000400101EB0010DC4901EB001030309DF8AA
:10E32000981000EB01108078C0F34000A8B99DF868
:10E33000AC1001EB410000EB0110D34901EB0010E0
:10E3400030309DF8981000EB0110801C0990007887
:10E3500020F0080008300999087000E064E09DF89A
:10E36000AC100220FBF7F4FD7AE09DF8AC0000EB66
:10E370008000C64901EB4021C0319DF8980000EBB8
:10E38000800202EB401011F820109DF8AC0000EB69
:10E390008000BE4A02E064E090E0CEE002EB402064
:10E3A000007981425CD19DF8AC0000EB8000114601
:10E3B00001EB4020C0309DF8981001EB810202EB88
:10E3C000411100EB81008078A1282ED0A3229DF876
:10E3D000AC0000EB8000AD4901EB4021C0319DF85D
:10E3E000980000EB800303EB401001EB80004271CA
:10E3F0009DF8AC0000EB8000A44901EB4020C03048
:10E400009DF8981001EB810202EB411100EB8100B5
:10E410008078A22824D000209DF8AC1001EB810167
:10E420009A4A02EB4121C8701AE0A1229DF8AC0083
:10E4300000EB8000954901EB4021C0319DF8980028
:10E4400000EB800303EB401001EB800042710121DF
:10E450009DF8AC0000EB80008C4A02EB4020C170BC
:10E4600050E4A1229DF8AC0000EB8000874901EB4D
:10E470004021C0319DF8980000EB800303EB401071
:10E4800001EB800082709DF8AC0000EB80007F49BA
:10E4900001EB4021C0319DF8980000EB800303EBB5
:10E4A000401001EB8000427100219DF8AC0000EBB0
:10E4B0008000764A02EB4020C17023E49DF8AC0056
:10E4C00000EB8000714901EB4020C0309DF89810AE
:10E4D00001EB810202EB411110F8210006282BDC30
:10E4E00000219DF8AC0000EB8000684A02EB402060
:10E4F000C17007229DF8AC0000EB8000634901EB7E
:10E500004021C0319DF8980000EB800303EB4010E0
:10E5100001F82020A7229DF8AC0000EB80005B49A9
:10E5200001EB4020C0309DF8981001EB810303EB14
:10E53000411100EB8100427192E400219DF8AC0092
:10E5400000EB8000514A02EB4020C170A7229DF8E9
:10E55000AC0000EB80004D4901EB4021C0319DF83B
:10E56000980000EB800303EB401001EB8000427148
:10E570009DF8AC1001EB4100C0EBC110444901EB28
:10E58000C000407930287DD19DF8AC0000EB8000C0
:10E590003E4901EB4021C0319DF8980000EB80021C
:10E5A00002EB401011F820109DF8AC0000EB800049
:10E5B000364A02EB40200079814263D19DF8AC10CD
:10E5C00001EB410000EB01102F4901EB001030304E
:10E5D0009DF8981000EB0110801C0990007820F045
:10E5E0000102099802709DF8AC1001EB410000EBAC
:10E5F0000110254901EB001030309DF8981000EB18
:10E600000110801C0990007820F002020998027025
:10E610009DF8AC0000EB80001C4901EB4020C030AD
:10E620009DF8981001EB810202EB411100EB810093
:10E63000C078312835D19DF8AC1001EB410000EBDA
:10E640000110114901EB001030309DF8981000EBDB
:10E650000110801C0990007820F0200209980270B7
:10E6600000229DF8AC0000EB8000084901EB40203F
:10E67000C0309DF8981001EB810303EB411100EBD2
:10E68000810007E034E0000000410020C045002088
:10E69000347C002080F83D209DF8AC100220FBF770
:10E6A00057FC9DF8AC0000EB8000FB4901EB4020DB
:10E6B000C0309DF8981001EB810202EB411100EB94
:10E6C000810090F83E00012811D1A9229DF8AC00EC
:10E6D00000EB8000F04901EB4020C0309DF898101D
:10E6E00001EB810303EB411100EB8100827065E2D5
:10E6F0009DF8AC1001EB4100C0EBC110E74901EB04
:10E70000C000407931287DD19DF8AC0000EB80003D
:10E71000E14901EB4021C0319DF8980000EB8002F7
:10E7200002EB401011F820109DF8AC0000EB8000C7
:10E73000D94A02EB40200079814263D19DF8AC00B8
:10E7400000EB8000114601EB4020C0309DF898108E
:10E7500001EB810202EB411100EB810090F83E00D9
:10E7600040BB01229DF8AC0000EB8000CA4901EBE0
:10E770004021C0319DF8980000EB800303EB40106E
:10E7800001EB800080F83D209DF8AC1001EB4100CA
:10E7900000EB0110C24901EB001130319DF89800E7
:10E7A00001EB0010801C0990007820F00100401C53
:10E7B000099908709DF8AC1001EB410000EB0110C5
:10E7C000B74901EB001030309DF8981000EB0110B4
:10E7D000801C0990007820F0020209980270B1486C
:10E7E00090F88C08002870D1AF48407F01286CD188
:10E7F000AD48D0F81402AC49C98B884265D29DF867
:10E80000AC0000E0A1E000EB8000A34901EB402058
:10E81000C0309DF8981001EB810202EB411100EB32
:10E82000810090F83D0001284FD19DF8AC0000EB2D
:10E830008000994901EB4020C0309DF8981001EB11
:10E84000810202EB411100EB810090F87D00E0BBFA
:10E850004FF010429DF8AC0000EB80008E4901EBB8
:10E860004021C0319DF8980000EB800303EB40107D
:10E8700001EB800082609DF8AC0000EB400101EBF1
:10E880000010874901EB001130319DF8980001EB31
:10E89000001001789DF8AC0000EB80007E4A02EB8E
:10E8A000402041709DF8AC0000EB8000114601EB68
:10E8B0004021C0319DF8980000EB800202EB40102F
:10E8C00011F820109DF8AC0000E03DE000EB800066
:10E8D000714A02EB40200079814235D100229DF837
:10E8E000AC0000EB80006C4901EB4021C0319DF889
:10E8F000980000EB800303EB401001EB8000C27135
:10E90000A4229DF8AC0000EB8000634901EB40219C
:10E91000C0319DF8980000EB800303EB401001EB41
:10E9200080008270A3229DF8AC0000EB80005A4961
:10E9300001EB4020C0309DF8981001EB810303EB00
:10E94000411100EB8100427138E19DF8AC0000EB11
:10E950004001C1EBC010514901EBC00040793328A0
:10E960007DD19DF8AC0000EB400101EB00104C495B
:10E9700001EB001030309DF8981000EB0110801C66
:10E980000990007820F00101491C099801709DF858
:10E99000AC0000EB400101EB0010414901EB00111C
:10E9A00030319DF8980001EB0010801C0990007830
:10E9B00020F02002099802709DF8AC0000EB4001A5
:10E9C00001EB0010364901EB001030309DF8981033
:10E9D00000EB0110801C0990007820F00200801CE0
:10E9E000099908709DF8AC0000EB80002A4901EB02
:10E9F000402002799DF8AC0000EB800001EB402044
:10EA0000C0309DF8981001EB810303EB411100F831
:10EA100021209DF8AC0000EB400101EB00102049E3
:10EA200001EB001030309DF8981000EB0110801CB5
:10EA30000990007820F080008030099908709DF8D6
:10EA4000AC0000EB400101EB0010154901EB001098
:10EA500030309DF8981000EB0110807800E025E040
:10EA6000C0F3400020B99DF8AC100220FBF770FA0B
:10EA7000A2229DF8AC0000EB8000074901EB402189
:10EA8000C0319DF8980000EB800303EB401001EBD0
:10EA90008000827092E030E3C0450020347C00208A
:10EAA00000410020BC320020BC1200209DF8AC00C8
:10EAB00000EB4001C1EBC010FE4901EBC000407902
:10EAC00034287BD19DF8AC0000EB400101EB001035
:10EAD000F94901EB001030309DF8981000EB01105F
:10EAE000801C0990007820F02002099802709DF89F
:10EAF000AC0000EB400101EB0010EF4901EB00100E
:10EB000030309DF8981000EB0110801C09900078BF
:10EB100020F002020998027001229DF8AC0000EB7F
:10EB20008000E64901EB4020C0309DF8981001EBD1
:10EB3000810303EB411100EB810080F83E20A92204
:10EB40009DF8AC0000EB8000DC4901EB4021C031B6
:10EB50009DF8980000EB800303EB401001EB800070
:10EB600082709DF8AC0000EB8000D44901EB40209E
:10EB700002799DF8AC0000EB800001EB4021C03130
:10EB80009DF8980000EB800303EB401001F8202073
:10EB90009DF8AC0000EB400101EB0010C64901EB11
:10EBA000001130319DF8980001EB0010801C099095
:10EBB000007820F0800080300999087000202C90A7
:10EBC0002D900021379122E0DDE92C10000140EA70
:10EBD00011720901CDE92C129DF8AC1001EB410036
:10EBE000C0EBC110B34901EBC001BDF8DC00801DD2
:10EBF000085C3038C117DDE92C34184341EA0402BF
:10EC0000CDE92C02BDF8DC00401C80B23790BDF885
:10EC1000DC000628D8DB9DF8AC002C9900EB8000C6
:10EC2000A64A02EB4022C0329DF8980000EB800318
:10EC300003EB401002EB8000C0F81A1000222C9267
:10EC40002D920021379122E0DDE92C10000140EAED
:10EC500011720901CDE92C129DF8AC1001EB4100B5
:10EC6000C0EBC110934901EBC001BDF8DC000D30D1
:10EC7000085C3038C117DDE92C34184341EA04023E
:10EC8000CDE92C02BDF8DC00401C80B23790BDF805
:10EC9000DC000428D8DB9DF8AC002C9900EB800048
:10ECA000864A02EB4022C0329DF8980000EB8003B8
:10ECB00003EB401002EB8000416300222C922D9266
:10ECC0000021379122E0DDE92C10000140EA1172A9
:10ECD0000901CDE92C129DF8AC1001EB4100C0EB0D
:10ECE000C110744901EBC001BDF8DC001130085CB3
:10ECF0003038C117DDE92C3440EA03022143CDE965
:10ED00002C21BDF8DC00401C81B23791BDF8DC003D
:10ED10000628D8DB9DF8AC002C9900EB8000674AF0
:10ED200002EB4022C0329DF8980000EB800303EB19
:10ED3000401002EB8000C0F81E109DF8AC1001EBF3
:10ED40004100C0EBC1105B4901EBC00042799DF866
:10ED5000AC0000EB8000594901EB4021C0319DF827
:10ED6000980000EB800303EB401001EB8000C270C1
:10ED70009DF8AC1001EB410000EB01104E4901EB96
:10ED8000001130319DF8980001EB001082789DF859
:10ED9000AC0000EB8000494901EB4021C0319DF8F7
:10EDA000980000EB800303EB401001EB800002763B
:10EDB0009DF8AC0000EB8000404901EB4021C031E0
:10EDC0009DF8980000EB800202EB401011F8201033
:10EDD0009DF8AC0000EB8000384A02EB402000793F
:10EDE000814266DA00219DF8AC0000EB800002EB66
:10EDF0004020C170A7229DF8AC0000EB80002F4995
:10EE000001EB4021C0319DF8980000EB800303EB3B
:10EE1000401001EB8000427101219DF8AC0000EB35
:10EE20008000264A02EB4020C1709DF8AC0000EB48
:10EE30008000114601EB402002799DF8AC0000EB08
:10EE4000800001EB4021C0319DF8980000EB800369
:10EE500003EB401001F82020A1229DF8AC0000EB4C
:10EE60008000164901EB4021C0319DF8980000EB6D
:10EE7000800303EB401001EB800042719DF8AC1061
:10EE800001EB410000EB01100B4901EB00113031A7
:10EE90009DF8980001EB0010801C0990007820F08C
:10EEA00080018031099801709DF8AC1001EB4100A0
:10EEB00006E067E0347C002000410020C0450020CF
:10EEC00000EB0110FE4901EB001130319DF8980074
:10EED00001EB0010801C0990007820F00400001D58
:10EEE000099908709DF8AC1001EB410000EB01108E
:10EEF000F34901EB001030309DF8981000EB011041
:10EF00008078C0F34010E8B39DF8AC1001EB4100ED
:10EF100000EB0110EA4901EB001030309DF8981029
:10EF200000EB0110801C0990007820F02002099865
:10EF300002709DF8AC1001EB410000EB0110E049BC
:10EF400001EB001030309DF8981000EB0110807834
:10EF5000C0F34000F0BB9DF8AC1001EB410000EBAA
:10EF60000110D74901EB001030309DF8981000EBEC
:10EF70000110801C0990007820F0080008300999E1
:10EF8000087000E0B8E09DF8AC009DF8981001EB27
:10EF90000010C217CDE92C0200222C9800EBC00112
:10EFA00001EB0011C74800EB8100C0F81D209DF85F
:10EFB000AC0000EB8000C44901EB4020C0309DF85C
:10EFC000981001EB810202EB411100EB810022302D
:10EFD000099000E08BE02C9800EBC00101EB0011E0
:10EFE000B84800EB81010D3110220891DDE90801DC
:10EFF000F9F72BF99DF8AC0000EB8000B24901EB6A
:10F000004021C0319DF8980000EB800202EB4010D7
:10F0100001EB80012C9800EBC00202EB0012A94822
:10F0200000EB820051F81A2F40F8012F4968416027
:10F030009DF8AC0000EB400101EB0010A04901EB92
:10F04000001130319DF8980001EB001001782C98E8
:10F0500000EBC00202EB00129A4800F822102C9834
:10F0600000EBC00101EB0011964800EB81019748CD
:10F07000826941F8212F808B88809DF8AC0000EBDD
:10F080008000914901EB4021C0319DF8980000EBD0
:10F09000800202EB401001EB8000416B2C9800EBEA
:10F0A000C00202EB0012874800EB8200C0F8091092
:10F0B0009DF8AC0000EB400101EB0010804901EB32
:10F0C000001130319DF8980001EB001041682C9838
:10F0D00000EBC00202EB00127A4800EB8200C0F89D
:10F0E00027102C9881B208200991FAF731FF9DF87A
:10F0F000AC100220FAF72CFFD4E200219DF8AC00FE
:10F1000000EB8000704A02EB4020C1709DF8AC001B
:10F1100000EB8000114601EB4020C0309DF89810B4
:10F1200001EB810202EB411110F821000A2811DCE9
:10F130000B229DF8AC0000EB8000634901EB4020FE
:10F14000C0309DF8981001EB810303EB411100F8EA
:10F150002120FEE19DF8AC0000EB80005A4901EB54
:10F160004021C0319DF8980000EB800202EB401076
:10F1700011F820109DF8AC0000EB8000524A02EB21
:10F180004020007981427DD1504890F88C08E8BB3E
:10F190004F48D0F814020521B0FBF1F201FB120038
:10F1A00000EBC00101EB00114948203000EB810069
:10F1B0000021C0F81D104648D0F814020521B0FB0C
:10F1C000F1F201FB120000EBC00101EB001140481D
:10F1D000203000EB81000D3009909DF8AC0000EB71
:10F1E0008000394901EB4021C0319DF8980000EBC7
:10F1F000800202EB401001EB800022301022014619
:10F2000008900998F9F721F8314800E0C1E0D0F8FA
:10F2100014020521B0FBF1F201FB120000EBC0016A
:10F2200001EB00112A48203000EB81029DF8AC0070
:10F2300000EB8000244901EB4021C0319DF898008B
:10F2400000EB800303EB401001EB800050F81A1F25
:10F2500042F8011F406850601D48D0F81402052193
:10F26000B0FBF1F201FB120000EBC00101EB001357
:10F27000174920319DF8AC0000EB400202EB001072
:10F280000F4A00E065E102EB001230329DF8980071
:10F2900002EB0010007801F823000D48D0F81402AA
:10F2A0000521B0FBF1F201FB120000EBC00101EB04
:10F2B00000110748203000EB81029DF8AC0009E006
:10F2C00000410020E0140020C0450020BC32002096
:10F2D000BC12002000EB8000FA4901EB4021C03154
:10F2E0009DF8980000EB800303EB401001EB8000D9
:10F2F000406BC2F80900F448D0F814020521B0FBB5
:10F30000F1F201FB120000EBC00101EB0011EE482D
:10F31000203000EB810100F5FF50826941F8212F78
:10F32000808B8880E848D0F814020521B0FBF1F00A
:10F3300081B202200991F9F7CBFE00210620FAF7ED
:10F3400007FEE148D0F81402DF49C98B884206D293
:10F35000DD48D0F81402401CDB49C1F8140200213A
:10F360000520FAF7F5FD9DF8AC0000EB400101EB3C
:10F370000010D64901EB001030309DF8981000EBDA
:10F380000110801C0990007820F008020998027092
:10F3900015E09DF8AC0000EB400101EB0010CB49FB
:10F3A00001EB001030309DF8981000EB0110801C2C
:10F3B0000990007820F008000830099908700022B0
:10F3C0009DF8AC0000EB8000BE4901EB4021C0314C
:10F3D0009DF8980000EB800303EB401001EB8000E8
:10F3E00080F83E209DF8AC100220FAF7B1FD9DF8A0
:10F3F000AC009DF8981001EB0010C217CDE92C026B
:10F4000000222C9800EBC00101EB0011B04800EB8A
:10F410008100C0F81D209DF8AC0000EB8000A949D8
:10F4200001EB4020C0309DF8981001EB810202EB07
:10F43000411100EB8100223009902C9800EBC001B3
:10F4400001EB0011A24800EB81010D31102208915F
:10F45000DDE90801F8F7F9FE9DF8AC0000EB80004B
:10F46000984901EB4021C0319DF8980000EB8002E3
:10F4700002EB401001EB80012C9800EBC00202EB84
:10F480000012934800EB820051F81A2F40F8012F28
:10F49000496841609DF8AC0000EB400101EB0010B1
:10F4A0008A4901EB001130319DF8980001EB001002
:10F4B00001782C9800EBC00202EB0012844800F89F
:10F4C00022102C9800EBC00101EB0011804800EBEA
:10F4D00081018048826941F8212F808B88809DF8C6
:10F4E000AC0000EB8000774901EB4021C0319DF872
:10F4F000980000EB800202EB401001EB8000416BB2
:10F500002C9800EBC00202EB0012714800EB820065
:10F51000C0F809109DF8AC0000EB400101EB0010B1
:10F520006A4901EB001130319DF8980001EB0010A1
:10F5300041682C9800EBC00202EB0012644800EB1B
:10F540008200C0F827102C9881B208200991FAF7A0
:10F55000FFFCA7229DF8AC0000EB8000594901EBAD
:10F560004021C0319DF8980000EB800303EB401070
:10F5700001EB80004271A2229DF8AC0000EB8000FC
:10F58000504901EB4021C0319DF8980000EB800309
:10F5900003EB401001EB8000827000222C922D9230
:10F5A0000021379122E0DDE92C10000140EA1172C0
:10F5B0000901CDE92C129DF8AC0000EB4001C1EB34
:10F5C000C010454901EBC001BDF8DC000B30085C00
:10F5D0003038C117DDE92C24104341EA0402CDE99B
:10F5E0002C02BDF8DC00401C80B23790BDF8DC0076
:10F5F0000A28D8DB9DF8AC00DDE92C1200EB800076
:10F60000304B03EB4023C0339DF8980000EB80049F
:10F6100004EB401003EB800040F8221F4260002200
:10F620002C922D920021379122E0DDE92C1000016F
:10F6300040EA11720901CDE92C129DF8AC0000EBF3
:10F640004001C1EBC010244901EBC001BDF8DC0052
:10F650001530085C3038C117DDE92C3440EA03026C
:10F660002143CDE92C21BDF8DC00401C81B237914B
:10F67000BDF8DC000A28D8DB9DF8AC00DDE92C21C0
:10F6800000EB80000F4B03EB4020C0309DF898301A
:10F6900003EB830404EB431300EB8300223082600E
:10F6A000C16000BF00BF06F0C1BD9DF8AC0000EB1B
:10F6B0004001C1EBC010084911F8300004280DD1F9
:10F6C000249017E0C0450020BC120020004100201B
:10F6D000E0140020BC320020347C00209DF8AC00F7
:10F6E00000EB4001C1EBC010FE4911F830001528B5
:10F6F00000D124909DF8AC0000EB4001C1EBC0109C
:10F70000F84901EBC00041789DF8AC0000EB4002E5
:10F71000C2EBC010F34A12F8300041EA002041F277
:10F720003001884202D1A62024903DE09DF8AC0033
:10F7300000EB4001C1EBC010EA4901EBC000417889
:10F740009DF8AC0000EB4002C2EBC010E54A12F895
:10F75000300041EA002041F23101884202D1A72065
:10F76000249021E09DF8AC0000EB4001C1EBC010FB
:10F77000DC4911F83000022816D19DF8AC0000EBEE
:10F780004001C1EBC010D74901EBC00001799DF8E1
:10F79000AC0000EB4002C2EBC010D24A02EBC0004A
:10F7A000C07841EA002124919DF8AC0000EB800074
:10F7B000CD4901EB4020817826910021CB4A9DF86C
:10F7C000AC0002EB00129DF898001154C848007F6D
:10F7D000012815D19DF8AC0000EB400101EB0010B1
:10F7E000C44901EB001030309DF8981000EB011077
:10F7F000801C0990007820F0800080300999087002
:10F800009DF8AC0000EB400101EB0010B94901EBA1
:10F81000001030309DF8981000EB0110801C09900A
:10F82000007820F04001403109980170BDF8900047
:10F83000A7287DD007DC04287BD015287AD0A628FD
:10F8400041F0B08346E0A0F55850303820B111287F
:10F8500071D01228F4D1FCE39DF8AC0000EB8000DD
:10F86000A14901EB4020C0309DF8981001EB8102C6
:10F8700002EB411110F8210058BB00219DF8AC00AB
:10F8800000EB8000984A02EB4020C17001229DF8F5
:10F89000AC0000EB8000944901EB4021C0319DF8A1
:10F8A000980000EB800303EB401001F82020A72212
:10F8B0009DF8AC0000EB80008B4901EB4020C0308C
:10F8C0009DF8981001EB810303EB411100EB8100DF
:10F8D0004271FDE300219DF8AC0000EB8000824AFC
:10F8E00002EB4020C1709DF8AC0000EB8000114697
:10F8F00001EB4020C0309DF8981001EB810202EB33
:10F90000411110F82100022828DC03229DF8AC00E8
:10F9100000EB8000744901EB4021C0319DF8980054
:10F9200000EB800303EB401001F82020A92203E044
:10F93000BBE022E13CE268E29DF8AC0000EB800015
:10F94000694901EB4020C0309DF8981001EB81031C
:10F9500003EB411100EB81004271A5E09DF8AC0082
:10F9600000EB8000604901EB4020C0309DF898100A
:10F9700001EB810202EB411110F82100052823DC84
:10F9800006229DF8AC0000EB8000574901EB4021B6
:10F99000C0319DF8980000EB800303EB401001F8A4
:10F9A0002020A2229DF8AC0000EB80004E4901EB24
:10F9B0004021C0319DF8980000EB800303EB40101C
:10F9C00001EB800042716FE09DF8AC0000EB80001D
:10F9D000454901EB4020C0309DF8981001EB8102B1
:10F9E00002EB411100EB81004079A52815D19DF86B
:10F9F000AC0000EB400101EB00103E4901EB0010B0
:10FA000030309DF8981000EB0110801C09900078B0
:10FA100020F00400001D099908709DF8AC0000EB6F
:10FA20008000314901EB4020C0309DF8981001EB77
:10FA3000810202EB411100EB81008078A12833D0D4
:10FA40009DF8AC0000EB8000274901EB4021C0315C
:10FA50009DF8980000EB800202EB401001EB800063
:10FA600082789DF8AC0000EB80001F4901EB40213B
:10FA7000C0319DF8980000EB800303EB401001EBD0
:10FA800080004271A1229DF8AC0000EB8000164975
:10FA900001EB4020C0309DF8981001EB810303EB8F
:10FAA000411100EB8100827013E79DF8AC0000EB80
:10FAB00080000D4901EB4020C0309DF8981001EB0B
:10FAC000810202EB411100EB81004079A42838D17A
:10FAD0009DF8AC0000EB400101EB0010054901EB83
:10FAE000001009E0347C0020C0450020343F002095
:10FAF000BC1200200041002030309DF8981000EB2F
:10FB00000110801C0990007820F020002030099915
:10FB1000087000229DF8AC0000EB8000FE4901EB6C
:10FB20004020C0309DF8981001EB810303EB411198
:10FB300000EB810080F83D209DF8AC100220FAF720
:10FB400007FA00219DF8AC0000EB8000F24A02EBBE
:10FB50004020C170A1229DF8AC0000EB8000EE496E
:10FB600001EB4020C0309DF8981001EB810303EBBE
:10FB7000411100EB81004271ABE69DF8AC0000EB57
:10FB80008000E54901EB4020C0309DF8981001EB62
:10FB9000810202EB411110F8210001282CDC002128
:10FBA0009DF8AC0000EB8000DB4A02EB4020C17006
:10FBB00002229DF8AC0000EB8000D74901EB402108
:10FBC000C0319DF8980000EB800303EB401001F872
:10FBD0002020A3229DF8AC0000EB8000CE4901EB71
:10FBE0004020C0309DF8981001EB810303EB4111D8
:10FBF00000EB81004271DAE09DF8AC0000EB800080
:10FC0000C54901EB4020C0309DF8981001EB8102FE
:10FC100002EB411110F8210004282CDC00219DF892
:10FC2000AC0000EB8000BC4A02EB4020C170052212
:10FC30009DF8AC0000EB8000B74901EB4021C031DA
:10FC40009DF8980000EB800303EB401001F82020A2
:10FC5000A3229DF8AC0000EB8000AF4901EB4021EE
:10FC6000C0319DF8980000EB800303EB401001EBDE
:10FC7000800042719BE09DF8AC0000EB8000A6493B
:10FC800001EB4020C0309DF8981001EB810202EB9F
:10FC9000411110F82100062812DCA1229DF8AC00C9
:10FCA00000EB80009C4901EB4020C0309DF898108B
:10FCB00001EB810303EB411100EB8100427176E01F
:10FCC0009DF8AC0000EB8000934901EB4021C0316E
:10FCD0009DF8980000EB800202EB401011F8201014
:10FCE0009DF8AC0000EB80008B4A02EB40200079CD
:10FCF00081425CD19DF8AC0000EB8000114601EB25
:10FD00004020C0309DF8981001EB810202EB4111B8
:10FD100000EB81008078A1282ED0A3229DF8AC00B2
:10FD200000EB80007C4901EB4021C0319DF8980038
:10FD300000EB800303EB401001EB800042719DF863
:10FD4000AC0000EB8000744901EB4020C0309DF80E
:10FD5000981001EB810202EB411100EB81008078E9
:10FD6000A22824D000209DF8AC1001EB81016A4A42
:10FD700002EB4121C8701AE0A1229DF8AC0000EB13
:10FD80008000654901EB4021C0319DF8980000EBEF
:10FD9000800303EB401001EB8000427101219DF8CC
:10FDA000AC0000EB80005C4A02EB4020C17090E5A3
:10FDB000A1229DF8AC0000EB8000574901EB4021E7
:10FDC000C0319DF8980000EB800303EB401001EB7D
:10FDD000800042719DF8AC0000EB80004E4901EBC1
:10FDE0004021C0319DF8980000EB800303EB4010E8
:10FDF00001EB8000827000219DF8AC0000EB8000D8
:10FE0000454A02EB4020C17063E500219DF8AC003B
:10FE100000EB8000404A02EB4020C170A7229DF811
:10FE2000AC0000EB80003C4901EB4021C0319DF863
:10FE3000980000EB800303EB401001EB800042715F
:10FE40009DF8AC0000EB4001C1EBC010334901EB61
:10FE5000C0004079302865D19DF8AC0000EB8000EF
:10FE60002D4901EB4021C0319DF8980000EB800244
:10FE700002EB401011F820109DF8AC0000EB800060
:10FE8000254A02EB4020007981424BD19DF8AC001D
:10FE900000EB400101EB0010A2F5986101EB0010AE
:10FEA00030309DF8981000EB0110801C099000780C
:10FEB00020F00102099802709DF8AC1001EB41009E
:10FEC00000EB0110164901EB001030309DF898103E
:10FED00000EB0110801C0990007820F002020998C4
:10FEE00002709DF8AC0000EB80000B4901EB402054
:10FEF000C0309DF8981001EB810202EB411100EB3C
:10FF00008100C078312834D19DF8AC1001EB41005C
:10FF100000EB0110024906E0C0450020347C0020BF
:10FF2000004100204CE001EB001030309DF89810AB
:10FF300000EB0110801C0990007820F02002099845
:10FF4000027000229DF8AC0000EB8000FE4901EB3E
:10FF50004020C0309DF8981001EB810303EB411164
:10FF600000EB810080F83D209DF8AC100220F9F7ED
:10FF7000EFFF9DF8AC0000EB8000F34901EB40205F
:10FF8000C0309DF8981001EB810202EB411100EBAB
:10FF9000810090F83E00012811D1A9229DF8AC0003
:10FFA00000EB8000E84901EB4020C0309DF898103C
:10FFB00001EB810303EB411100EB8100827067E2EA
:10FFC0009DF8AC1001EB4100C0EBC110DF4901EB23
:10FFD000C000407931287CD19DF8AC0000EB800056
:10FFE000D94901EB4021C0319DF8980000EB800217
:10FFF00002EB401011F820109DF8AC0000EB8000DF
:020000040801F1
:10000000D14A02EB40200079814262D19DF8AC00D8
:1000100000EB8000114601EB4020C0309DF89810A5
:1000200001EB810202EB411100EB810090F83E00F0
:1000300050BB01229DF8AC0000EB8000C24901EBEF
:100040004021C0319DF8980000EB800303EB401085
:1000500000E0FDE301EB800080F83D209DF8AC104E
:1000600001EB410000EB0110B94901EB0011303107
:100070009DF8980001EB0010801C0990007820F09A
:100080000100401C099908709DF8AC1001EB41007B
:1000900000EB0110AE4901EB001030309DF89810D4
:1000A00000EB0110801C0990007820F002020998F2
:1000B0000270A84890F88C08F0BBA748407F012840
:1000C0003AD1A548D0F81402A349C98B884201E06F
:1000D000EBE3A4E030D29DF8AC0000EB80009A493D
:1000E00001EB4020C0309DF8981001EB810202EB3B
:1000F000411100EB810090F83D0001281CD19DF8D2
:10010000AC0000EB8000904901EB4020C0309DF82E
:10011000981001EB810202EB411100EB810090F895
:100120007D0048B94FF010429DF8AC0000EB800014
:10013000854901EB402100E070E0C0319DF8980056
:1001400000EB800303EB401001EB800082609DF820
:10015000AC1001EB410000EB01107D4901EB0011F7
:1001600030319DF8980001EB001001789DF8AC004B
:1001700000EB8000744A02EB402041709DF8AC0017
:1001800000EB8000114601EB4021C0319DF8980042
:1001900000EB800202EB401011F820109DF8AC003B
:1001A00000EB8000684A02EB40200079814235D1A3
:1001B00000229DF8AC0000EB8000634901EB402178
:1001C000C0319DF8980000EB800303EB401001EB79
:1001D0008000C271A4229DF8AC0000EB80005A4957
:1001E00001EB4021C0319DF8980000EB800303EB48
:1001F000401001EB80008270A3229DF8AC0000EB60
:100200008000514901EB4020C0309DF8981001EB6F
:10021000810303EB411100EB8100427138E19DF84D
:10022000AC1001EB4100C0EBC110484901EBC0002C
:10023000407933287DD19DF8AC1001EB410000EBF3
:100240000110434901EB001030309DF8981000EB8D
:100250000110801C0990007820F00101491C0998C8
:1002600001709DF8AC1001EB410000EB0110384922
:1002700001EB001130319DF8980001EB0010801C5B
:100280000990007820F02002099802709DF8AC10C7
:1002900001EB410000EB01102D4901EB0010303063
:1002A0009DF8981000EB0110801C0990007820F058
:1002B0000200801C099908709DF8AC0000EB8000DA
:1002C000214901EB402002799DF8AC0000EB800051
:1002D00001EB4020C0309DF8981001EB810303EB47
:1002E000411100F821209DF8AC1001EB410000EB1A
:1002F0000110174901EB001030309DF8981000EB09
:100300000110801C0990007820F08000803009994D
:1003100008709DF8AC1001EB410000EB01100C4996
:1003200001EB001030309DF8981000EB0110807840
:1003300000E025E0C0F3400020B99DF8AC10022099
:10034000F9F706FEA22209E0C0450020347C002017
:1003500000410020BC320020BC1200209DF8AC00FF
:1003600000EB8000FE4901EB4020C0309DF8981062
:1003700001EB810303EB411100EB8100827087E008
:100380009DF8AC1001EB4100C0EBC110F54901EB49
:10039000C000407934287BD19DF8AC1001EB4100BE
:1003A00000EB0110F04901EB001030309DF898107F
:1003B00000EB0110801C0990007820F020020998C1
:1003C00002709DF8AC1001EB410000EB0110E64912
:1003D00001EB001030309DF8981000EB0110801CEC
:1003E0000990007820F002020998027001229DF81D
:1003F000AC0000EB8000DA4901EB4020C0309DF8F2
:10040000981001EB810303EB411100EB810080F8B0
:100410003E20A9229DF8AC0000EB8000D04901EB02
:100420004020C0309DF8981001EB810303EB41118F
:1004300000EB810082709DF8AC0000EB8000C849A1
:1004400001EB402002799DF8AC0000EB800001EB4D
:100450004020C0309DF8981001EB810303EB41115F
:1004600000F821209DF8AC1001EB410000EB0110D9
:10047000BD4901EB001030309DF8981000EB0110E1
:10048000801C0990007820F0800080300999087065
:1004900000202C902D900021379122E0DDE92C10D6
:1004A000000140EA11720901CDE92C129DF8AC104F
:1004B00001EB4100C0EBC110AA4901EBC001BDF83E
:1004C000DC00801D085C3038C117DDE92C3418438E
:1004D00041EA0402CDE92C02BDF8DC00401C80B2E8
:1004E0003790BDF8DC000828D8DB9DF8AC002C99CB
:1004F00000EB80009A4A02EB4022C0329DF898003F
:1005000000EB800303EB401002EB8000C0F81A10F0
:1005100000222C922D920021379122E0DDE92C104F
:10052000000140EA11720901CDE92C129DF8AC10CE
:1005300001EB4100C0EBC1108A4901EBC001BDF8DD
:10054000DC000F30085C3038C117DDE92C3418436B
:1005500041EA0402CDE92C02BDF8DC00401C80B267
:100560003790BDF8DC000628D8DB9DF8AC002C994C
:1005700000EB80007A4A02EB4022C0329DF89800DE
:1005800000EB800303EB401002EB8000416300228C
:100590002C922D920021379122E0DDE92C100001F0
:1005A00040EA11720901CDE92C129DF8AC1001EB63
:1005B0004100C0EBC1106B4901EBC001BDF8DC008C
:1005C0001530085C3038C117DDE92C3440EA0302ED
:1005D0002143CDE92C21BDF8DC00401C81B23791CC
:1005E000BDF8DC000828D8DB9DF8AC002C9900EBA6
:1005F00080005B4A02EB4022C0329DF8980000EB7D
:10060000800303EB401002EB8000C0F81E109DF841
:10061000AC1001EB4100C0EBC110524901EBC0002E
:1006200042799DF8AC0000EB80004D4901EB402180
:10063000C0319DF8980000EB800303EB401001EB04
:100640008000C2709DF8AC1001EB410000EB01107E
:10065000454901EB001130319DF8980001EB001085
:1006600082789DF8AC0000EB80003D4901EB402111
:10067000C0319DF8980000EB800303EB401001EBC4
:10068000800002769DF8AC0000EB8000344901EB5D
:100690004021C0319DF8980000EB800202EB401031
:1006A00011F820109DF8AC0000EB80002C4A02EB02
:1006B0004020007981427DDA00219DF8AC0000EBFA
:1006C000800002EB4020C170A7229DF8AC0000EB37
:1006D0008000234901EB4021C0319DF8980000EBD8
:1006E000800303EB401001EB8000427101219DF873
:1006F000AC0000EB80001A4A02EB4020C1709DF86C
:10070000AC0000EB8000114601EB402002799DF81F
:10071000AC0000EB800001EB4021C0319DF8980057
:1007200000EB800303EB401001F82020A1229DF88C
:10073000AC0000EB80000A4901EB4021C0319DF87C
:10074000980000EB800303EB401001EB8000427146
:100750009DF8AC1001EB410000EB0110024905E0EF
:10076000C0450020347C00200041002001EB001136
:1007700030319DF8980001EB0010801C0990007842
:1007800020F080008030099908709DF8AC1001EBD2
:10079000410000EB0110FE4901EB001030309DF8E4
:1007A000981000EB0110801C0990007820F00400E4
:1007B000001D00E04DE0099908709DF8AC1001EBB8
:1007C000410000EB0110F24901EB001030309DF8C0
:1007D000981000EB01108078C0F34010C8B39DF86A
:1007E000AC1001EB410000EB0110E94901EB0010F6
:1007F00030309DF8981000EB0110801C09900078B3
:1008000020F02002099802709DF8AC1001EB410025
:1008100000EB0110DE4901EB001030309DF898101C
:1008200000EB01108078C0F34000E8BB9DF8AC10ED
:1008300001EB410000EB0110D54901EB0010303015
:100840009DF8981000EB0110801C0990007801E0E1
:10085000C0E0BEE020F008000830099908709DF85B
:10086000AC009DF8981001EB0010C217CDE92C02E6
:1008700000222C9800EBC00101EB0011C54800EBF1
:100880008100C0F81D209DF8AC0000EB8000C2493B
:1008900001EB4020C0309DF8981001EB810202EB83
:1008A000411100EB810001E08EE07BE322300990F2
:1008B0002C9800EBC00101EB0011B64800EB810160
:1008C0000D3110220891DDE90801F7F7BEFC9DF813
:1008D000AC0000EB8000B04901EB4021C0319DF835
:1008E000980000EB800202EB401001EB80012C9895
:1008F00000EBC00202EB0012A64800EB820051F8A8
:100900001A2F40F8012F496841609DF8AC1001EBA7
:10091000410000EB01109E4901EB001130319DF8C0
:10092000980001EB001001782C9800EBC00202EB5C
:100930000012984800F822102C9800EBC00101EB3F
:100940000011944800EB81019448826941F8212FFD
:10095000808B88809DF8AC0000EB80008E4901EB15
:100960004021C0319DF8980000EB800202EB40105E
:1009700001EB8000416B2C9800EBC00202EB0012EF
:10098000844800EB8200C0F809109DF8AC0000EB31
:10099000400101EB00107E4901EB001130319DF860
:1009A000980001EB001041682C9800EBC00202EBAC
:1009B0000012784800EB8200C0F827102C9881B212
:1009C00008200991F9F7C4FA9DF8AC100220F9F754
:1009D000BFFAE7E200219DF8AC0000EB80006E4A10
:1009E00002EB4020C1709DF8AC0000EB8000114686
:1009F00001EB4020C0309DF8981001EB810202EB22
:100A0000411110F82100032811DC04229DF8AC00EC
:100A100000EB8000604901EB4020C0309DF8981049
:100A200001EB810303EB411100F82120FEE19DF869
:100A3000AC0000EB8000584901EB4021C0319DF82B
:100A4000980000EB800202EB401011F820109DF896
:100A5000AC0000EB8000504A02EB4020007981425C
:100A60007DD14E4890F88C08E8BB4D48D0F8140270
:100A70000521B0FBF1F201FB120000EBC00101EB1C
:100A800000114748203000EB81000021C0F81D1004
:100A90004348D0F814020521B0FBF1F201FB12002B
:100AA00000EBC00101EB00113D48203000EB81005C
:100AB0000D3009909DF8AC0000EB8000364901EB49
:100AC0004021C0319DF8980000EB800202EB4010FD
:100AD00001EB800022301022014608900998F7F7B8
:100AE000B4FB2F4800E0C1E0D0F814020521B0FBB0
:100AF000F1F201FB120000EBC00101EB00112848EC
:100B0000203000EB81029DF8AC0000EB8000224910
:100B100001EB4021C0319DF8980000EB800303EB0E
:100B2000401001EB800050F81A1F42F8011F406886
:100B300050601B48D0F814020521B0FBF1F201FB14
:100B4000120000EBC00101EB0013154920319DF8A4
:100B5000AC0000EB400202EB00100D4A00E065E142
:100B600002EB001230329DF8980002EB0010007882
:100B700001F823000A48D0F814020521B0FBF1F275
:100B800001FB120000EBC00101EB0011044809E079
:100B900000410020E0140020C0450020BC320020AD
:100BA000BC120020203000EB81029DF8AC0000EB6D
:100BB0008000FE4901EB4021C0319DF8980000EB18
:100BC000800303EB401001EB8000406BC2F809008A
:100BD000F748D0F814020521B0FBF1F201FB120036
:100BE00000EBC00101EB0011F148203000EB810166
:100BF00000F5FF50826941F8212F808B8880EC48F6
:100C0000D0F814020521B0FBF1F081B20220099165
:100C1000F8F75EFA00210620F9F79AF9E448D0F8CF
:100C20001402E349C98B884206D2E148D0F8140285
:100C3000401CDF49C1F8140200210520F9F788F9AA
:100C40009DF8AC0000EB400101EB0010D94901EB2D
:100C5000001030309DF8981000EB0110801C0990B6
:100C6000007820F008020998027015E09DF8AC00A9
:100C700000EB400101EB0010CE4901EB00103030D9
:100C80009DF8981000EB0110801C0990007820F06E
:100C9000080008300999087000229DF8AC0000EBAC
:100CA0008000C24901EB4021C0319DF8980000EB63
:100CB000800303EB401001EB800080F83E209DF89C
:100CC000AC100220F9F744F99DF8AC109DF898009B
:100CD00000EB0110C217CDE92C0200222C9800EB8A
:100CE000C00101EB0011B44800EB8100C0F81D20E9
:100CF0009DF8AC0000EB8001AC4800EB4120C03017
:100D00009DF8981001EB810202EB411100EB81008C
:100D1000223009902C9800EBC00101EB0011A6488D
:100D200000EB81010D3110220891DDE90801F7F790
:100D30008CFA9DF8AC0000EB80009C4901EB40214F
:100D4000C0319DF8980000EB800202EB401001EBEF
:100D500080012C9800EBC00202EB0012964800EBD9
:100D6000820051F81A2F40F8012F496841609DF820
:100D7000AC0000EB400101EB00108E4901EB0011CB
:100D800030319DF8980001EB001001782C9800EBB1
:100D9000C00202EB0012884800F822102C9800EBE9
:100DA000C00101EB0011844800EB81018348826996
:100DB00041F8212F808B88809DF8AC0000EB8000EB
:100DC0007A4901EB4021C0319DF8980000EB800288
:100DD00002EB401001EB8000416B2C9800EBC0024D
:100DE00002EB0012744800EB8200C0F809109DF875
:100DF000AC0000EB400101EB00106E4901EB00116B
:100E000030319DF8980001EB001041682C9800EB00
:100E1000C00202EB0012684800EB8200C0F8271005
:100E20002C9881B208200991F9F792F800229DF8D8
:100E3000AC0000EB80005D4901EB4021C0319DF822
:100E4000980000EB800303EB401001EB800080F87A
:100E50003E20A7229DF8AC0000EB8000534901EB37
:100E60004021C0319DF8980000EB800303EB401057
:100E700001EB80004271A2229DF8AC0000EB8000E3
:100E80004A4901EB4021C0319DF8980000EB8003F6
:100E900003EB401001EB8000827000222C922D9217
:100EA0000021379122E0DDE92C10000140EA1172A7
:100EB0000901CDE92C129DF8AC0000EB4001C1EB1B
:100EC000C0103F4901EBC001BDF8DC000B30085CED
:100ED0003038C117DDE92C3440EA03022143CDE963
:100EE0002C21BDF8DC00401C81B23791BDF8DC003C
:100EF0000C28D8DB9DF8AC00DDE92C2100EB80004C
:100F00002A4B03EB4023C0339DF8980000EB80048C
:100F100004EB401003EB800040F8222F41600022D8
:100F20002C922D920021379122E0DDE92C10000156
:100F300040EA11720901CDE92C129DF8AC0000EBDA
:100F40004001C1EBC0101E4901EBC001BDF8DC003F
:100F50001730085C3038C117DDE92C3440EA030251
:100F60002143CDE92C21BDF8DC00401C81B2379132
:100F7000BDF8DC000C28D8DB9DF8AC00DDE92C21A5
:100F800000EB8000094B03EB4020C0309DF8983007
:100F900003EB830404EB431300EB830022308260F5
:100FA000C16000BF00BF05F041B90000C04500208E
:100FB000BC12002000410020E0140020BC320020C0
:100FC000347C00200021FE4A9DF8AC0002EB0012A8
:100FD0009DF8980011549DF8AC0000EB4001C1EB66
:100FE000C010F84901EBC000407870280ED19DF880
:100FF000AC0000EB4001C1EBC010F24901EBC000B6
:101000008078FA2802D1B121249142E09DF8AC0009
:1010100000EB4001C1EBC010EA4901EBC000407891
:1010200000F0F000C0280ED19DF8AC0000EB4001AC
:10103000C1EBC010E34901EBC0008078FA2802D16F
:10104000B621249125E09DF8AC0000EB4001C1EBF6
:10105000C010DC4911F8300000F0F000502818D121
:101060009DF8AC0000EB4001C1EBC010D54901EB8D
:10107000C000407800F0F00030280AD19DF8AC00A4
:1010800000EB4001C1EBC010CE4901EBC0008178FC
:1010900024919DF8AC0000EB8000CB4901EB40208F
:1010A000817826910021C64A9DF8AC0002EB00121F
:1010B0009DF8980011549DF8AC0000EB400101EB45
:1010C0000010C24901EB001130319DF8980001EB8E
:1010D0000010801C0990007820F0400040300999F1
:1010E0000870BB48007F012815D19DF8AC0000EBCB
:1010F000400101EB0010B54901EB001030309DF8C4
:10110000981000EB0110801C0990007820F08000FE
:10111000803009990870BDF89000652874D004DC0F
:10112000012809D0032805D16FE0B12802D0B628E4
:1011300000D100E075E174E19DF8AC0000EB4001E6
:10114000C1EBC0109F4901EBC0000079012806D017
:10115000022805D0032804D0052853D102E051E02D
:1011600050E04FE09DF8AC0000EB8000964901EBA9
:101170004020C0309DF8981001EB810202EB411134
:1011800010F82100E8BB00219DF8AC0000EB8000C6
:101190008D4A02EB4020C17001229DF8AC0000EBAB
:1011A0008000894901EB4021C0319DF8980000EB97
:1011B000800303EB401001F82020B6229DF8AC001C
:1011C00000EB8000804901EB4021C0319DF8980080
:1011D00000EB800303EB401001EB80004271B22270
:1011E0009DF8AC0000EB8000774901EB4021C03155
:1011F0009DF8980000EB800303EB401001EB8000AA
:10120000827000BF00BF0CE127E09DF8AC0000EB4E
:101210004001C1EBC0106B4901EBC000C1796D48C2
:1012200080F8101E9DF8AC0000EB400101EB0010AF
:10123000664901EB001130319DF8980001EB001078
:10124000801C0990634890F8100EC2080998007835
:1012500062F3000009990870E3E09DF8AC0000EB30
:101260004001C1EBC010574901EBC000007900F00C
:10127000F00010B9B821249101E0B92124919DF822
:10128000AC0000EB4001C1EBC0104E4901EBC000C7
:10129000007900F00F0125910021379120E09DF8A1
:1012A000AC0000EB400101EB0010484901EB0011DC
:1012B0003031BDF8DC0001EB001041789DF8AC0046
:1012C00000EB4002C2EBC0103E4A12F8300050382A
:1012D000814200D112E0BDF8DC00401C81B23791A0
:1012E0009DF8AC0000EB400101EB0010374901EB29
:1012F0000010C179BDF8DC008142D0DC00BFBDF830
:10130000DC109DF894000844C1B226919DF8AC0011
:1013100000EB80002C4901EB4020C0309DF8981074
:1013200001EB810202EB411110F8210001282CD1C0
:1013300000219DF8AC0000EB8000234A02EB402026
:10134000C17002229DF8AC0000EB80001E4901EB49
:101350004021C0319DF8980000EB800303EB401062
:1013600001F82020B9229DF8AC0000EB800016495E
:1013700001EB4020C0309DF8981001EB810303EB96
:10138000411100EB810042714AE09DF8AC0000EB96
:1013900080000D4901EB4020C0309DF8981001EB12
:1013A000810202EB411110F82100012838D10021FF
:1013B0009DF8AC0000EB8000034A02EB40200BE0FC
:1013C000343F0020347C0020C04500200041002034
:1013D000BC120020BC220020C17002229DF8AC008B
:1013E00000EB8000FE4901EB4021C0319DF89800E0
:1013F00000EB800303EB401001F82020B9229DF898
:10140000AC0000EB8000F64901EB4020C0309DF8B5
:10141000981001EB810303EB411100EB8100427155
:1014200000BF00BFBFE59DF8AC0000EB400101EB41
:101430000010EC4901EB0010007B20B101287DD0A9
:1014400002287CD1E7E2E8499DF8AC0031F81000B1
:10145000801F81B209919DF8AC0000EB4001C1EB07
:10146000C010E24901EBC000401C08900999F8F750
:1014700031FA0022CDE92E029DF8AC0000EB4001CC
:10148000C1EBC010D94901EBC002D7489DF8AC10A0
:1014900030F81100401F111809910421099815F026
:1014A00037FCC217CDE92C02DDE92E42DDE92C1014
:1014B0006140504001437DD10022CD499DF8AC00F0
:1014C00001EB001002709DF8AC0000EB4001C1EB95
:1014D000C010C64901EBC00001792491BDF890000D
:1014E000312802D0452866D1EAE0BF489DF8AC100B
:1014F00030F811001838412190FBF1F0C217C1B249
:10150000CDE92C02BB4880F8B81100203790CDE01F
:101510009DF8AC0000EB4001C1EBC010B34901EBFA
:10152000C001BDF8DC0000EB80101430095CB24A49
:10153000BDF8DC0011549DF8AC0001E0C3E069E2A5
:1015400000EB4001C1EBC010A84901EBC001BDF8A0
:10155000DC0000EB80101A30014409910821099841
:1015600015F094FB8DED0E0AA34A0C32BDF8DC0099
:101570000E9902EB001041609DF8AC0000EB4001B9
:10158000C1EBC010994901EBC001BDF8DC0000EBD4
:1015900080103230014409910821099815F076FB3A
:1015A0008DED0E0A944A0C32BDF8DC000E9902EB68
:1015B000001001E086E084E001609DF8AC1001EBD2
:1015C0004100C0EBC110894901EBC001BDF8DC004E
:1015D00000EB80103A30014409910821099815F078
:1015E00055FB8DED0E0A844A0C32BDF8DC000E99D5
:1015F00002EB001081609DF8AC1001EB4100C0EBE4
:10160000C1107A4901EBC001BDF8DC0000EB80108D
:101610004230014409910821099815F037FB8DEDFE
:101620000E0A754A0C32BDF8DC000E9902EB001070
:10163000C1609DF8AC1001EB410000EB011069495D
:1016400001EB00113031BDF8DC0001EB0010801C13
:101650000990007820F080018031099801709DF890
:10166000AC1001EB4100C0EBC110604901EBC001BF
:101670005D4A9DF8AC0032F81000401E0A5C9DF8EF
:10168000AC0000EB8000564901EB4021C0319DF8D1
:10169000980000EB800303EB401001EB800080F822
:1016A0003C20BDF8DC00401C81B23791BDF8DC0065
:1016B0000021DDE92C34C01AA141FFF629AF00E07A
:1016C00000BF00BF9EE29DF8AC1001EB4100C0EBF3
:1016D000C110464901EBC000407D9DF8AC1001EB04
:1016E0004102C2EBC111414A02EBC101897D40EACE
:1016F0000120C217CDE92C029DF8AC1001EB41008E
:10170000C0EBC110394901EBC001099115210998BD
:10171000F8F7C4F80022CDE92E02DDE92E42DDE91A
:101720002C1061405040014359D19DF8AC1001EBA1
:101730004100C0EBC1102D4911F83000401EC1B26C
:10174000269100212A4A9DF8AC0002EB00129DF878
:1017500098001154284A9DF8980011549FED270ACB
:1017600010EE101A0C329DF8980002EB0010416048
:101770009DF8AC0000EB4001C1EBC0101B4901EB30
:10178000C00081799DF8AC0000EB4002C2EBC010B4
:10179000164A02EBC000407941EA002000EE100A30
:1017A000B8EEC00A9FED161AC0EE010A9DF8AC0013
:1017B00000EB4001C1EBC010114601EBC000017904
:1017C0009DF8AC0000EB4002C2EBC010074A02EBF0
:1017D000C000C07841EA002000EE100A12E019E1D2
:1017E000C045002000410020C06D0020347C002056
:1017F000343F0020BC32002075340020000000007F
:1018000000FF7F47B8EEC00A30EE800A10EE101AD3
:10181000FD4A9DF8980002EB001001609DF8AC00B5
:1018200000EB4001C1EBC010F84901EBC000817A28
:101830009DF8AC0000EB4002C2EBC010F34A02EB93
:10184000C000407A41EA002000EE100AB8EEC00A5B
:101850001FED151AC0EE010A9DF8AC0000EB400127
:10186000C1EBC010114601EBC000017A9DF8AC003D
:1018700000EB4002C2EBC010E44A02EBC000C079AA
:1018800041EA002000EE100AB8EEC00A30EE800AED
:1018900010EE101ADC4A9DF8980002EB00108160EF
:1018A0009DF8AC0000EB4001C1EBC010D74901EB43
:1018B000C000C07A00F0800030BB9DF8AC0000EBA7
:1018C0004001C1EBC010D14901EBC000017B9DF884
:1018D000AC0000EB4002C2EBC010CC4A02EBC000EF
:1018E000C07A41EA002000EE100AF8EEC00AB3EE1A
:1018F000001A80EE810A10EE100AC34A9DF8981073
:1019000002EB0111C86046E09DF8AC0000EB40011D
:10191000C1EBC010BD4901EBC000017B9DF8AC00DC
:1019200000EB4002C2EBC010B84A02EBC000C07A24
:1019300041EA0020404280B200EE100AB8EEC00A30
:101940008DED030A0398F6F7E9FE9FEDB10B53EC1A
:10195000102BCDE904019DED040B51EC100BF6F7B3
:10196000C1FD9FEDAD0B53EC102BCDE906019DEDB4
:10197000060B51EC100BF6F740FDCDE908019DED8B
:10198000080B51EC100BF6F7DCFE9F4A9DF89810FF
:1019900002EB0111C8609DF8AC1001EB410000EBB7
:1019A00001109F4901EB001030309DF8981000EBBA
:1019B0000110801C0990007820F080008030099987
:1019C00008709DF8AC1001EB4100C0EBC1108F49CD
:1019D00001EBC000C27D9DF8AC0000EB8000914996
:1019E00001EB4020C0309DF8981001EB810303EB20
:1019F000411100EB810080F83C209DF8AC1001EB18
:101A0000410000EB0110864901EB0010C1798648C6
:101A100080F8B811F6E09DF8AC1001EB4100C0EB86
:101A2000C1107A4901EBC000C0799DF8AC1001EB00
:101A30004102C2EBC111754A02EBC101097A40EAC9
:101A40000120C217CDE92C029DF8AC1001EB41003A
:101A5000C0EBC1106D4901EBC00109910721099844
:101A6000F7F71CFF0022CDE92E022DA819C82C99EA
:101A70005940604001437BD19DF8AC1001EB41001F
:101A8000C0EBC110614911F83000401EC1B226916F
:101A90000021664A9DF8AC0002EB00100170A2F62E
:101AA000BF229DF8980011549DF8AC1001EB410045
:101AB000C0EBC110554901EBC00081790846019186
:101AC000F6F7A6FDCDE902019DED021B9FED580B37
:101AD00018F02EFF8DED060B9DF8AC1001EB4100C8
:101AE000C0EBC110494901EBC00001799DF8AC0081
:101AF00000EB4002C2EBC010444A02EBC000C078C9
:101B000041EA002000EE100AB8EEC00A8DED030A8B
:101B10000398F6F703FECDE904019DED060B53ECA7
:101B2000102B9DED040B51EC100BF6F7DBFCCDE90F
:101B300008019DED080B51EC100BF6F702FE324A3E
:101B40009DF8981002EB011148601FEDD40A10EEC9
:101B5000100A9DF8981002EB011108601FEDD90AD8
:101B600010EE100A9DF8981002EB0111886000E059
:101B700047E01FEDDE0A10EE100A9DF8981002EB08
:101B80000111C8609DF8AC1001EB410000EB0110A1
:101B9000234901EB001030309DF8981000EB011044
:101BA000801C0990007820F080008030099908702E
:101BB0009DF8AC1001EB4100C0EBC110134901EBE3
:101BC000C000427A9DF8AC0000EB8000154901EBA3
:101BD0004020C0309DF8981001EB810303EB4111C8
:101BE00000EB810080F83C209DF8AC1001EB410037
:101BF00000EB01100A4901EB0010C1790A4880F896
:101C0000B81100BF00BF0DE481340020347C0020F7
:101C10000000000000003040000000000000000054
:101C200000410020C0450020BC320020343F00208D
:101C300000000000000024409DF8AC1001EB4100C2
:101C4000C0EBC110FE4901EBC000C1789DF8AC00AB
:101C500000EB4002C2EBC010F94A02EBC0008078F2
:101C600041EA002127919DF8AC1001EB4100C0EB47
:101C7000C110114601EBC001BDF89C00401C095C7D
:101C80009DF8AC0000EB4002C2EBC010EC4A02EB46
:101C9000C002BDF89C00105C41EA0020C217CDE9EB
:101CA0002C029DF8AC1001EB4100C0EBC110E449DF
:101CB00001EBC0000990BDF89C10F7F7EFFD002282
:101CC000CDE92E022DA819C82C9959406040014336
:101CD0007ED19DF8AC1001EB4100C0EBC110D8499A
:101CE00001EBC00041782691002137911CE09DF85E
:101CF000AC1001EB410000EB0110D24901EB0011E7
:101D00003031BDF8DC0001EB001041789DF89800FF
:101D1000814204D1BDF8DC00C1B2269112E0BDF8C9
:101D2000DC00401C81B237919DF8AC1001EB410002
:101D300000EB0110C34901EB0010C179BDF8DC00D4
:101D40008142D4DC00BF9DF8AC1001EB410000EBF8
:101D50000110BC4901EB001030309DF8981000EBE9
:101D60000110801C0990007820F0800080300999D3
:101D700008709DF8AC1001EB4100C0EBC110B049F8
:101D800001EBC000007924900020AF4A9DF8AC1010
:101D900002EB01129DF8981050549DF8AC1001EB25
:101DA000410000EB0110A74901EB001030309DF815
:101DB000981000EB0110801C0990007820F0400082
:101DC000403009990870BDF89000F2287DD000E0FD
:101DD000FDE306DC052879D0062809D0F12876D164
:101DE000F6E3F32874D0F42873D0F628F7D1F0E3A3
:101DF0000621109100213491ECE3BDF84000401C15
:101E000081B210919DF8AC1001EB4100C0EBC11004
:101E10008B4901EBC001BDF84000095C2491BDF87D
:101E20004000401C81B21091BDF89000F12804D010
:101E3000F2287CD0F3287BD1FDE39DF8AC1001EBB8
:101E40004100C0EBC1107E4901EBC001BDF840006C
:101E5000095C2791BDF84000401C81B210919DF8AB
:101E6000AC1001EB410000EB0110764901EB0011D1
:101E700030319DF89820BDF8D000104401EB0010DF
:101E8000407A00F0010028B39DF8AC0000EB800020
:101E90006E4901EB4021C0319DF89820BDF8D0007B
:101EA000104400EB800202EB401001EB800090F840
:101EB0008E0000F0010068B99DF8AC0000EB8000D6
:101EC000624901EB4021C03105E0FDE3FDE3FDE3A4
:101ED000FDE3FDE34CE09DF89820BDF8D0001044F0
:101EE00000EB800202EB401001EB800090F88000D4
:101EF000F0B3002137912FE09DF8AC0000EB80009B
:101F0000524901EB4021C0319DF89820BDF8D00026
:101F1000104400EB800202EB401001EB800000F166
:101F20008101BDF8DC000A5C9DF8AC0001E0A1E392
:101F30009FE300EB400101EB0010424901EB001070
:101F40000E30BDF8DC10405C824200D008E0BDF8E5
:101F5000DC00401C81B23791BDF8DC000428CBDBEB
:101F600000BFBDF8DC00042854D1042137912DE0D6
:101F700050E09DF8AC0000EB8000344901EB4021BB
:101F8000C0319DF89820BDF8D000104400EB8002CD
:101F900002EB401001EB800000F18101BDF8DC0094
:101FA0000A5C9DF8AC0000EB400101EB00102549F4
:101FB00001EB00100E30BDF8DC10405C824200D016
:101FC00008E0BDF8DC00401C81B23791BDF8DC00B0
:101FD0000A28CEDB00BFBDF8DC000A281AD09DF825
:101FE000AC0000EB8000194901EB4020C0309DF8A7
:101FF0009820BDF8D010114401EB810202EB411191
:1020000000EB81008E300990007820F00100401C28
:1020100009990870BDF89C000F287CD19DF8AC1080
:1020200001EB410000EB0110064901EB00113031DA
:102030009DF89820BDF8D000104401EB001007E097
:10204000347C002000410020343F0020C0450020A7
:10205000801C0990007820F00400001D0999087088
:10206000002037902AE09DF8AC1001EB4100C0EB56
:10207000C110FE4901EBC001BDF84020BDF8DC00F5
:1020800010440A5C9DF8AC0000EB8000F84901EBBD
:102090004021C0319DF89830BDF8D000184400EBC5
:1020A000800303EB401001EB80013F31BDF8DC0001
:1020B0000A54BDF8DC00401C81B23791BDF8DC0049
:1020C0000A28D0DBBDF840000A3081B2109100210F
:1020D00037912CE09DF8AC1001EB4100C0EBC11032
:1020E000E24901EBC001BDF84020BDF8DC0010441E
:1020F0000A5C9DF8AC0000EB8000DD4901EB40215B
:10210000C0319DF89830BDF8D000184400EB800332
:1021100003EB401000E04AE201EB80015831BDF8CA
:10212000DC000A54BDF8DC00401C81B23791BDF8D8
:10213000DC000228CEDBBDF84000801C81B210918B
:102140009DF8AC1001EB4100C0EBC110C74901EB99
:10215000C001BDF84000085C01049DF8AC0000EB34
:102160004002C2EBC010C14A02EBC002BDF8400001
:10217000401C105C41EA00219DF8AC0000EB4002DD
:10218000C2EBC010B94A02EBC002BDF84000801C8F
:10219000105C01439DF8AC0000EB8000B44A02EBF8
:1021A0004022C0329DF89830BDF8D000184400EBB2
:1021B000800303EB401002EB8000C166BDF84000D5
:1021C000C01C81B21091AB4890F88C08F0BB002184
:1021D00037911DE09DF8AC0000EB8000A44901EBB5
:1021E0004021C0319DF89820BDF8D000104400EB8C
:1021F000800202EB401001EB80003F30BDF8DC10A4
:10220000405C00B108E0BDF8DC00401C81B23791B1
:10221000BDF8DC000A28DDDB00BFBDF8DC000A28C1
:1022200018D140229DF8AC0000EB8000904901EBF2
:102230004021C0319DF89830BDF8D000184400EB23
:10224000800303EB401001EB800000E055E080F8D4
:1022500076204DE19DF8AC0000EB8000844901EB55
:102260004021C0319DF89820BDF8D000104400EB0B
:10227000800202EB401001EB800090F87600E0BB9A
:10228000002128910EE10021359129E09DF8AC0054
:1022900000EB8000764901EB4021C0319DF8982089
:1022A000BDF8D000104400EB800202EB401001EBBF
:1022B00080013F31BDF8D400001D095C9DF8A000ED
:1022C00000EB40026C4800EB4202BDF8D400105C09
:1022D000814200D008E0BDF8D400401C81B23591A5
:1022E000BDF8D4000628D1DB00BFBDF8D400062815
:1022F0007ED103229DF8AC0000E0F9E000EB800005
:102300005B4901EB4021C0319DF89830BDF8D00009
:10231000184400EB800303EB401001EB800080F8D1
:1023200076209DF8AC1001EB410000EB0110534901
:1023300001EB001130319DF89820BDF8D000104419
:1023400001EB0010801C0990007820F0040209982D
:102350000270002037901CE020229DF8AC0000EBBA
:102360008000434901EB4021C0319DF89830BDF811
:10237000D000184400EB800303EB401001EB800118
:102380004931BDF8DC000A54BDF8DC00401C81B2C4
:102390003791BDF8DC000F28DEDB002137911CE00F
:1023A00020229DF8AC0000EB8000314901EB402178
:1023B000C0319DF89830BDF8D000184400EB800380
:1023C00003EB401001EB80015B31BDF8DC000A54E7
:1023D000BDF8DC00401C81B23791BDF8DC000A2852
:1023E000DEDB00229DF8AC0000EB8000204900E01D
:1023F00053E001EB4021C0319DF89830BDF8D0008A
:10240000184400EB800303EB401001EB800080F8E0
:102410007020002137911CE000229DF8AC0000EBF9
:102420008000134901EB4021C0319DF89830BDF880
:10243000D000184400EB800303EB401001EB800157
:102440007131BDF8DC000A54BDF8DC00401C81B2DB
:102450003791BDF8DC000528DEDB9DF8AC0000EB11
:102460008000034901EB4021C03109E0347C0020A9
:10247000C0450020BC32002044350020004100202F
:102480009DF89820BDF8D000104400EB800202EBCC
:10249000401001EB8000C06E0CE09DF8A000401CD5
:1024A000C1B22891FB48B0F886129DF8A000814285
:1024B0003FF7E9AE00BFF748B0F886129DF8A000DC
:1024C000814215D140229DF8AC0000EB8000F2491A
:1024D00001EB4021C0319DF89830BDF8D000184480
:1024E00000EB800303EB401001EB800080F87620C6
:1024F0009DF8AC0000EB8000E74901EB4021C031C2
:102500009DF89820BDF8D000104400EB800202EB4B
:10251000401001EB800090F87600032804D01128C9
:1025200018D0402842D12BE0F2229DF8AC0000EBFD
:102530008000D94901EB4021C0319DF89830BDF8A9
:10254000D000184400EB800303EB401001EB800047
:1025500042712BE0F3229DF8AC0000EB8000CE49E5
:1025600001EB4021C0319DF89830BDF8D0001844EF
:1025700000EB800303EB401001EB8000427115E09B
:10258000F2229DF8AC0000EB8000C34901EB402132
:10259000C0319DF89830BDF8D000184400EB80039E
:1025A00003EB401001EB8000427100BF61E09DF839
:1025B000AC0000EB400101EB0010B84901EB00104A
:1025C00030309DF89820BDF8D010114403E0EAE3C4
:1025D000C7E0E9E3B5E000EB0110801C099000784A
:1025E00020F00402099802709DF8AC0000EB800016
:1025F000A94901EB4021C0319DF89820BDF8D000D9
:10260000104400EB800202EB401001EB800090F8D8
:102610008E0000F0010060B300229DF8AC0000EBDA
:1026200080009D4901EB4021C0319DF89830BDF8F4
:10263000D000184400E068E000EB800303EB40109A
:1026400001EB8000A0F88C2005229DF8AC0000EB87
:102650008000914901EB4021C0319DF89830BDF8D0
:10266000D000184400EB800303EB401001EB800026
:10267000427160E09DF8AC0000EB8000864901EB00
:102680004021C0319DF89820BDF8D000104400EBE7
:10269000800202EB401001EB800090F876004028A9
:1026A0001CD100229DF8AC0000EB80007A4901EBC0
:1026B0004021C0319DF89830BDF8D000184400EB9F
:1026C000800303EB401004E0F0E3F0E3F0E3F0E319
:1026D000F0E301EB800080F8762000BF00BFF1221C
:1026E0009DF8AC0000EB80006B4901EB4021C0314C
:1026F0009DF89830BDF8D000184400EB800303EB40
:10270000401001EB8000427115E0F1229DF8AC0011
:1027100000EB8000604901EB4021C0319DF898300A
:10272000BDF8D000184400EB800303EB401001EB30
:102730008000427100BF00BFBDF8D000401C81B2D4
:1027400034919DF8AC0000EB4001C1EBC01054493E
:1027500001EBC0004179BDF8D00081423FF74DAB9D
:10276000A6E39DF8AC0000EB80004B4901EB402054
:10277000C0309DF8981001EB810202EB411110F876
:10278000210018BB01229DF8AC0000EB80004249FB
:1027900001EB4021C0319DF8980000EB800303EB72
:1027A000401001F82020F4229DF8AC0000EB8000DE
:1027B000394901EB4020C0309DF8981001EB8103AE
:1027C00003EB411100EB81004271C6E09DF8AC00C3
:1027D00000EB400101EB0010304901EB00103030FC
:1027E0009DF8981000EB0110407A00F00100E8B36A
:1027F0009DF8AC0000EB8000274901EB4020C03081
:102800009DF8981001EB810202EB411100EB810071
:1028100090F88E0000F0010040BB9DF8AC0000EB8A
:1028200080001D4901EB4020C0309DF8981001EB5D
:10283000810202EB411100EB810090F88000A8B109
:102840000020379033E09DF8AC0000EB8000124987
:1028500001EB4021C0319DF8980000EB800202EBB3
:10286000401001EB800000F1810100E075E0BDF84F
:10287000DC000A5C9DF8AC0000EB400101EB0010AD
:10288000064901EB00100E30BDF8DC10405C8242BE
:1028900008D010E0BC320020C045002000410020DC
:1028A000347C0020BDF8DC00401C81B23791BDF8BB
:1028B000DC000428C7DB00BFBDF8DC0004284CD1D5
:1028C000379029E09DF8AC0000EB8000FE4901EB59
:1028D0004021C0319DF8980000EB800202EB4010CF
:1028E00001EB800000F18101BDF8DC000A5C9DF87D
:1028F000AC0000EB400101EB0010F44901EB0010CB
:102900000E30BDF8DC10405C824200D008E0BDF81B
:10291000DC00401C81B23791BDF8DC000A28D1DB15
:1029200000BFBDF8DC000A2817D09DF8AC0000EB12
:102930008000E54901EB4020C0309DF8981001EB84
:10294000810202EB411100EB81008E30099000788A
:1029500020F00100401C09990870BDF89C00112866
:1029600071D19DF8AC0000EB400101EB0010D7499C
:1029700001EB001030309DF8981000EB0110801C26
:102980000990007820F00400001D099908700020CB
:10299000379025E09DF8AC0000EB4001C1EBC01082
:1029A000CB4901EBC001BDF8DC00401D0A5C9DF87D
:1029B000AC0000EB8000C44901EB4021C0319DF820
:1029C000980000EB800303EB401001EB80013F31E6
:1029D000BDF8DC000A54BDF8DC00401C81B2379120
:1029E000BDF8DC000A28D5DB0020379025E09DF8F3
:1029F000AC0000EB4001C1EBC010B54901EBC001D8
:102A0000BDF8DC000F300A5C9DF8AC0000EB8000E4
:102A1000AD4901EB4021C0319DF8980000EB8003E7
:102A200003EB401001EB80015831BDF8DC000A5483
:102A3000BDF8DC00401C81B23791BDF8DC000228F3
:102A4000D5DBC1E2FFE7BDF89C0014287DD19DF8DD
:102A5000AC0000EB400101EB00109C4901EB0010C1
:102A600030309DF8981000EB0110801C0990007820
:102A700020F00400001D099908700020379025E01F
:102A80009DF8AC0000EB4001C1EBC010904901EB98
:102A9000C001BDF8DC00401D0A5C9DF8AC0000EBF5
:102AA0008000894901EB4021C0319DF8980000EB7E
:102AB000800303EB401001EB80013F31BDF8DC00E7
:102AC0000A54BDF8DC00401C81B23791BDF8DC002F
:102AD0000A28D5DB0020379025E09DF8AC0000EBFC
:102AE0004001C1EBC0107A4901EBC001BDF8DC0028
:102AF0000F300A5C9DF8AC0000EB8000724901EBDE
:102B00004021C0319DF8980000EB800303EB40109A
:102B100001EB80015831BDF8DC000A54BDF8DC003F
:102B2000401C81B23791BDF8DC000228D5DB9DF84E
:102B3000AC0000EB4001C1EBC010654901EBC000E7
:102B4000407C01049DF8AC0000E0EEE100EB4002A7
:102B5000C2EBC0105E4A02EBC000807C41EA00215B
:102B60009DF8AC0000EB4002C2EBC010584A02EBEB
:102B7000C000C07C01439DF8AC0000EB8000524ACD
:102B800002EB4020C0309DF8982002EB820303EB5B
:102B9000421200EB8200C1664E4890F88C08C8BB18
:102BA000002037901AE09DF8AC0000EB8000464909
:102BB00001EB4021C0319DF8980000EB800202EB50
:102BC000401001EB80003F30BDF8DC10405C00B1EC
:102BD00008E0BDF8DC00401C81B23791BDF8DC0094
:102BE0000A28E0DB00BFBDF8DC000A2813D1402230
:102BF0009DF8AC0000EB8000334901EB4020C03071
:102C00009DF8981001EB810303EB411100EB81006B
:102C100080F8762031E19DF8AC0000EB80002A4975
:102C200001EB4020C0309DF8981001EB810202EBCF
:102C3000411100EB810090F87600E0BB0020289065
:102C4000F8E00020359026E09DF8AC0000EB800015
:102C50001D4901EB4021C0319DF8980000EB800236
:102C600002EB401001EB80013F31BDF8D400001DA4
:102C7000095C9DF8A00000EB4002174800EB4202FF
:102C8000BDF8D400105C814200D008E0BDF8D4004B
:102C9000401C81B23591BDF8D4000628D4DB00BFBA
:102CA000BDF8D40006287DD103229DF8AC0000EBCE
:102CB0008000054900E0E0E001EB4021C0319DF8D3
:102CC000980000EB800309E0C0450020004100208F
:102CD000347C0020BC3200204435002003EB40103F
:102CE00001EB800080F876209DF8AC0000EB4001FD
:102CF00001EB0010FE4901EB001130319DF8980006
:102D000001EB0010801C0990007820F00402099863
:102D100002700020379019E020229DF8AC0000EBF3
:102D20008000F44901EB4021C0319DF8980000EB90
:102D3000800303EB401001EB80014931BDF8DC005A
:102D40000A54BDF8DC00401C81B23791BDF8DC00AC
:102D50000F28E1DB0021379119E020229DF8AC001B
:102D600000EB8000E34901EB4021C0319DF8980061
:102D700000EB800303EB401001EB80015B31BDF8F9
:102D8000DC000A54BDF8DC00401C81B23791BDF86C
:102D9000DC000A28E1DB00229DF8AC0000EB80009B
:102DA000D44902E041E0AFE25EE101EB4021C031F5
:102DB0009DF8980000EB800303EB401001EB8000CE
:102DC00080F870200021379119E000229DF8AC00B6
:102DD00000EB8000C74901EB4021C0319DF898000D
:102DE00000EB800303EB401001EB80017131BDF873
:102DF000DC000A54BDF8DC00401C81B23791BDF8FC
:102E0000DC000528E1DB9DF8AC0000EB8000B9494F
:102E100001EB4020C0309DF8981001EB810202EBDD
:102E2000411100EB8100C06E0CE09DF8A000401C39
:102E3000C1B22891B048B0F886129DF8A000814236
:102E40003FF7FFAE00BFAC48B0F886129DF8A00077
:102E5000814212D140229DF8AC0000EB8000A549D0
:102E600001EB4020C0309DF8981001EB810303EB8B
:102E7000411100EB810080F876209DF8AC0000EB5A
:102E800080009C4901EB4020C0309DF8981001EB78
:102E9000810202EB411100EB810090F876000328DB
:102EA00009D011281AD040283ED12AE08DE0BAE19D
:102EB00029E2C6E0FCE0F2229DF8AC0000EB8000C5
:102EC0008C4901EB4020C0309DF8981001EB810344
:102ED00003EB411100EB8100427125E0F3229DF8E4
:102EE000AC0000EB8000834901EB4020C0309DF82E
:102EF000981001EB810303EB411100EB810042715B
:102F000012E0F2229DF8AC0000EB8000794901EB61
:102F10004020C0309DF8981001EB810303EB411174
:102F200000EB8100427100BF4EE09DF8AC1001EB58
:102F3000410000EB01106E4901EB001030309DF8AC
:102F4000981000EB0110801C0990007820F004021A
:102F5000099802709DF8AC0000EB8000654901EB18
:102F60004020C0309DF8981001EB810202EB411126
:102F700000EB810090F88E0000F0010020B30022E9
:102F80009DF8AC0000EB80005A4901EB4021C031B4
:102F90009DF8980000EB800303EB401001EB8000EC
:102FA000A0F88C2005229DF8AC0000EB8000514970
:102FB00001EB4020C0309DF8981001EB810303EB3A
:102FC000411100EB810042719DE19DF8AC0000EBE6
:102FD0008000484901EB4020C0309DF8981001EB7B
:102FE000810202EB411100EB810090F8760040284D
:102FF00013D100229DF8AC0000EB80003D4901EBAD
:103000004020C0309DF8981001EB810303EB411183
:1030100000EB810080F8762000BF00BFF1229DF810
:10302000AC0000EB8000334901EB4020C0309DF83C
:10303000981001EB810303EB411100EB8100427119
:1030400061E1F1229DF8AC0000EB8000294901EB21
:103050004020C0309DF8981001EB810303EB411133
:1030600000EB810042714EE103229DF8AC0000EBC1
:103070008000204901EB4021C0319DF8980000EB11
:10308000800303EB401001F82020F1229DF8AC00F2
:1030900000EB8000174901EB4020C0309DF89810EC
:1030A00001EB810303EB411100EB810042712AE146
:1030B00002229DF8AC0000EB80000E4901EB40219C
:1030C000C0319DF8980000EB800303EB401001F83D
:1030D0002020F6229DF8AC0000EB8000054901EBB2
:1030E0004021C0319DF8980000EB800306E000000D
:1030F00000410020C0450020BC32002003EB4010FE
:1031000001EB8000427101229DF8AC0000EB8000D1
:10311000FE4901EB4021C0319DF8980000EB80038F
:1031200003EB401001EB800080F8802000213791F4
:1031300026E09DF8AC1001EB4100C0EBC110F44952
:1031400001EBC001BDF8DC00401D0A5C9DF8AC003D
:1031500000EB8000ED4901EB4021C0319DF8980063
:1031600000EB800303EB401001EB800000F18101D4
:10317000BDF8DC000A54BDF8DC00401C81B2379178
:10318000BDF8DC000A28D4DBBDF89C00142849D126
:103190009DF8AC1001EB4100C0EBC110DC4901EB24
:1031A000C000C27B9DF8AC0000EB8000D74901EB6A
:1031B0004021C0319DF8980000EB800303EB4010E4
:1031C00001EB800080F877200021379126E09DF800
:1031D000AC1001EB4100C0EBC110CD4901EBC001C7
:1031E000BDF8DC0010300A5C9DF8AC0000EB8000FC
:1031F000C64901EB4021C0319DF8980000EB8003E7
:1032000003EB401001EB800000F17901BDF8DC0018
:103210000A54BDF8DC00401C81B23791BDF8DC00D7
:103220000428D4DB6FE09DF8AC1001EB4100C0EB4B
:10323000C110B74901EBC00081799DF8AC0000EBEB
:103240004002C2EBC010B24A02EBC000407941EA32
:1032500000229DF8AC0000EB8000AC4901EB40215E
:10326000C0319DF8980000EB800303EB401001EBA8
:103270008000A0F88C209DF8AC0000EB8000A349F2
:1032800001EB4021C0319DF8980000EB800202EB79
:10329000401001EB8000B0F88C109DF8AC0000EB02
:1032A000400202EB00109B4A02EB0010408B81426F
:1032B00028DBF1229DF8AC0000EB8000934901EB84
:1032C0004021C0319DF8980000EB800303EB4010D3
:1032D00001EB800042719DF8AC0000EB80008B494F
:1032E00001EB4021C0319DF8980000EB800202EB19
:1032F000401001EB80008E300990007820F0010230
:103300000998027000BF00BF02F090BF9DF8AC109A
:1033100001EB4100C0EBC1107D4901EBC000017918
:103320002691002134911CE09DF8AC1001EB410086
:1033300000EB0110774901EB00113031BDF8D000EE
:1033400001EB001041789DF89800814204D1BDF84E
:10335000D000C1B2269112E0BDF8D000401C81B26D
:1033600034919DF8AC1001EB410000EB011069496C
:1033700001EB0010C179BDF8D0008142D4DC00BF60
:103380009DF8AC1001EB410000EB0110614901EB2D
:10339000001030309DF8981000EB0110801C09904F
:1033A000007820F040004030099908709DF8AC107A
:1033B00001EB4100C0EBC110554901EBC000C078E2
:1033C0002490BDF89000172834D2DFE800F0330CC9
:1033D0000F331215181B1E33333333333321242795
:1033E00033332A2D30000721279123E0072127912D
:1033F00020E0062027901DE0062127911AE00621F3
:10340000279117E01221279114E00720279011E05F
:10341000092127910EE0062127910BE00621279133
:1034200008E00B21279105E00B21279102E02A21DA
:10343000279100BF00BFBDF89C00001FC1B20991D9
:103440009DF8AC1001EB4100C0EBC110304901EB1D
:10345000C000C01C08900999F6F73CF835909DF81B
:10346000AC1001EB4100C0EBC110294901EBC001D8
:10347000BDF89C00401E095CBDF8D40081427DD19E
:103480009DF8AC1001EB4100C0EBC110204901EBED
:10349000C0004078002871DD9DF8AC1001EB4100C0
:1034A000C0EBC1101A4901EBC001BDF89C000A5CD9
:1034B0009DF8AC0000EB8000144901EB4021C031C5
:1034C0009DF8980000EB800303EB401001EB8000B7
:1034D00080F83C200021104A9DF8AC0002EB00125D
:1034E0009DF8980011540D48007F012820D19DF8C7
:1034F000AC1001EB410000EB0110064901EB00109C
:1035000030309DF8981000EB011009E0C045002014
:10351000347C002000410020343F0020BC120020F9
:10352000801C0990007820F0800080300999087094
:10353000BDF8900007287CD00ADC07287AD2DFE8A3
:1035400010F07900C7041B057900B40481045F09F9
:1035500010380728F2D2DFE810F0B0099D096D009D
:103560006D0007000800410500BFBDF89000142859
:103570007ED19DF8AC0000EB400100E0FEE3C1EB22
:10358000C010FE4901EBC000407901069DF8AC0077
:1035900000EB4002C2EBC010F84A02EBC000807999
:1035A00041EA00419DF8AC0000EB4002C2EBC010C4
:1035B000F24A02EBC000C07941EA00219DF8AC005C
:1035C00000EB4002C2EBC010EC4A02EBC000007AF4
:1035D00001439DF8AC0000EB8000E94A02EB402279
:1035E000C0329DF8980000EB800303EB401002EB23
:1035F0008000C0F81A109DF8AC0000EB8000E04994
:1036000001EB4021C0319DF8980000EB800202EBF5
:10361000401001EB8000D0F81A10084609910021F3
:1036200009F068FDCDE92C019DF8AC0000EB4001EC
:1036300001E0FDE3FDE301EB0010D24901EB0010D6
:10364000007F00F003019DF8AC0000EB400202EBAC
:103650000010CC4A02EB0010007FC0F301100144BF
:103660009DF8AC0000EB400202EB0010C54A00E000
:1036700061E002EB0010007FC0F38100091A0846E8
:103680000591F4F7B4FFCDE906019DED061B9FED12
:10369000BE0B17F04DF98DED080B9DED080B51ECAD
:1036A000100BF5F716F8CDE92E019DF8AC0000EBF4
:1036B0008000B34901EB4021C0319DF8980000EB38
:1036C000800202EB401001EB8000416B084607913D
:1036D000002109F00FFDDDE92C32A0FB034501FBC1
:1036E000035100FB021502220023DDE92E01F4F74D
:1036F00069FD20186941CDE90801DDE92E23F4F7C1
:1037000061FDCDE92C01DDE92C010AF0A7FA0146A3
:103710009DF8AC0000EB8000994A02EB4020C030DD
:103720009DF8982002EB820303EB421200EB82002B
:10373000C0F81E1043E0BDF8900015283FD19DF859
:10374000AC0000EB4001C1EBC0108C4901EBC000A4
:10375000407901069DF8AC0000EB4002C2EBC010BE
:10376000864A02EBC000807941EA00419DF8AC0036
:1037700000EB4002C2EBC010804A02EBC000C079EF
:1037800041EA00219DF8AC0000EB4002C2EBC01002
:103790007A4A02EBC000007A01439DF8AC0000EBCE
:1037A0008000774A02EB4020C0309DF8982002EB61
:1037B000820303EB421200EB8200C0F81E109DF85A
:1037C000AC0000EB4001C1EBC0106C4901EBC00044
:1037D000417A6F4880F80F1E9DF8AC0000EB400165
:1037E00001EB0010674901EB001130319DF89800A2
:1037F00001EB0010801C0990654890F80F0EC2097B
:103800000998007862F3000009990870604890F800
:103810000F0E00F00300012806D05D4890F80F0E4F
:1038200000F0030003282BD19DF8AC0000EB400111
:1038300001EB0010534901EB001030309DF8981057
:1038400000EB0110801C0990007820F00201891C17
:10385000099801709DF8AC0000EB400101EB0010ED
:10386000484901EB001130319DF8980001EB001040
:10387000801C0990007820F020020998027014E062
:103880009DF8AC0000EB400101EB00103D4901EB5D
:10389000001030309DF8981000EB0110801C09904A
:1038A000007820F00202099802709DF8AC0000EB4D
:1038B000400101EB0010334901EB001130319DF85C
:1038C000980001EB00108078C0F340029DF8AC0036
:1038D00000EB80002A4901EB4020C0309DF8981091
:1038E00001EB810303EB411100EB8100007EC0F38B
:1038F0004000824274D09DF8AC0000EB800020496B
:1039000001EB4020C0309DF8981001EB810202EBE2
:10391000411100EB8100183009909DF8AC0000EBDC
:10392000400101EB0010174901EB001030309DF809
:10393000981000EB0110807842080998007862F333
:103940004100099908709DF8AC0000EB400101EBC3
:1039500000100C4901EB001030309DF8981000EB7E
:1039600001108078C0F34000A8BB9DF8AC0000EBCC
:10397000400101EB001003490CE00000347C002002
:10398000C04500200041002000000000000024404D
:10399000BC22002001EB001030309DF8981000EBA5
:1039A0000110801C0990007820F020020998027014
:1039B00001229DF8AC0000EB8000FE4901EB4020A5
:1039C000C0309DF8981001EB810303EB411100EB2F
:1039D000810080F83E209DF8AC100220F6F7B8FA7E
:1039E0009DF8AC0000EB400101EB0010F24901EB47
:1039F000001130319DF8980001EB0010807800F044
:103A000001029DF8AC0000EB8000EA4901EB402088
:103A1000C0309DF8981001EB810303EB411100EBDE
:103A20008100007E00F0010082425FD09DF8AC0072
:103A300000EB8000DF4901EB4020C0309DF898107A
:103A400001EB810202EB411100EB8100183009907B
:103A50009DF8AC0000EB400101EB0010D64901EBF2
:103A6000001030309DF8981000EB01108078099913
:103A70000A7860F300020A709DF8AC0000EB400188
:103A800001EB0010CC4901EB001030309DF898108C
:103A900000EB0110807800F0010040BB9DF8AC0005
:103AA00000EB400101EB0010C34901EB0010303086
:103AB0009DF8981000EB0110801C0990007820F010
:103AC00020020998027000229DF8AC0000EB8000F3
:103AD000B84901EB4020C0309DF8981001EB8103FC
:103AE00003EB411100EB810080F83D2006E19DF8D9
:103AF000AC0000EB8000AF4901EB4020C0309DF8E6
:103B0000981001EB810202EB411100EB810090F86B
:103B10003E0098B901229DF8AC0000EB8000A54959
:103B200001EB4020C0309DF8981001EB810303EBBE
:103B3000411100EB810080F83D2027E000229DF834
:103B4000AC0000EB80009B4901EB4021C0319DF8A7
:103B5000980000EB800303EB401001EB800080F83D
:103B60003D209DF8AC0000EB400101EB00109249B4
:103B700001EB001030309DF8981000EB0110801C14
:103B80000990007820F00102099802708B4890F8A3
:103B90008C08E0BB8A48407F012838D18848D0F89B
:103BA00014028749C98B884231D29DF8AC0000EBE2
:103BB0008000804901EB4020C0309DF8981001EB57
:103BC000810202EB411100EB810090F83D000128D9
:103BD0001DD19DF8AC0000EB8000764901EB402040
:103BE000C0309DF8981001EB810202EB411100EB0F
:103BF000810090F87D0050B99DF8AC0000EB4001C9
:103C000001EB00106C4901EB0011303100E075E070
:103C10009DF8980001EB001001789DF8AC0000EBD6
:103C20008000644A02EB4020417005229DF8AC0000
:103C300000EB80005F4901EB4021C0319DF8980006
:103C400000EB800303EB401001EB80004271002287
:103C50009DF8AC0000EB400101EB0010564901EB70
:103C6000001130319DF8980001EB001042609DF882
:103C7000AC100220F6F76CF90021379119E0002210
:103C80009DF8AC0000EB80004A4901EB4021C031B7
:103C90009DF8980000EB800303EB401001EB8001DE
:103CA0003F31BDF8DC000A54BDF8DC00401C81B295
:103CB0003791BDF8DC001428E1DB0021379119E0D1
:103CC00000229DF8AC0000EB80003A4901EB402156
:103CD000C0319DF8980000EB800303EB401001EB2E
:103CE00080015B31BDF8DC000A54BDF8DC00401CEB
:103CF00081B23791BDF8DC000A28E1DB9DF8AC0009
:103D000000EB80002B4901EB4020C0309DF898105B
:103D100001EB810202EB411110F82100012811DCB6
:103D200002229DF8AC0000EB8000224901EB40200C
:103D3000C0309DF8981001EB810303EB411100F8AE
:103D400021207EE09DF8AC0000EB8000194901EBDA
:103D50004020C0309DF8981001EB810202EB411128
:103D600010F82100022837DC00219DF8AC0000EBA0
:103D70008000104A02EB4020C17000E0FEE3032205
:103D80009DF8AC0000EB80000A4901EB4021C031F6
:103D90009DF8980000EB800303EB401001F8202011
:103DA00007229DF8AC0000EB8000024901EB4020A7
:103DB000C03007E0C045002000410020BC32002098
:103DC000BC1200209DF8981001EB810303EB411118
:103DD00000EB8100427134E09DF8AC0000EB800004
:103DE000FE4901EB4021C0319DF8980000EB8002B4
:103DF00002EB401011F820109DF8AC0000EB8000A1
:103E0000F64A02EB4020007981421AD1F44890F83A
:103E10000F0EC0F34010A0B116229DF8AC0000EBCD
:103E20008000EE4901EB4020C0309DF8981001E081
:103E3000A2E1D8E301EB810303EB411100EB810028
:103E40004271D0E314229DF8AC0000EB8000E349FE
:103E500001EB4021C0319DF8980000EB800303EB9B
:103E6000401001EB8000427101219DF8AC0000EB95
:103E70008000DA4A02EB4020C1709DF8AC0000EBF4
:103E8000400101EB0010A2F5986101EB0010303009
:103E90009DF8981000EB0110801C0990007820F02C
:103EA00020002030099908709DE314229DF8AC0091
:103EB00000EB8000C94901EB4020C0309DF898100C
:103EC00001EB810303EB411100EB810042718AE3B6
:103ED0009DF8AC0000EB8000C04901EB4020C030F1
:103EE000BDF8D01001EB810202EB411100EB810023
:103EF0008079012824D100229DF8AC0000EB8000DD
:103F0000B64901EB4021C031BDF8D00000EB800381
:103F100003EB401001EB8000827114229DF8AC008D
:103F200000EB8000AD4901EB4020C0309DF89810B7
:103F300001EB810303EB411100EB810042711AE0B8
:103F400000219DF8AC0000EB8000A44A02EB402069
:103F5000C17005229DF8AC0000EB80009F4901EB89
:103F60004020C0309DF8981001EB810303EB411114
:103F700000EB8100427136E301219DF8AC0000EBBB
:103F80008000964A02EB4020C17014229DF8AC00DC
:103F900000EB8000914901EB4021C0319DF8980071
:103FA00000EB800303EB401001EB800042719DF8B1
:103FB000AC0000EB400101EB00108A4901EB00115D
:103FC00030319DF8980001EB0010801C09900078BA
:103FD00020F00400001D0999087004E300202C90D3
:103FE0002D90002137911EE0DDE92C10000240EAFF
:103FF00011620902CDE92C129DF8AC0000EB4001E2
:10400000C1EBC010784901EBC001BDF8DC00401DD8
:10401000085CDDE92C341843CDE92C04BDF8DC0044
:10402000401C80B23790BDF8DC000328DCDBDDE902
:104030002C0109F013FE01469DF8AC0000EB800056
:10404000664A02EB4022C0329DF8980000EB8003E4
:1040500003EB401002EB8000C0F81E1000222C92EF
:104060002D92002137911FE0DDE92C10000240EA7B
:1040700011620902CDE92C129DF8AC0000EB400161
:10408000C1EBC010584901EBC001BDF8DC0008309D
:10409000085CDDE92C3440EA0302CDE92C24BDF8AC
:1040A000DC00401C81B23791BDF8DC000328DBDB6B
:1040B000DDE92C0109F0D2FD01469DF8AC0000EBD2
:1040C0008000464A02EB4022C0329DF8980000EB87
:1040D000800303EB401002EB8000C0F81A100021AF
:1040E0002C912D9137911EE0DDE92C10000240EA61
:1040F00011620902CDE92C129DF8AC0000EB4001E1
:10410000C1EBC010384901EBC001BDF8DC00133031
:10411000085CDDE92C341843CDE92C04BDF8DC0043
:10412000401C80B23790BDF8DC000328DCDB9DF832
:10413000AC002C9900EB8000284A02EB4022C032F0
:104140009DF8980000EB800303EB401002EB800029
:10415000416307229DF8AC0000EB80001F4901EB92
:104160004020C0309DF8981001EB810303EB411112
:1041700000EB81004271B3E300202C902D900021D0
:1041800037911EE0DDE92C10000240EA11620902BD
:10419000CDE92C129DF8AC0000EB4001C1EBC01042
:1041A000114901EBC001BDF8DC00401D085CDDE9F0
:1041B0002C341843CDE92C04BDF8DC00401C80B23F
:1041C0003790BDF8DC000428DCDBDDE92C0109F0C8
:1041D00045FD9DF8AC2002EB820207E0C0450020BF
:1041E000BC22002000410020347C0020FE4B03EB69
:1041F0004223C0339DF8982002EB820404EB421264
:1042000003EB820222329060D16000212C912D912B
:10421000002037901FE0DDE92C10000240EA116217
:104220000902CDE92C129DF8AC0000EB4001C1EB76
:10423000C010EE4901EBC001BDF8DC000930085C9C
:10424000DDE92C3440EA0302CDE92C24BDF8DC0082
:10425000401C81B23791BDF8DC000428DBDBDDE9CE
:104260002C0109F0FBFC9DF8AC2002EB8202DE4B36
:1042700003EB4223C0339DF8982002EB820404EB49
:10428000421203EB820242F8220F51609DF8AC000B
:1042900000EB8000D44901EB4021C0319DF898002B
:1042A00000EB800202EB401011F820109DF8AC00EA
:1042B00000EB8000CC4A02EB4020007981426DD1B6
:1042C000CB4890F80F0EC0F3401090B117229DF824
:1042D000AC0000EB8000C44901EB4021C0319DF8E7
:1042E000980000EB800303EB401001EB800042716B
:1042F00011E014229DF8AC0000EB8000BA4901EBFC
:104300004020C0309DF8981001EB810303EB411170
:1043100000EB81004271B74890F88C08E8BB00229E
:104320009DF8AC0000EB8000AF4901EB4020C030AD
:104330009DF8981001EB810303EB411100EB810024
:1043400080F83E20AC48D0F814020521B0FBF1F211
:1043500001FB120000EBC00101EB0011A648203068
:1043600000EB81000021C0F81D10A348D0F8140212
:104370000521B0FBF1F201FB120000EBC00101EBE3
:1043800000119D48203000EB81000D3009909DF810
:10439000AC0000EB8000944901E0C7E0B8E101EB1C
:1043A0004020C0309DF8981001EB810202EB4111D2
:1043B00000EB810022301022014608900998F3F7A3
:1043C00044FF8D48D0F814020521B0FBF1F201FB47
:1043D000120000EBC00101EB00118748203000EB18
:1043E00081029DF8AC0000EB80007F4901EB402189
:1043F000C0319DF8980000EB800303EB401001EB07
:10440000800050F81A1F42F8011F406850607A4837
:10441000D0F814020521B0FBF1F201FB120000EB11
:10442000C00101EB0013744920319DF8AC0000EB92
:10443000400202EB0010714A02EB001230329DF88C
:10444000980002EB0010007801F823006A48D0F8C9
:1044500014020521B0FBF1F201FB120000EBC001D8
:1044600001EB00116448203000EB81029DF8AC00A4
:1044700000EB80005C4901EB4021C0319DF89800C1
:1044800000EB800303EB401001EB8000406BC2F8AF
:1044900009005948D0F814020521B0FBF1F201FBE4
:1044A000120000EBC00101EB00115348203000EB7B
:1044B00081015048826941F8212F808B88804E48C5
:1044C000D0F814020521B0FBF1F081B2022009916D
:1044D000F4F7FEFD00210620F5F73AFD4648D0F836
:1044E00014024549C98B884206D24348D0F81402C9
:1044F000401C4149C1F8140200210520F5F728FDB0
:104500009DF8AC0000EB400101EB00103B4901EBD2
:10451000001030309DF8981000EB0110801C0990BD
:10452000007820F00802099802702AE09DF8AC009B
:1045300000EB400101EB0010304901EB001030307E
:104540009DF8981000EB0110801C0990007820F075
:10455000080008300999087000229DF8AC0000EBB3
:104560008000214901EB4020C0309DF8981001EBFC
:10457000810303EB411100EB810000E0B1E180F821
:104580003E209DF8AC100220F5F7E2FC9DF8AC103F
:104590009DF8980000EB0110C217CDE92C02002213
:1045A0002C9800EBC00101EB0011154800EB8100D5
:1045B000C0F81D209DF8AC0000EB80000A4901EB1B
:1045C0004020C0309DF8981001EB810202EB4111B0
:1045D00000EB8100223009902C9800EBC00101EB28
:1045E000001107480EE07BE1C0450020347C00202C
:1045F000BC220020BC320020BC1200200041002060
:10460000E014002000EB81000D3010220890099981
:10461000F3F71BFE9DF8AC0000EB8000FE4901EBB8
:104620004021C0319DF8980000EB800202EB401061
:1046300001EB80012C9800EBC00202EB0012F7485E
:1046400000EB820051F81A2F40F8012F49684160B1
:104650009DF8AC0000EB400101EB0010F04901EBCC
:10466000001130319DF8980001EB001001782C9872
:1046700000EBC00202EB0012E84800F822102C9870
:1046800000EBC00101EB0011E44800EB8101E548BB
:10469000826941F8212F808B88809DF8AC0000EB67
:1046A0008000DD4901EB4021C0319DF8980000EB0E
:1046B000800202EB401001EB8000416B2C9800EB74
:1046C000C00202EB0012D54800EB8200C0F80910CE
:1046D0009DF8AC0000EB400101EB0010D04901EB6C
:1046E000001130319DF8980001EB001041682C98C2
:1046F00000EBC00202EB0012C84800EB8200C0F8D9
:1047000027102C9881B208200991F5F721FC76E05A
:104710009DF8AC0000EB8000BF4901EB4021C031A7
:104720009DF8980000EB800202EB401011F8201079
:104730009DF8AC0000EB8000B74A02EB4020007906
:1047400081425CDA9DF8AC0000EB400101EB001007
:10475000B34901EB001030309DF8981000EB0110C8
:10476000801C0990007820F00400001D0999087051
:104770009DF8AC0000EB400101EB0010A84901EBF3
:10478000001030309DF8981000EB0110801C09904B
:10479000007820F0800080300999087001209DF891
:1047A000AC1001EB810102EB4121C8709DF8AC0017
:1047B00000EB8000114601EB402002799DF8AC002F
:1047C00000EB800001EB4020C0309DF8981001EB19
:1047D000810303EB411100F8212014229DF8AC0065
:1047E00000EB80008C4901EB4020C0309DF8981010
:1047F00001EB810303EB411100EB810042716FE09B
:104800000121884880F8B0179DF8AC0000EB8000CB
:10481000814901EB4021C0319DF8980000EB8002F6
:1048200002EB401011F820109DF8AC0000EB800066
:10483000794A02EB4020007981422ADA00219DF872
:10484000AC0000EB800002EB4020C17001229DF81B
:10485000AC0000EB8000704901EB4021C0319DF8B5
:10486000980000EB800303EB401001F82020142295
:104870009DF8AC0000EB8000674901EB4020C030A0
:104880009DF8981001EB810303EB411100EB8100CF
:10489000427125E014229DF8AC0000EB80005E49D7
:1048A00001EB4020C0309DF8981001EB810303EB31
:1048B000411100EB8100427112E014229DF8AC001E
:1048C00000EB8000544901EB4020C0309DF8981067
:1048D00001EB810303EB411100EB8100427100BF4A
:1048E00000BFFCE39DF8AC0000EB80004A4901EBFF
:1048F0004020817826919DF8AC0000EB4001C1EB8F
:10490000C010494911F8301027919DF8AC0000EB18
:104910008000414901EB4021C0319DF8980000EB37
:10492000800202EB401001EB8000417924919DF858
:10493000AC0000EB4001C1EBC0103B4901EBC001F2
:104940000991BDF89C100998F6F78AF835909DF802
:10495000AC0000EB4001C1EBC010334901EBC001DA
:10496000BDF89C00095CBDF8D40081427DD19DF862
:10497000AC0000EB4001C1EBC0102B4901EBC000C3
:104980004078002871DD0021284A9DF8AC0002EB38
:1049900000129DF898001154BDF89000892865D048
:1049A0000CDC14287ED004DC08287CD010287BD1B5
:1049B000FEE3152879D08028F9D1FAE38B2875D049
:1049C0008C2874D08E2873D08F28F0D1BDF89C002D
:1049D0000D286ED19DF8AC0000EB4001C1EBC0107A
:1049E000114901EBC0004178114880F8111E9DF873
:1049F000AC0000EB4001C1EBC0100B4901EBC00063
:104A0000C17A0B4880F8121E9DF8AC0000EB8000C4
:104A1000014901EB40200DE0C0450020E0140020DA
:104A200000410020BC320020347C0020343F0020B4
:104A3000BC220020C0309DF8981001EB810202EBEF
:104A4000411110F8210003287EDCFE4890F8120E78
:104A500000287ADD9DF8AC0000EB8000FA4901EBFC
:104A60004021C0319DF8980001E0F0E3F8E300EB4D
:104A7000800202EB401001EB800109910878401C94
:104A8000C1B2099801709DF8AC0000EB8000EE49BE
:104A900001EB4020C0309DF8981001EB810202EB41
:104AA000411107E0FDE3FDE3FDE3FDE3FDE3FDE38D
:104AB000FDE3FDE310F82100042846DB9DF8AC007F
:104AC00000EB400101EB0010E04901EB0010303039
:104AD0009DF8981000EB0110801C0990D94890F8BF
:104AE000120EC0F30010C0F101000999097860F3BB
:104AF000000109980170D34890F8110EC0F3C0006E
:104B0000F0BB9DF8AC0000EB400101EB0010CF4979
:104B100001EB001030309DF8981000EB0110807808
:104B2000C0F3401060B39DF8AC0000EB400101EB16
:104B30000010C64901EB001030309DF8981000EBD2
:104B40000110801C099001E052E0E9E0007820F0BB
:104B50000201891C099801709DF8AC0000EB8000EF
:104B6000B94901EB4021C0319DF8980000EB80026B
:104B700002EB401001EB800018300990007800E053
:104B800009E020F00200801C099908709DF8AC1023
:104B90000220F5F7DDF900219DF8AC0000EB800064
:104BA000A94A02EB4020C17004229DF8AC0000EB42
:104BB0008000A54901EB4021C0319DF8980000EB31
:104BC000800303EB401001F820208C229DF8AC00FC
:104BD00000EB80009C4901EB4020C0309DF898100C
:104BE00001EB810303EB411100EB81004271A6E36D
:104BF0009DF8AC0000EB8000934901EB4021C031EF
:104C00009DF8980000EB800202EB401011F8201094
:104C10009DF8AC0000EB80008B4A02EB402000794D
:104C200081427DD19DF8AC0000EB400101EB00100A
:104C3000864901EB001030309DF8981000EB011010
:104C4000801C09907F4890F8120EC0F30010C0F14C
:104C5000010009990A7860F300020A709DF8AC001F
:104C600000EB400101EB0010784901EB00103030FF
:104C70009DF8981000EB0110801C0990714890F885
:104C8000110EC2080998017862F3410101709DF884
:104C9000AC0000EB400101EB00106C4901EB00118E
:104CA00030319DF8980001EB00108078C0F340028D
:104CB0009DF8AC0000EB8000634901EB4020C03060
:104CC0009DF8981001EB810303EB411100EB81008B
:104CD000007EC0F34000824263D09DF8AC0000EB40
:104CE0008000594901EB4020C0309DF8981001EB3D
:104CF000810202EB411100EB8100183009909DF810
:104D0000AC0000EB400101EB0010504901EB00103A
:104D100030309DF8981000EB01108078420800E0D8
:104D2000CCE20998017862F3410101709DF8AC0072
:104D300000EB400101EB0010444901EB0010303062
:104D40009DF8981000EB01108078C0F3400018BB6C
:104D500001229DF8AC0000EB80003B4901EB4021B3
:104D6000C0319DF8980000EB800303EB401001EB8D
:104D7000800042739DF8AC0000EB8000324901EBEB
:104D80004020C0309DF8981001EB810303EB4111E6
:104D900000EB810080F83E209DF8AC100220F5F772
:104DA000D7F89DF8AC0000EB400101EB001027495B
:104DB00001EB001130319DF8980001EB0010807874
:104DC00000F001029DF8AC0000EB80001E4901EBF1
:104DD0004020C0309DF8981001EB810303EB411196
:104DE00000EB8100007E00F0010082427DD09DF842
:104DF000AC0000EB8000144901EB4020C0309DF86E
:104E0000981001EB810202EB411100EB8100183098
:104E100009909DF8AC0000EB400101EB00100B493C
:104E200001EB001130319DF8980001EB0010817802
:104E30000998027861F3000202709DF8AC0000EB63
:104E4000400105E0BC220020C045002000410020B8
:104E500001EB0010FE4901EB001030309DF8981076
:104E600000EB0110807800F00100E8BB9DF8AC0079
:104E700000EB400101EB0010F54901EB0010303070
:104E80009DF8981000EB01108078C0F3401068B3D3
:104E90009DF8AC0000EB8000EE4901EB4020C030F3
:104EA0009DF8981001EB810202EB411100EB8100AB
:104EB00090F83E00D0B99DF8AC0000EB8000E549C9
:104EC00001EB4020C0309DF8981001EB810202EB0D
:104ED000411100EB8100407B40B99DF8AC0000EB34
:104EE000400101EB001002E045E066E12FE0D84907
:104EF00001EB001030309DF8981000EB0110807825
:104F0000C0F3400018BB01229DF8AC0000EB80000C
:104F1000D04901EB4021C0319DF8980000EB80039F
:104F200003EB401001EB800042739DF8AC0000EBF6
:104F30008000C84901EB4020C0309DF8981001EB7B
:104F4000810303EB411100EB810080F83E20002239
:104F50009DF8AC0000EB8000BE4901EB4020C03062
:104F60009DF8981001EB810303EB411100EB8100E8
:104F700080F83D2019E19DF8AC0000EB8000B549B8
:104F800001EB4020C0309DF8981001EB810202EB4C
:104F9000411100EB810090F83E0098B901229DF884
:104FA000AC0000EB8001AB4800EB4120C0309DF825
:104FB000981001EB810303EB411100EB810080F8B5
:104FC0003D2027E000229DF8AC0000EB8000A149C5
:104FD00001EB4021C0319DF8980000EB800303EB0A
:104FE000401001EB800080F83D209DF8AC0000EB04
:104FF000400101EB0010964901EB001130319DF8A2
:10500000980001EB0010801C0990007820F001024C
:1050100009980270904890F88C0880B19DF8AC0017
:1050200000EB400101EB0010894901EB001030302A
:105030009DF8981000EB0110807A022870D1874803
:10504000407F01286CD18548D0F814028349C98B70
:10505000884265D29DF8AC0000EB80007D4901EBF1
:105060004020C0309DF8981001EB810202EB411105
:1050700000EB810090F83D00012851D19DF8AC0073
:1050800000EB8000734901EB4020C0309DF8981080
:1050900001EB810202EB411100EB810090F87D00F1
:1050A000F0BB9DF8AC0000EB400101EB001068493B
:1050B00001EB001130319DF8980001EB00100178F0
:1050C0009DF8AC0000EB8000624A02EB402041708A
:1050D00008229DF8AC0000EB80005E4900E0F9E397
:1050E00001EB4021C0319DF8980000EB800303EBF9
:1050F000401001EB8000427100229DF8AC0000EBF3
:10510000400101EB0010524901EB001130319DF8D4
:10511000980001EB001042609DF8AC10022000E006
:1051200043E0F4F715FF0021379119E000229DF8C4
:10513000AC0000EB8000474901EB4021C0319DF8F5
:10514000980000EB800303EB401001EB80013F313E
:10515000BDF8DC000A54BDF8DC00401C81B2379178
:10516000BDF8DC001428E1DB0020379019E00022B4
:105170009DF8AC0000EB8000364901EB4021C031C6
:105180009DF8980000EB800303EB401001EB8001D9
:105190005B31BDF8DC000A54BDF8DC00401C81B274
:1051A0003791BDF8DC000A28E1DB9DF8AC1001E086
:1051B000F1E1ACE30220F4F7CBFE9DF8AC0000EB8C
:1051C0008000244901EB4020C0309DF8981001EB8D
:1051D000810202EB411100EB81008078802835D1FB
:1051E0009DF8AC0000EB400101EB0010184901EB09
:1051F000001030309DF8981000EB01108078C0F35B
:10520000400018BB9DF8AC0000EB400101EB001022
:105210000F4901EB001030309DF8981000EB0110A1
:105220008078C0F3401088B915229DF8AC0000EBDF
:105230008000084901EB4020C0309DF8981001EB38
:10524000810303EB411100EB8100427109E0FDE3B2
:1052500000410020C0450020BC320020BC120020CC
:10526000B0E19DF8AC0000EB400101EB0010FE49FD
:1052700001EB001030309DF8981000EB01108078A1
:10528000C0F34000D8B18F229DF8AC0000EB800045
:10529000F64901EB4020C0309DF8981001EB8103E6
:1052A00007E0EDE357E143E2EBE3EAE141E260E3EB
:1052B00050E103EB411100EB810042713FE09DF8AA
:1052C000AC0000EB8000E94901EB4020C0309DF8C4
:1052D000981001EB810202EB411100EB8100807B11
:1052E00001282CD100229DF8AC0000EB8000DF49A2
:1052F00001EB4021C0319DF8980000EB800303EBE7
:10530000401001EB800082738C229DF8AC0000EB12
:105310008000D64901EB4021C0319DF8980000EB98
:10532000800303EB401001EB8000427100219DF8E7
:10533000AC0000EB8000CD4A02EB4020C1709DF82C
:10534000AC0000EB400101EB0010C74901EB00107D
:10535000007BE8BB9DF8AC0000EB4001C1EBC01046
:10536000C34901EBC000807801049DF8AC0000EB5C
:105370004002C2EBC010BE4A02EBC000C07841EA56
:1053800000219DF8AC0000EB4002C2EBC010B84A0F
:1053900002EBC00000790843C117CDE9080108F00D
:1053A0005DFC9DF8AC1001EB8101B04A02EB41229B
:1053B000C0329DF8981001EB810303EB411102EB21
:1053C0008101C1F81E009DF8AC0000EB400100E037
:1053D00035E0C1EBC010A64901EBC00040790004E4
:1053E0009DF8AC1001EB4102C2EBC111A04A02EBE7
:1053F000C101897940EA01209DF8AC1001EB41021E
:10540000C2EBC1119A4A02EBC101C9790843C11725
:10541000CDE9080108F022FC9DF8AC1001EB8101F8
:10542000924A02EB4121C0319DF8982002EB8203A1
:1054300003EB421201EB8201C1F81A008AE09DF8E9
:10544000AC0000EB4001C1EBC010894901EBC0008A
:10545000807801069DF8AC0000EB4002C2EBC01062
:10546000834A02EBC000C07841EA00419DF8AC00DD
:1054700000EB4002C2EBC0107D4A02EBC000007995
:1054800041EA00219DF8AC0000EB4002C2EBC010E5
:10549000774A02EBC00040790843C117CDE9080103
:1054A00008F0DCFB9DF8AC1001EB81016F4A02EBC8
:1054B0004122C0329DF8981001EB810303EB4111AA
:1054C00002EB8101C1F81E009DF8AC0000EB400129
:1054D000C1EBC010664901EBC000807900069DF861
:1054E000AC1001EB4102C2EBC111614A02EBC101F8
:1054F000C97940EA01409DF8AC1001EB4102C2EBD2
:10550000C1115B4A02EBC101097A40EA01209DF812
:10551000AC1001EB4102C2EBC111554A02EBC101D3
:10552000497A0843C117CDE9080108F097FB024604
:105530009DF8AC0000EB80004C4901EB4020C030EE
:105540009DF8981001EB810303EB411100EB810002
:10555000C0F81A20ECE0BDF89C0003281AD18F2275
:105560009DF8AC0000EB8000404901EB4021C031C8
:105570009DF8980000EB800303EB401001EB8000E6
:10558000427101219DF8AC0000EB8000374A02EB2C
:105590004020C170CCE0BDF89C00032811D18F22BF
:1055A0009DF8AC0000EB8000304901EB4020C0309A
:1055B0009DF8981001EB810303EB411100EB810092
:1055C0004271B5E0BDF89C00032859D19DF8AC00AC
:1055D00000EB8000254901EB4020C030BDF8D01021
:1055E00001EB810202EB411100EB8100807901287F
:1055F00024D100229DF8AC0000EB80001B4901EB98
:105600004021C031BDF8D00000EB800303EB401017
:1056100001EB800082718F229DF8AC0000EB8000CE
:10562000124901EB4020C0309DF8981001EB810336
:1056300003EB411100EB8100427121E008229DF84B
:10564000AC0000EB8000094901EB4021C0319DF81E
:10565000980000EB800303EB401001EB80004271E7
:1056600000219DF8AC0005E000410020C04500206D
:10567000347C002000EB8000FE4A02EB4020C17029
:1056800056E0BDF89C00032852D19DF8AC0000EB19
:105690008000F84901EB4020C030BDF8D01001EB8C
:1056A000810202EB411100EB81008079012824D1B5
:1056B00000229DF8AC0000EB8000EE4901EB402198
:1056C000C031BDF8D00000EB800303EB401001EBCC
:1056D000800082718F229DF8AC0000EB8000E549CC
:1056E00001EB4020C0309DF8981001EB810303EBE3
:1056F000411100EB810042711AE008229DF8AC00D4
:1057000000EB8000DB4901EB4021C0319DF898009F
:1057100000EB800303EB401001EB8000427100219D
:105720009DF8AC0000EB8000D24A02EB4020C17033
:10573000FDE3BDF89C0008287DD19DF8AC0000EB8E
:105740004001C1EBC010CC4901EBC00080780106DC
:105750009DF8AC0000EB4002C2EBC010C64A02EB61
:10576000C000C07841EA00419DF8AC0000EB400267
:10577000C2EBC010C04A02EBC000007941EA002031
:105780009DF8AC1001EB4102C2EBC111BA4A02EB29
:10579000C10149790843C117CDE9080108F05EFA53
:1057A0009DF8AC1001EB8101B24A02EB4122C032FC
:1057B0009DF8981001EB810303EB411102EB81018D
:1057C00048639DF8AC0000EB8000AA4901EB402043
:1057D000C0309DF8981001EB810202EB411110F8E6
:1057E00021009DF8AC1001EB8101A24A02EB41219E
:1057F000097988422DDA00219DF8AC0000EB800089
:1058000002EB4020C17005229DF8AC0000EB800047
:10581000984901EB4021C0319DF8980000EB8003CE
:1058200003EB401001F820208E229DF8AC0000EB25
:105830008000904900E069E001EB4021C0319DF813
:10584000980000EB800303EB401001EB80004271F5
:105850005CE09DF8AC0000EB8000864901EB402045
:10586000C030BDF8D01001EB810202EB411100EB1A
:105870008100807901282ED100229DF8AC0000EB38
:1058800080007C4901EB4021C031BDF8D00000EB25
:10589000800303EB401001EB800082718F229DF8A2
:1058A000AC0000EB8000734901EB4021C0319DF852
:1058B000980000EB800303EB401001EB8000427185
:1058C00001219DF8AC0000EB80006A4A02EB402009
:1058D000C1701BE0FDE38E229DF8AC0000EB800060
:1058E000644901EB4021C0319DF8980000EB800332
:1058F00003EB401001EB8000427100219DF8AC00E9
:1059000000EB80005B4A02EB4020C1700FE3BDF862
:105910009C0003282CD100219DF8AC0000EB8000F6
:10592000544A02EB4020C17001229DF8AC0000EB0C
:105930008000504901EB4021C031BDF8D00000EBA0
:10594000800303EB401001EB800082718C229DF8F4
:10595000AC0000EB8000474901EB4020C0309DF8CF
:10596000981001EB810303EB411100EB81004271C0
:10597000DDE2BDF89C000F2869D19DF8AC0000EB7A
:10598000400101EB00103D4901EB0010007BE8BB3A
:1059900000202C902D900021379120E0DDE92C1083
:1059A000000240EA11620902CDE92C129DF8AC0018
:1059B00000EB4001C1EBC0102F4901EBC001BDF865
:1059C000DC00C0F10600085CDDE92C3440EA03028B
:1059D000CDE92C24BDF8DC00401C81B23791BDF824
:1059E000DC000528DADB9DF8AC00DDE92C1200EBC9
:1059F0008000204B03EB4023C0339DF8980000EB60
:105A0000800404EB401003EB800000E04EE040F81F
:105A1000221F426000222C922D920021379122E019
:105A2000DDE92C10000240EA11620902CDE92C12D6
:105A30009DF8AC0000EB4001C1EBC0100E4901EB3A
:105A4000C001BDF8DC00C0F10B0001E0EDE33FE375
:105A5000085CDDE92C341843CDE92C04BDF8DC00EA
:105A6000401C80B23790BDF8DC000528D8DB9DF8DB
:105A7000AC0007E0C0450020347C0020004100203D
:105A8000B7E327E3DDE92C2100EB8000FE4B03EBBD
:105A90004020C0309DF8983003EB830404EB43139F
:105AA00000EB830022308260C1607DE000202C90FA
:105AB0002D90002137911FE0DDE92C10000240EA13
:105AC00011620902CDE92C129DF8AC0000EB4001F7
:105AD000C1EBC010ED4901EBC001BDF8DC00C0F125
:105AE0000700085CDDE92C341843CDE92C04BDF82F
:105AF000DC00401C80B23790BDF8DC000628DBDB00
:105B00009DF8AC00DDE92C1200EB8000DE4B03EBCE
:105B10004023C0339DF8980000EB800404EB401054
:105B200003EB800040F8221F426000222C922D924D
:105B3000002137911FE0DDE92C10000240EA1162DC
:105B40000902CDE92C129DF8AC0000EB4001C1EB3D
:105B5000C010CE4901EBC001BDF8DC00C0F10D0062
:105B6000085CDDE92C341843CDE92C04BDF8DC00D9
:105B7000401C80B23790BDF8DC000628DBDB9DF8C6
:105B8000AC00DDE92C1200EB8000BF4B03EB4020A2
:105B9000C0309DF8983003EB830404EB431300EB13
:105BA000830022308160C2609DF8AC0000EB800071
:105BB000B54901EB4021C0319DF8980000EB80020F
:105BC00002EB401011F820109DF8AC0000EB8000B3
:105BD000AD4A02EB4020007981427DD1AC4890F87B
:105BE0008C08E8BBAB48D0F814020521B0FBF1F2F9
:105BF00001FB120000EBC00101EB0011A5482030B1
:105C000000EB81000021C0F81D10A248D0F814025A
:105C10000521B0FBF1F201FB120000EBC00101EB2A
:105C200000119C48203000EB81000D3009909DF858
:105C3000AC0000EB8000944901EB4021C0319DF89D
:105C4000982002EB820000EB421001EB8000223032
:105C50001022014608900998F2F7F7FA8D4800E003
:105C6000D6E0D0F814020521B0FBF1F201FB1200DE
:105C700000EBC00101EB00118648203000EB8102EF
:105C80009DF8AC0000EB80007F4901EB4021C03162
:105C90009DF8980000EB800303EB401001EB8000BF
:105CA00050F81A1F42F8011F406850607948D0F838
:105CB00014020521B0FBF1F201FB120000EBC00160
:105CC00001EB0013734920319DF8AC0000EB40025A
:105CD00002EB0010704A00E09DE102EB001230324E
:105CE0009DF8980002EB0010007801F82300694845
:105CF000D0F814020521B0FBF1F201FB120000EB19
:105D0000C00101EB00116348203000EB81016048C5
:105D1000826941F8212F808B88805E48D0F8140278
:105D20000521B0FBF1F201FB120000EBC00101EB19
:105D300000115848203000EB81029DF8AC0000EBC8
:105D40008000514901EB4021C0319DF8980000EBE3
:105D5000800303EB401001EB8000406BC2F80900A8
:105D60004C48D0F814020521B0FBF1F201FB1200FF
:105D700000EBC00101EB00114648203000EB81022E
:105D80009DF8AC0000EB400101EB0010424901EB33
:105D9000001130319DF8980001EB00104068C2F806
:105DA00027003C48D0F814020521B0FBF1F081B285
:105DB00002200991F3F78CF900210620F4F7C8F8C6
:105DC0003448D0F814023349C98B884206D231488E
:105DD000D0F81402401C2F49C1F8140200210520FC
:105DE000F4F7B6F89DF8AC0000EB400101EB0010B1
:105DF000294901EB001030309DF8981000EB01109C
:105E0000801C0990007820F008020998027015E0C3
:105E10009DF8AC0000EB400101EB00101E4901EBC6
:105E2000001030309DF8981000EB0110801C099094
:105E3000007820F008000830099908709DF8AC003F
:105E400000EB400101EB0010134901EB0010303072
:105E50009DF8981000EB0110801C0990007820F04C
:105E60002002099802709DF8AC100220F4F770F837
:105E70009DF8AC009DF8981001EB0010C217CDE919
:105E80002C0200222C9809E0C0450020347C002020
:105E9000BC320020BC1200200041002000EBC001F9
:105EA00001EB0011FC4800EB8100C0F81D209DF8BB
:105EB000AC0000EB8000F94901EB4020C0309DF8B8
:105EC000981001EB810202EB411100EB81002230BE
:105ED00009902C9800EBC00101EB0011EE4800EB9B
:105EE00081010D3110220891DDE90801F2F7ADF9C9
:105EF0009DF8AC0000EB8000E84901EB4021C03187
:105F00009DF8980000EB800202EB401001EB80014D
:105F10002C9800EBC00202EB0012DF4800EB82007D
:105F200051F81A2F40F8012F4968416000E07BE1E9
:105F30009DF8AC0000EB400101EB0010D84901EBEB
:105F4000001130319DF8980001EB001001782C9879
:105F500000EBC00202EB0012CF4800F822102C9890
:105F600000EBC00101EB0011CB4800EB8101CD48F3
:105F7000826941F8212F808B88809DF8AC0000EB6E
:105F80008000C64901EB4021C0319DF8980000EB2C
:105F9000800202EB401001EB8000416B2C9800EB7B
:105FA000C00202EB0012BC4800EB8200C0F80910EE
:105FB0009DF8AC0000EB400101EB0010B84901EB8B
:105FC000001130319DF8980001EB001041682C98C9
:105FD00000EBC00202EB0012AF4800EB8200C0F8F9
:105FE00027102C9881B208200991F3F7B1FF002205
:105FF0009DF8AC0000EB8000A84901EB4020C030C8
:106000009DF8981001EB810303EB411100EB810037
:1060100080F83E204AE09DF8AC0000EB400101EB27
:1060200000109F4901EB001030309DF8981000EBF4
:106030000110801C0990007820F00401091D0998C6
:1060400001709DF8AC0000EB400101EB0010944999
:1060500001EB001130319DF8980001EB0010801C1D
:106060000990007820F080008030099908700122A2
:106070009DF8AC0000EB8000884901EB4020C27025
:106080009DF8AC0000EB800001EB402002799DF808
:10609000AC0000EB800001EB4020C0309DF8981070
:1060A00001EB810303EB411100F821208F229DF8C1
:1060B000AC0000EB8000794901EB4020C0309DF836
:1060C000981001EB810303EB411100EB8100427159
:1060D000AAE0ABE0BDF89C00032848D1012171483B
:1060E00080F8B0179DF8AC0000EB80006B4901EB25
:1060F0004021C0319DF8980000EB800202EB401077
:1061000011F820109DF8AC0000EB8000634A02EB10
:106110004020007981422BDA00219DF8AC0000EB91
:10612000800002EB4020C17001229DF8AC0000EB22
:1061300080005A4901EB4021C0319DF8980000EBE6
:10614000800303EB401001F820208F229DF8AC0063
:1061500000EB8000514901EB4020C0309DF89810C1
:1061600001EB810303EB411100EB810042713FE041
:106170009DF8AC0000EB8000484901EB4020C030A6
:106180009DF8981001EB810202EB411100EB8100B8
:10619000807880282CD100219DF8AC0000EB800095
:1061A0003E4A02EB4020C17080229DF8AC0000EB1B
:1061B00080003A4901EB4021C0319DF8980000EB86
:1061C000800303EB401001EB8000427100229DF838
:1061D000AC0000EB8000314901EB4020C0309DF85D
:1061E000981001EB810303EB411100EB81008270F9
:1061F0001AE0BDF89C00032815D10021294880F839
:10620000B0178F229DF8AC0000EB8000234901EB12
:106210004020C0309DF8981001EB810303EB411141
:1062200000EB8100427100BF00BF00BF00BF1D48EE
:10623000C07DB0B11C499DF8AC0031F81010099137
:106240009DF8AC1001EB4100C0EBC110174901EB08
:10625000C001012308919DF8AC20DDE90801F4F7A5
:1062600017FC0021379111E000219DF8AC0000EBF4
:106270004002C2EBC0100D4A02EBC002BDF8DC00C8
:106280001154BDF8DC00401C81B23791BDF8DC0030
:10629000142850DAE8E70000E0140020C045002090
:1062A00000410020BC320020C06D0020347C002062
:1062B000D0499DF8AC0011F81000C009D8BB9DF87A
:1062C000AC0011F81000C0F3C300062832D2DFE89A
:1062D00000F0036291FEFD339DF8AC0000EB40013D
:1062E000C1EBC010C44901EBC0010991C3A10998D9
:1062F00015F060FE11901198E0B100219DF8AC00FE
:1063000000EB4000BB4A3C3202EB800041600121BF
:106310009DF8AC0000EB400002EB80008170B549B5
:106320009DF8AC0001EB40010991087820F078005D
:10633000283008704DE14DE19DF8AC0000EB4001C4
:10634000C1EBC010AC4901EBC0010991ABA10998A8
:1063500015F030FE11901198E0B100219DF8AC00CD
:1063600000EB4000A34A3C3202EB80004160012177
:106370009DF8AC0000EB400002EB800081709D496D
:106380009DF8AC0001EB40010991087820F07800FD
:10639000203008701DE19DF8AC0000EB4001C1EB1E
:1063A000C010954901EBC001099194A1099815F01D
:1063B00001FE11901198E0B100219DF8AC0000EBB6
:1063C00040008C4A3C3202EB8000416001219DF884
:1063D000AC0000EB400002EB8000817085499DF825
:1063E000AC0001EB40010991087820F078001830EA
:1063F0000870EEE000219DF8AC0000EB40007D4A03
:106400003C3202EB8000416001219DF8AC0000EBC2
:10641000400002EB800081709DF8AC0000EB400171
:10642000C1EBC010744901EBC0011198801D095CDB
:1064300030399DF8AC0000EB4002C2EBC0106E4A50
:1064400002EBC0021198401D105C303841EA001088
:10645000C117CDE9080106F04DFE694988719DF824
:10646000AC0000EB4001C1EBC010634901EBC0017F
:10647000099164A1099815F09DFD1190119838B308
:106480009DF8AC0000EB4001C1EBC0105A4901EB94
:10649000C0011198401C085C302826DB9DF8AC0038
:1064A00000EB4001C1EBC010534901EBC001119852
:1064B000401C085C30389DF8AC1001EB4102C2EB87
:1064C000C1114D4A02EBC103119902E058E02BE0E3
:1064D0001EE0595C303940EA0110C117CDE90801CE
:1064E00006F008FE4649C87112E09DF8AC1001EBB9
:1064F0004100C0EBC110404901EBC0011198085C9C
:106500003038C117CDE9080106F0F4FD3C49C871E7
:1065100038499DF8AC0001EB40010991087820F062
:1065200078001830087054E09DF8AC1001EB410081
:10653000C0EBC110304901EBC00109912FA10998AE
:1065400015F038FD11901198C8B100202E4908604F
:1065500028499DF8AC0001EB40010991087820F032
:1065600080018031099801704FF47A719DF8AC0078
:1065700000EB40001F4A3C3202EB8000816028E0C3
:106580009DF8AC1001EB4100C0EBC1101A4901EBC2
:10659000C001099119A1099815F00CFD11901198ED
:1065A000B0B11A4890F8B20720F08001174880F87F
:1065B000B21710499DF8AC0001EB40010991087831
:1065C00020F0780008300870002011498870486079
:1065D00000BF00BF0F4800780F49097808440F49F1
:1065E000097808440E4909780844002874F464AC1A
:1065F00038B070BDC83E0020347C00204F4B0000F6
:10660000483B00202C00000088024242BC3200209F
:10661000006E002012000020130000201400002053
:106620001500002007B5D4B000211A9119911891D6
:1066300017911691159114910022129213921092B3
:1066400011920F910E910D910C910B910A91FBA05B
:1066500006C8CDE90812FBA006C8CDE90612002144
:1066600005910020F9490870549800EB400101EBB6
:106670000010F74901EB001081791691F549549803
:1066800001EB00115598085C05287CDD0621F14AD4
:10669000549802EB0012559811540022549800EBC4
:1066A0008000ED4901EB4021C031559800EB80039B
:1066B00003EB401001F82020549800EB400101EB5F
:1066C0000010E34901EB00113031559801EB001047
:1066D000807820F08002549800EB400101EB00101C
:1066E000DB4901EB00113031559801EB001082704D
:1066F000549800EB8000D84901EB4021C0315598F7
:1067000000EB800202EB401001EB800090F88E005D
:1067100020F00802549800EB8000CF4901EB4021A3
:10672000C031559800EB800303EB401001EB800073
:1067300080F88E20549800EB8000C74901EB40217F
:10674000C031559800EB800202EB401001EB800055
:1067500090F88E0020F00102549800EB8000BE49B2
:1067600001EB4021C031559800EB800303EB401052
:1067700001EB800080F88E20549800EB400101EB83
:106780000010B34900E094E001EB00108079092883
:1067900016D2DFE800F08D05162738495A6B7C00C9
:1067A000E522549800EB8000AB4901EB4021C03159
:1067B000559800EB800303EB401001EB8000427121
:1067C00076E0A122549800EB8000A34901EB402021
:1067D000C030559901EB810303EB411100EB8100BF
:1067E000427165E0A122549800EB80009A4901EBC8
:1067F0004020C030559901EB810303EB411100EBC0
:106800008100427154E0B122549800EB800092491B
:1068100001EB4020C030559901EB810303EB41119E
:1068200000EB8100427143E03122549800EB80007C
:10683000894901EB4021C031559800EB800303EBFF
:10684000401001EB8000427132E0F422549800EBDA
:106850008000814901EB4020C030559901EB810354
:1068600003EB411100EB8100427121E006225498B4
:1068700000EB8000784901EB4021C031559800EBD6
:10688000800303EB401001EB8000427110E0152201
:10689000549800EB8000704901EB4020C0305599BE
:1068A00001EB810303EB411100EB8100427100BF5A
:1068B00000BF68496C39549811F810000121B1EB00
:1068C000D01F46F03B826548007F012806F02782F2
:1068D0009DF858000028F9D09DF858000A2886F045
:1068E000A681DFE810F04C2B0A005709600ED81281
:1068F0005F16961791204E27DB2D549800EB400130
:1069000001EB0010524901EB00113031559801EBB9
:106910000010417808460491002107F09FF9C1B2A8
:106920001591549800EB80004B4901EB4021C03198
:10693000559800EB800202EB401011F8201054989B
:1069400000EB8000444A02EB40200079814206D1EE
:106950000121549800EB800002EB4020C1703D49BA
:10696000549801EB00115598085C401CC1B2394A9B
:10697000549802EB001255981154549800EB800083
:10698000354901EB4020C030559901EB810202EB03
:10699000411100EB810090F88E00C0F3C00090B16F
:1069A000549800EB400101EB0010294901EB001065
:1069B00041790B464FF4805204914FF4E1315498E1
:1069C00007F03AF819E0549800EB400101EB001091
:1069D0001F4901EB001041790491549800EB4001EC
:1069E00001EB00101A4901EB0010016803914FF40C
:1069F0008052049B549807F01FF85698C52875D00C
:106A000012DCB52873D008DC112871D0122870D0A0
:106A100013286FD0B22868D1A4E3B6286BD0B92868
:106A20006AD0C328F7D1E0E2D92866D018DCCA289A
:106A30007DD0CE287CD0D528EDD118E00169323048
:106A4000313030000169323045303000160000200E
:106A500000410020343F0020C0450020BC1200202F
:106A6000E12866D0E52865D0E728D4D1F3E3F52105
:106A70005498C0EB001000EB8000F84A02F8301088
:106A80009DF854105498C0EB001000EB800002EB0E
:106A9000C0004170A2215498C0EB001000EB8000B0
:106AA00002EBC0008170D5215498C0EB001000EBC0
:106AB000800002EBC000C1705498C0EB001000EBE6
:106AC0008000114601EBC00104910321049806F0F7
:106AD000A1FF01465498C0EB001000EB8000DF4A94
:106AE00002EBC000017105210F91FDE3FDE348E0D9
:106AF000FCE3FCE3FCE3F6E25BE1F5215498C0EB38
:106B0000001000EB8000D54A02F830109DF85410B8
:106B10005498C0EB001000EB800002EBC000417005
:106B2000A2215498C0EB001000EB800003E09BE230
:106B3000FAE3FAE3FAE302EBC0008170D92154983A
:106B4000C0EB001000EB800002EBC000C170549855
:106B5000C0EB001000EB8000114601EBC001049176
:106B60000321049806F056FF01465498C0EB00102C
:106B700000EB8000B94A02EBC000017105210F91C2
:106B8000B3E7F5215498C0EB001000EB8000B34A46
:106B900002F830109DF854105498C0EB001000EB30
:106BA000800002EBC0004170549800EB400101EB03
:106BB0000010AB4901EB0010007B00287DD15498F8
:106BC00000EB800001F5986101EB4020C030559941
:106BD00001EB810202EB411100EB81008068B0F50E
:106BE000100F05D34FF410010020CDE9101011E073
:106BF000549800EB80009B4901EB4020C030559930
:106C000001EB810202EB411100EB81008068002260
:106C1000CDE91002A5215498C0EB001000EB8000D4
:106C20008E4A02EBC000817000211A911CE0BDF871
:106C30006800C0F10200C200DDE91001CDE91B10BF
:106C4000F1F7F1FAC2B25498C0EB001000EB8000EB
:106C5000824901EBC003BDF86800C01C1A54BDF89E
:106C60006800401C80B21A90BDF868000328DEDB83
:106C7000B5215498C0EB001000EB8000774A02EB7E
:106C8000C00081715498C0EB001000EB80001146E9
:106C900001EBC00104910621049806F0BBFE0146F9
:106CA0005498C0EB001000EB80006C4A02EBC0006F
:106CB000C17108210F917BE0FFE7549800EB800041
:106CC000684901EB4020C030559901EB810202EB8D
:106CD000411100EB81008068B0F1104F05D34FF0F7
:106CE00010400021CDE9100111E0549800EB800024
:106CF0005C4901EB4020C030559901EB810202EB69
:106D0000411100EB810080680022CDE91002A6212C
:106D10005498C0EB001000EB8000504A02EBC0001A
:106D2000817000211A911CE0BDF86800C0F10300D9
:106D3000C200DDE91001CDE91D10F1F774FAC2B20D
:106D40005498C0EB001000EB8000444901EBC003F5
:106D5000BDF86800C01C1A54BDF86800401C80B221
:106D60001A90BDF868000428DEDBB5215498C0EB0A
:106D7000001000EB8000394A02EBC000C17154984A
:106D8000C0EB001000EB8000114601EBC001049144
:106D90000721049806F03EFE01465498C0EB00100F
:106DA00000EB80002D4A02EBC000017209210F9117
:106DB0009BE6F5215498C0EB001000EB8000274AB9
:106DC00002F830109DF854105498C0EB001000EBFE
:106DD000800002EBC0004170549800EB400101EBD1
:106DE00000101F4901EB0010007BB0BB549800EB72
:106DF00080001C4901EB4020C030559901EB810215
:106E000002EB411100EB81008068B0F5100F05D155
:106E10004FF410010020CDE9101011E0549800EB60
:106E20008000104901EB4020C030559901EB8102F0
:106E300002EB411100EB810080680022CDE91002D5
:106E4000A5215498C0EB001000EB8000034A02EB30
:106E5000C000817000211A9123E04AE0D472002022
:106E600000410020C0450020BDF86800C0F10200CC
:106E7000C200DDE91001CDE91F10F1F7D4F9C2B26B
:106E80005498C0EB001000EB8000FA4901EBC003FE
:106E9000BDF86800C01C1A54BDF86800401C80B2E0
:106EA0001A90BDF868000328DEDBB9215498C0EBC6
:106EB000001000EB8000EF4A02EBC0008171549893
:106EC000C0EB001000EB8000114601EBC001049103
:106ED0000621049806F09EFD01465498C0EB001070
:106EE00000EB8000E34A02EBC000C17108210F9162
:106EF0007AE0549800EB8000DF4901EB4020C0307D
:106F0000559901EB810202EB411100EB8100806891
:106F1000B0F1104F05D14FF010400021CDE9100124
:106F200011E0549800EB8000D34901EB4020C030C1
:106F3000559901EB810202EB411100EB8100806861
:106F40000022CDE91002A6215498C0EB001000EBFE
:106F50008000C84A02EBC000817000211A911CE039
:106F6000BDF86800C0F10300C200DDE91001CDE901
:106F70002110F1F758F9C2B25498C0EB001000EBA1
:106F80008000BC4901EBC003BDF86800C01C1A5466
:106F9000BDF86800401C80B21A90BDF86800042853
:106FA000DEDBB9215498C0EB001000EB8000B14A41
:106FB00002EBC000C1715498C0EB001000EB8000E0
:106FC000114601EBC00104910721049806F022FD4F
:106FD00001465498C0EB001000EB8000A54A02EB7C
:106FE000C000017209210F917FE5F5215498C0EB93
:106FF000001000EB80009F4A02F830109DF85410FA
:107000005498C0EB001000EB800002EBC000417010
:10701000A2215498C0EB001000EB800002EBC000EE
:107020008170C3215498C0EB001000EB800002EB8C
:10703000C000C1705498C0EB001000EB80001146F6
:1070400001EBC00104910321049806F0E3FC014622
:107050005498C0EB001000EB8000864A02EBC000A1
:10706000017105210F9140E5F5215498C0EB001006
:1070700000EB80007F4A02F830109DF854105498BD
:10708000C0EB001000EB800002EBC0004170A221B9
:107090005498C0EB001000EB800002EBC000817040
:1070A000CA215498C0EB001000EB800002EBC00036
:1070B000C1705498C0EB001000EB8000114601EB4A
:1070C000C00104910321049806F0A4FC01465498E1
:1070D000C0EB001000EB8000664A02EBC0000171BB
:1070E00005210F9101E5F5215498C0EB001000EB4C
:1070F0008000604A02F830109DF854105498C0EB9C
:10710000001000EB800002EBC0004170A2215498F7
:10711000C0EB001000EB800002EBC0008170B621D4
:107120005498C0EB001000EB800002EBC000C1706F
:107130005498C0EB001000EB8000114601EBC00139
:1071400004910321049806F065FC01465498C0EBB5
:10715000001000EB8000474A02EBC00001710521DE
:107160000F91C2E4F5215498C0EB001000EB8000B1
:10717000404A02F830109DF854105498C0EB0010AB
:1071800000EB800002EBC0004170549800EB40011E
:1071900001EB0010394901EB0010007BE8BBA42192
:1071A0005498C0EB001000EB800002EBC00081702F
:1071B00000211A9125E0549800EB80002E4901EB44
:1071C0004021C031559800EB800202EB401001EBEA
:1071D0008000416BBDF86800C0F10100C000C140F3
:1071E0005498C0EB001000EB8000224A02EBC00272
:1071F000BDF86800C01C1154BDF86800401C81B285
:107200001A91BDF868000228D5DBB2215498C0EB72
:10721000001000EB8000174A00E01DE002EBC00008
:1072200041715498C0EB001000EB8000114601EB57
:10723000C00104910521049806F0ECFB0146549826
:10724000C0EB001000EB80000A4A02EBC000817125
:1072500007210F9167E0A6E2A5215498C0EB00102A
:1072600000EB8000034A02EBC000817000211A91FC
:107270002CE00000D4720020C04500200041002016
:10728000549800EB8000FB4901EB4021C031559838
:1072900000EB800202EB401001EB8000416BBDF877
:1072A0006800C0F10200C000C1405498C0EB00105B
:1072B00000EB8000F04A02EBC002BDF86800C01C81
:1072C0001154BDF86800401C81B21A91BDF86800E5
:1072D0000328D5DBB2215498C0EB001000EB8000EE
:1072E000E54A02EBC00004E01DE28DE09AE2F7E21D
:1072F00050E381715498C0EB001000EB8000114600
:1073000001EBC00104910621049806F083FB0146BD
:107310005498C0EB001000EB8000D74A02EBC0008D
:10732000C17108210F91FEE1ADE000E0FCE1F52123
:107330005498C0EB001000EB8000CF4A02F83010E8
:107340009DF854105498C0EB001000EB800002EB45
:10735000C0004170A6215498C0EB001000EB8000E3
:1073600002EBC000817000211A9125E0549800EBD7
:107370008000C04901EB4021C031559800EB8002EC
:1073800002EB401001EB8000816BBDF86800C0F19A
:107390000300C000C1405498C0EB001000EB800017
:1073A000B54A02EBC002BDF86800C01C1154BDF81C
:1073B0006800401C81B21A91BDF868000428D5DB32
:1073C000E1215498C0EB001000EB8000AA4A02EBC8
:1073D000C000C1715498C0EB001000EB8000114652
:1073E00001EBC00104910721049806F013FB01464C
:1073F0005498C0EB001000EB80009F4A02EBC000E5
:10740000017209210F91C2E3F5215498C0EB0010DD
:1074100000EB8000984A02F830109DF85410549800
:10742000C0EB001000EB800002EBC0004170A22115
:107430005498C0EB001000EB800002EBC00081709C
:10744000C5215498C0EB001000EB800002EBC00097
:10745000C1705498C0EB001000EB8000114601EBA6
:10746000C00104910321049806F0D4FA014654980F
:10747000C0EB001000EB80007F4A02EBC0000171FE
:1074800005210F9183E3F5215498C0EB001000EB28
:107490008000794A02F830109DF854105498C0EBDF
:1074A000001000EB800002EBC0004170549800EB2C
:1074B000400101EB0010714901EB0010007BE8BBBB
:1074C000AC215498C0EB001000EB800002EBC00030
:1074D000817000211A912DE0549800EB80006549DD
:1074E00001EB4020C030559901EB810202EB4111C4
:1074F00000EB810050F8221F4068BDF86820C2F1FF
:107500000402D200CDE9230108462399F0F78BFE4F
:10751000C2B25498C0EB001000EB8000564901EB5A
:10752000C003BDF86800C01C1A54BDF86800401CB8
:1075300080B21A90BDF86800052800E057E0CBDB68
:1075400000201A902BE0549800EB8000494901EB91
:107550004020C030559901EB810202EB411100EB54
:10756000810122318868C968BDF86820C2F104022F
:10757000D200CDE92510F0F756FEC2B25498C0EB08
:10758000001000EB80003C4901EBC003BDF868002F
:1075900008301A54BDF86800401C80B21A90BDF83B
:1075A00068000528CFDBCE215498C0EB001000EB1B
:1075B0008000314A02EBC00041735498C0EB0010C8
:1075C00000EB8000114601EBC00104910D210498ED
:1075D00006F020FA01465498C0EB001000EB800042
:1075E000254A02EBC00081730F210F919BE0AE2171
:1075F0005498C0EB001000EB80001F4A02EBC00063
:10760000817000211A912DE0549800EB80001949F7
:1076100001EB4020C030559901EB810202EB411192
:1076200000EB810050F8221F4068BDF86820C2F1CD
:107630000502D200CDE9270108462799F0F7F3FDAE
:10764000C2B25498C0EB001000EB80000A4901EB75
:10765000C003BDF86800C01C1A54BDF86800401C87
:1076600080B21A90BDF868000628CDDB00201A9081
:1076700032E00000C0450020D4720020004100200C
:10768000549800EB8000FE4901EB4020C030559932
:1076900001EB810202EB411100EB8101223188688C
:1076A000C968BDF86820C2F10502D200CDE92910F1
:1076B000F0F7B9FDC2B25498C0EB001000EB8000A7
:1076C000F04901EBC003BDF8680009301A54BDF859
:1076D0006800401C80B21A90BDF868000628CFDB15
:1076E000CE215498C0EB001000EB8000E54A02EB7D
:1076F000C000C1735498C0EB001000EB800011462D
:1077000001EBC00104910F21049806F083F90146B2
:107710005498C0EB001000EB8000DA4A02EBC00086
:10772000017411210F9132E2F5215498C0EB001041
:1077300000EB8000D34A02F830109DF854105498A2
:10774000C0EB001000EB800002EBC0004170A221F2
:107750005498C0EB001000EB800002EBC000817079
:10776000E5215498C0EB001000EB800002EBC00054
:10777000C1705498C0EB001000EB8000114601EB83
:10778000C00104910321049806F044F9014654987D
:10779000C0EB001000EB8000BA4A02EBC0000171A0
:1077A00005210F91F3E1F5215498C0EB001000EB97
:1077B0008000B44A02F830109DF854105498C0EB81
:1077C000001000EB800002EBC0004170A221549831
:1077D000C0EB001000EB800002EBC0008170E721DD
:1077E0005498C0EB001000EB800002EBC000C170A9
:1077F0005498C0EB001000EB8000114601EBC00173
:1078000004910321049806F005F901465498C0EB51
:10781000001000EB80009B4A02EBC00001710521C3
:107820000F91B4E1F5215498C0EB001000EB8000FB
:10783000944A02F830109DF854105498C0EB001090
:1078400000EB800002EBC0004170A2215498C0EB15
:10785000001000EB800002EBC000817011215498F1
:10786000C0EB001000EB800002EBC000C170549828
:10787000C0EB001000EB8000114601EBC001049149
:107880000321049806F0C6F801465498C0EB001096
:1078900000EB80007B4A02EBC000017105210F91D3
:1078A0000122549800EB8001754800EB4121C03162
:1078B000559800EB800303EB401001F82020D522FF
:1078C000549800EB80006E4901EB4020C030559980
:1078D00001EB810303EB411100EB8100427156E1A2
:1078E000F5215498C0EB001000EB8000654A02F8C7
:1078F00030109DF854105498C0EB001000EB80003D
:1079000002EBC0004170A5215498C0EB001000EBC1
:10791000800002EBC000817001215498C0EB001080
:1079200000EB800002EBC000C170C2215498C0EB94
:10793000001000EB800002EBC000017100215498A0
:10794000C0EB001000EB800002EBC000417112217F
:107950005498C0EB001000EB800002EBC000817176
:107960005498C0EB001000EB8000114601EBC00101
:1079700004910621049806F04DF801465498C0EB96
:10798000001000EB80003F4A02EBC000C1710821EB
:107990000F91FCE0F5215498C0EB001000EB800043
:1079A000384A02F830109DF854105498C0EB00107B
:1079B00000EB800002EBC0004170FF215498C0EB47
:1079C000001000EB800002EBC000817000211A91D2
:1079D0001CE0549800EB400101EB00102A4901EB38
:1079E00000110E31BDF86800095C5498C0EB00101E
:1079F00000EB8000234A02EBC002BDF86800C01C07
:107A00001154BDF86800401C81B21A91BDF868009D
:107A10000A28DEDB549800EB400101EB00101A4904
:107A200001EB0010408B01125498C0EB001000EBEA
:107A30008000144A02EBC0004173549800EB4001EF
:107A400001EB0010104901EB0010408BC1B25498BB
:107A5000C0EB001000EB800002EBC0008173549873
:107A600000EB8000064901EB4021C031559800EB46
:107A7000800202EB401001EB8000B0F88C0005E0C2
:107A8000C0450020D472002000410020011254980B
:107A9000C0EB001000EB8000FB4A02EBC000C1739A
:107AA000549800EB8000F94901EB4021C031559812
:107AB00000EB800202EB401001EB8000B0F88C007C
:107AC000C1B25498C0EB001000EB8000EE4A02EB0C
:107AD000C0000174549800EB8000EC4901EB402198
:107AE000C031559800EB800202EB401001EB8000A2
:107AF000B0F88C10549801EB802081B203200491DF
:107B0000F1F74AFA00211A9114E0E149BDF8680042
:107B1000095C5498C0EB001000EB8000DA4A02EBDD
:107B2000C002BDF8680011301154BDF86800401C57
:107B300081B21A91BDF86800B0F5007FE5DB132132
:107B40005498C0EB001000EB8000CF4A02EBC0005D
:107B500080F811125498C0EB001000EB8000114621
:107B600001EBC001049140F21121049805F052FF8D
:107B700001465498C0EB001000EB8000C24A02EBB3
:107B8000C00080F8121240F213210F9100BF00BF15
:107B900005F04DB8549800EB400101EB0010BD49D1
:107BA00001EB00113031559801EB0010417815912F
:107BB000549800EB8000B54901EB4021C031559845
:107BC00000EB800202EB401011F82010549800EBFB
:107BD0008000AE4A02EB40200079814206D10121AB
:107BE000549800EB800002EB4020C170AA495498E1
:107BF00001EB00115598085C401CC1B2A64A54988C
:107C000002EB0012559811549DF85400002804DD31
:107C10009DF85400401EC1B215915698A1380A280B
:107C20007ED2DFE800F0FCFBFAF9F8F7F605F5F490
:107C300002215498C0EB001000EB8000924A02F839
:107C400030109DF854004030C1B25498C0EB001081
:107C500000EB800002EBC000417041215498C0EB62
:107C6000001000EB800002EBC000817030215498BE
:107C7000C0EB001000EB800002EBC000C170549814
:107C8000C0EB001000EB800002EBC00001715498C3
:107C900000EB80007D4901EB4021C031559800EB9D
:107CA000800202EB401001EB80000079010954983A
:107CB000C0EB001000EB8000734A02EBC000417182
:107CC0005498C0EB001000EB8000114601EBC0009F
:107CD00040790A2812DA5498C0EB001000EB8000BB
:107CE00001EBC00040793030C1B25498C0EB0010B5
:107CF00000EB800002EBC000417115E05498C0EB2E
:107D0000001000EB8000604901EBC0004079373083
:107D1000C1B25498C0EB001000EB80005A4A00E05A
:107D200043E202EBC0004171549800EB80005749D8
:107D300001EB4021C031559800EB800202EB40106E
:107D400001EB8000007900F00F015498C0EB0010A7
:107D500000EB80004C4A02EBC00081715498C0EBEC
:107D6000001000EB8000114601EBC00080790A286A
:107D700012DA5498C0EB001000EB800001EBC00059
:107D800080793030C1B25498C0EB001000EB800015
:107D900002EBC000817113E05498C0EB001000EBBF
:107DA0008000394901EBC00080793730C1B2549866
:107DB000C0EB001000EB8000334A02EBC000817181
:107DC00003225498C0EB001000EB80002E4901EB19
:107DD000C000C2715498C0EB001000EB800001EBB2
:107DE000C000401C07210490F1F774FB0146549831
:107DF000C0EB001000EB8000234A02EBC0000172D0
:107E000009210F91549800EB8000204908E05EE1C1
:107E1000C1E0B0E39AE3EAE2C8E10FE168E03DE0E7
:107E200001EB4020C030559901EB810202EB41117A
:107E300010F8210004280ED10522549800EB800090
:107E4000124901EB4020C030559901EB810303EB4F
:107E5000411100F821200021549800EB80000B4ACA
:107E600002EB4020C1700622549800EB80000749C5
:107E700001EB4020C030559901EB810303EB411128
:107E800000F821208CE30000D4720020C0450020BF
:107E9000D230002000410020343F002004215498BB
:107EA000C0EB001000EB8000FA4A02F830109DF899
:107EB00054004030C1B25498C0EB001000EB800079
:107EC00002EBC000417051215498C0EB001000EB50
:107ED000800002EBC000817005215498C0EB0010B7
:107EE00000EB800002EBC000C17004210F9157E34A
:107EF00002215498C0EB001000EB8000E54A02F824
:107F000030109DF854004030C1B25498C0EB0010BE
:107F100000EB800002EBC000417041215498C0EB9F
:107F2000001000EB800002EBC000817031215498FA
:107F3000C0EB001000EB800002EBC000C1703521E7
:107F40005498C0EB001000EB800002EBC000017100
:107F500003215498C0EB001000EB800002EBC0003E
:107F600041715498C0EB001000EB8000114601EB0A
:107F7000C000401C05210490F1F7ACFA014654986A
:107F8000C0EB001000EB8000C24A02EBC000817120
:107F900007210F9104E302215498C0EB001000EB7D
:107FA0008000BC4A02F830109DF854004030C1B245
:107FB0005498C0EB001000EB800002EBC000417051
:107FC00041215498C0EB001000EB800002EBC00090
:107FD000817032215498C0EB001000EB800002EB5E
:107FE000C000C17030215498C0EB001000EB80003D
:107FF00002EBC000017103215498C0EB001000EBAC
:10800000800002EBC00041715498C0EB001000EBFF
:108010008000114601EBC000401C05210490F1F7DF
:1080200059FA01465498C0EB001000EB8000994AC1
:1080300002EBC000817107210F91B1E20421549835
:10804000C0EB001000EB8000924A02F830109DF85F
:1080500054004030C1B25498C0EB001000EB8000D7
:1080600002EBC000417041215498C0EB001000EBBE
:10807000800002EBC000817005215498C0EB001015
:1080800000EB800002EBC000C17004210F915498F6
:1080900000EB8000804901EB4020C030559901EB96
:1080A000810202EB411110F8210002280ED10322B7
:1080B000549800EB8000784901EB4020C03055997E
:1080C00001EB810303EB411100F8212068E202215A
:1080D0005498C0EB001000EB80006E4A02F830109C
:1080E0009DF854004030C1B25498C0EB001000EB32
:1080F000800002EBC000417041215498C0EB001099
:1081000000EB800002EBC000817031215498C0EB7D
:10811000001000EB800002EBC000C17032215498C7
:10812000C0EB001000EB800002EBC00001710321E6
:108130005498C0EB001000EB800002EBC0004171CE
:108140005498C0EB001000EB8000114601EBC0001A
:10815000401C05210490F1F7BDF901465498C0EB8D
:10816000001000EB80004B4A02EBC0008171072138
:108170000F91549800EB400101EB0010474901EBCF
:1081800000113031559801EB0010807820F020026A
:10819000549800EB400101EB0010404901EB001046
:1081A0003030559900EB01108270F9E102215498AA
:1081B000C0EB001000EB8000364A02F830109DF84A
:1081C00054004030C1B25498C0EB001000EB800066
:1081D00002EBC000417041215498C0EB001000EB4D
:1081E000800002EBC000817031215498C0EB001078
:1081F00000EB800002EBC000C17030215498C0EB4E
:10820000001000EB800002EBC0000171549800EBFD
:108210008000214901EB4020C030559901EB8102DB
:1082200002EB411100EB81008068B0F5100F0AD31A
:1082300030215498C0EB001000EB8000154A02EB8F
:10824000C000417109E032215498C0EB001000EBEE
:108250008000104A02EBC0004171549800EB80008E
:108260000D4901EB4020C030559901EB810202EB32
:10827000411100EB8100C079012811D131215498BE
:10828000C0EB001000EB8000024A02EBC0008171DD
:1082900020E00000D4720020C045002000410020F2
:1082A000549800EB8000FC4901EB4020C030559908
:1082B00001EB810202EB411100EB8100C07948B96A
:1082C00032215498C0EB001000EB8000F34A02EB1F
:1082D000C000817100201A9028E0549800EB8000C3
:1082E000ED4901EB4021C031559800EB800202EBD3
:1082F000401001EB80008168BDF86800C0F1050006
:108300008000C14001F00F0130315498C0EB0010E3
:1083100000EB8000E14A02EBC002BDF86800C01D1E
:108320001154BDF86800401C81B21A91BDF8680074
:108330000628D2DB32215498C0EB001000EB8000FD
:10834000D64A02EBC000417300211A9128E05498EC
:1083500000EB8000D04901EB4021C031559800EB83
:10836000800202EB401001EB8000416BBDF8680019
:10837000C0F103008000C14001F00F01303154987A
:10838000C0EB001000EB8000C44A02EBC002BDF855
:1083900068000E301154BDF86800401C81B21A917B
:1083A000BDF868000428D2DB03225498C0EB00100B
:1083B00000EB8000B94901EBC00082745498C0EB17
:1083C000001000EB800001EBC000401C1221049063
:1083D000F1F780F801465498C0EB001000EB8000E4
:1083E000AE4A02EBC000C17414210F91D8E0022103
:1083F0005498C0EB001000EB8000A84A02F830103F
:108400009DF854004030C1B25498C0EB001000EB0E
:10841000800002EBC000417041215498C0EB001075
:1084200000EB800002EBC000817032215498C0EB59
:10843000001000EB800002EBC000C17031215498A5
:10844000C0EB001000EB800002EBC0000171322194
:108450005498C0EB001000EB800002EBC0004171AB
:108460005498C0EB001000EB800002EBC00081715B
:1084700000211A9128E0549800EB8000864901EB16
:108480004021C031559800EB800202EB401001EB17
:108490008000416BBDF86800C0F103008000C1405E
:1084A00001F00F0130315498C0EB001000EB800058
:1084B0007A4A02EBC002BDF86800C01D1154BDF835
:1084C0006800401C81B21A91BDF868000428D2DB14
:1084D00000201A9011E030215498C0EB001000EBFE
:1084E00080006E4A02EBC002BDF868000B301154E8
:1084F000BDF86800401C81B21A91BDF868001928C7
:10850000E9DB03225498C0EB001000EB80006349C4
:1085100001EBC00080F824205498C0EB001000EB61
:10852000800001EBC000401C24210490F0F7D2FF32
:1085300001465498C0EB001000EB8000574A02EB54
:10854000C00080F8251026210F9129E010215498B1
:10855000C0EB001000EB8000504A02F830103021D0
:108560005498C0EB001000EB800002EBC00041709B
:1085700002210F9114E010215498C0EB001000EB81
:108580008000464A02F8301031215498C0EB0010A8
:1085900000EB800002EBC000417002210F9100BF90
:1085A00000BF04F044BB549800EB400101EB001005
:1085B0003B4901EB00113031559801EB0010417837
:1085C0001591549800EB8000334901EB4021C031F4
:1085D000559800EB800202EB401011F820105498DF
:1085E00000EB80002C4A02EB40200079814206D14A
:1085F0000121549800EB800002EB4020C170294912
:10860000549801EB00115598085C401CC1B2254AF2
:10861000549802EB0012559811549DF8540000280C
:1086200004DD9DF85400401EC1B215915698A13842
:108630000A282FD2DFE800F00538DEFEFDFCFB2E15
:108640008BFA04215498C0EB001000EB8000134A11
:1086500002F830109DF854004030C1B25498C0EB7D
:10866000001000EB800002EBC000417051215498D3
:10867000C0EB001000EB800002EBC0008170052110
:108680005498C0EB001000EB800002EBC000C170FA
:1086900004210F91FCE30000C0450020D4720020AB
:1086A00000410020343F002002215498C0EB00100C
:1086B00000EB8000FE4A02F830109DF85400403074
:1086C000C1B25498C0EB001000EB800002EBC00078
:1086D000417041215498C0EB001000EB800002EB88
:1086E000C000817031215498C0EB001000EB800075
:1086F00002EBC000C17035215498C0EB001000EBB4
:10870000800002EBC000017103215498C0EB0010FF
:1087100000EB800002EBC00041715498C0EB0010E8
:1087200000EB8000114601EBC000401C05210490C5
:10873000F0F7D0FE01465498C0EB001000EB80002B
:10874000DB4A02EBC000817107210F91A0E30221F7
:108750005498C0EB001000EB8000D54A02F83010AE
:108760009DF854004030C1B25498C0EB001000EBAB
:10877000800002EBC000417041215498C0EB001012
:1087800000EB800002EBC000817032215498C0EBF6
:10879000001000EB800002EBC000C1703021549843
:1087A000C0EB001000EB800002EBC0000171032160
:1087B0005498C0EB001000EB800002EBC000417148
:1087C0005498C0EB001000EB8000114601EBC00094
:1087D000401C05210490F0F77DFE01465498C0EB43
:1087E000001000EB8000B24A02EBC000817107214B
:1087F0000F914DE304215498C0EB001000EB800072
:10880000AB4A02F830109DF854004030C1B2549881
:10881000C0EB001000EB800002EBC0004170412172
:108820005498C0EB001000EB800004E012E01AE363
:1088300004E353E27DE002EBC0008170052154980F
:10884000C0EB001000EB800002EBC000C1700421FF
:108850000F911DE302215498C0EB001000EB800043
:10886000934A02F830109DF854004030C1B2549839
:10887000C0EB001000EB800002EBC0004170412112
:108880005498C0EB001000EB800002EBC000817038
:1088900031215498C0EB001000EB800002EBC000C7
:1088A000C17032215498C0EB001000EB800002EB45
:1088B000C000017103215498C0EB001000EB800050
:1088C00002EBC00041715498C0EB001000EB800037
:1088D000114601EBC000401C05210490F0F7FAFDA1
:1088E00001465498C0EB001000EB8000704A02EB88
:1088F000C0008171549800EB400101EB00106D49FC
:1089000001EB00113031559801EB0010807820F018
:108910002002549800EB400101EB0010654901EB87
:1089200000113031559801EB0010827007210F9132
:10893000AEE202215498C0EB001000EB80005C4ACC
:1089400002F830109DF854004030C1B25498C0EB8A
:10895000001000EB800002EBC000417041215498F0
:10896000C0EB001000EB800002EBC00081703121F1
:108970005498C0EB001000EB800002EBC000C17007
:1089800041215498C0EB001000EB800002EBC000C6
:108990000171549800EB8000474901EB4020C03042
:1089A000559901EB810202EB411100EB81008068D7
:1089B000B0F1104F0AD130215498C0EB001000EBF9
:1089C00080003B4A02EBC000417109E0322154981B
:1089D000C0EB001000EB8000354A02EBC000417193
:1089E000549800EB8000344901EB4020C030559989
:1089F00001EB810202EB411100EB8100C0790128FB
:108A00000AD131215498C0EB001000EB8000284AB5
:108A100002EBC000817119E0549800EB80002649F8
:108A200001EB4020C030559901EB810202EB41116E
:108A300000EB8100C07948B932215498C0EB001096
:108A400000EB80001A4A02EBC000817100201A90EE
:108A500028E0549800EB8000174901EB4021C03119
:108A6000559800EB800202EB401001EB800081681A
:108A7000BDF86800C0F107008000C14001F00F019F
:108A800030315498C0EB001000EB8000084A02EB34
:108A9000C002BDF86800C01D1154BDF86800401C3C
:108AA00081B21A91BDF868000828D2DB322105E0B6
:108AB000D472002000410020C04500205498C0EB33
:108AC000001000EB8000FE4A02EBC000C1730021E1
:108AD0001A9128E0549800EB8000FA4901EB4021FC
:108AE000C031559800EB800202EB401001EB800092
:108AF000416BBDF86800C0F105008000C14001F085
:108B00000F0130315498C0EB001000EB8000EC4AAC
:108B100002EBC002BDF8680010301154BDF86800C7
:108B2000401C81B21A91BDF868000628D2DB3021C2
:108B30005498C0EB001000EB8000E14A02EBC0004B
:108B4000817500211A9111E030215498C0EB00107A
:108B500000EB8000DA4A02EBC002BDF86800173073
:108B60001154BDF86800401C81B21A91BDF868002C
:108B70000628E9DB30215498C0EB001000EB8000A0
:108B8000CF4A02EBC000417700211A9111E0302159
:108B90005498C0EB001000EB8000C94A02EBC00201
:108BA000BDF868001E301154BDF86800401C81B249
:108BB0001A91BDF868000628E9DB30215498C0EB13
:108BC000001000EB8000BE4A02EBC00080F82410C9
:108BD00000211A9111E030215498C0EB001000EBF5
:108BE0008000B74A02EBC002BDF86800253011547E
:108BF000BDF86800401C81B21A91BDF868000628D3
:108C0000E9DB30215498C0EB001000EB8000AC4A47
:108C100002EBC00080F82B1000211A9111E03021E6
:108C20005498C0EB001000EB8000A54A02EBC00294
:108C3000BDF868002C301154BDF86800401C81B2AA
:108C40001A91BDF868000628E9DB30215498C0EB82
:108C5000001000EB80009A4A02EBC00080F832104E
:108C600000211A9111E030215498C0EB001000EB64
:108C70008000934A02EBC002BDF868003330115403
:108C8000BDF86800401C81B21A91BDF86800062842
:108C9000E9DB03225498C0EB001000EB8000884908
:108CA00001EBC00080F839205498C0EB001000EBB5
:108CB000800001EBC000401C39210490F0F70AFC51
:108CC00001465498C0EB001000EB80007C4A02EB98
:108CD000C00080F83A103B210F91D9E0022154984E
:108CE000C0EB001000EB8000754A02F830109DF8D0
:108CF00054004030C1B25498C0EB001000EB80002B
:108D000002EBC000417041215498C0EB001000EB11
:108D1000800002EBC000817032215498C0EB00103B
:108D200000EB800002EBC000C17031215498C0EB11
:108D3000001000EB800002EBC00001713321549859
:108D4000C0EB001000EB800002EBC000417132214B
:108D50005498C0EB001000EB800002EBC000817162
:108D600000211A9128E0549800EB8000554901EB4E
:108D70004021C031559800EB800202EB401001EB1E
:108D80008000416BBDF86800C0F105008000C14063
:108D900001F00F0130315498C0EB001000EB80005F
:108DA000474A02EBC002BDF86800C01D1154BDF86F
:108DB0006800401C81B21A91BDF868000628D2DB19
:108DC00000201A9011E030215498C0EB001000EB05
:108DD00080003B4A02EBC002BDF868000D30115420
:108DE000BDF86800401C81B21A91BDF868001928CE
:108DF000E9DB03225498C0EB001000EB80003049FF
:108E000001EBC00080F826205498C0EB001000EB66
:108E1000800001EBC000401C26210490F0F75AFBB3
:108E200001465498C0EB001000EB8000244A02EB8E
:108E3000C00080F8271028210F9129E010215498B4
:108E4000C0EB001000EB80001D4A02F8301030210A
:108E50005498C0EB001000EB800002EBC0004170A2
:108E600002210F9114E010215498C0EB001000EB88
:108E70008000134A02F8301031215498C0EB0010E2
:108E800000EB800002EBC000417002210F9100BF97
:108E900000BF03F0CCBE549800EB400101EB001082
:108EA000094901EB00113031559801EB0010417870
:108EB0001591549800EB8000024901EB402105E038
:108EC000D4720020C045002000410020C031BDF810
:108ED000680000EB800202EB401011F8201054985B
:108EE00000EB8000FE4A02EB40200079814206D16F
:108EF0000121549800EB800002EB4020C170F94939
:108F0000549801EB00115598085C401CC1B2F54A19
:108F1000549802EB00125598115400211A9117E051
:108F2000549800EB400101EB0010EF4901EB0011F8
:108F30003031BDF8680001EB001041789DF8540015
:108F4000814200D111E0BDF86800401C81B21A9145
:108F5000549800EB400101EB0010E34901EB0010D5
:108F6000C179BDF868008142DADC00BF549800EB9B
:108F7000400101EB0010DC4901EB00113031BDF87C
:108F8000680001EB001001785598401A401CC1B2EE
:108F900014919DF85400002804DD9DF85400401EF3
:108FA000C1B21591549800EB8000CD4901EB4020EF
:108FB000C030559901EB810202EB411100EB8100B9
:108FC00040780F2820DA549800EB8000C44901EB68
:108FD0004021C031559800EB800202EB401001EBBC
:108FE00080004078401CC2B2549800EB8000BC491D
:108FF00001EB4020C030559901EB810303EB411197
:1090000000EB810042700FE00022549800EB8000DA
:10901000B34901EB4020C030559901EB810303EBCC
:10902000411100EB810042705698B138092826D2D0
:10903000DFE800F00526FD2525FC25B5FB009DF8A1
:1090400054005030C1B25498C0EB001000EB8000C7
:10905000A64A02F8301020215498C0EB001000EB13
:10906000800002EBC0004170FA215498C0EB001060
:1090700000EB800002EBC000817003210F918FE2B2
:109080009DF854005030C1B25498C0EB001000EB72
:109090008000964A02F83010549800EB8000904906
:1090A00001EB4021C031559800EB800202EB4010EB
:1090B00001EB8000407840F030015498C0EB001084
:1090C00000EB8000894A02EBC000417001215498F6
:1090D000C0EB001000EB800002EBC00081705498E0
:1090E000C0EB001000EB800002EBC000C17000215B
:1090F0005498C0EB001000EB800002EBC00001713F
:109100005498C0EB001000EB8000114601EBC00149
:10911000049105210498F0F70BFE0022CDE910021E
:109120001098C2B25498C0EB001000EB80006F4959
:1091300001EBC0004271DDE91020010641EA122076
:10914000C2B25498C0EB001000EB8000674901EBFD
:10915000C000827103225498C0EB001000EB800025
:1091600001EBC000C271FA225498C0EB001000EB72
:10917000800001EBC000027209200F90B1225498C8
:1091800000EB8000564901EB4020C030559901EBBF
:10919000810303EB411100EB8100427100E29DF875
:1091A00054005030C1B25498C0EB001000EB800066
:1091B0004E4A02F83010549800EB8000484901EB09
:1091C0004021C031559800EB800202EB401001EBCA
:1091D0008000407840F030015498C0EB001000EB64
:1091E0008000424A02EBC000417065215498C0EBF8
:1091F000001000EB800002EBC00081700121549848
:10920000C0EB001000EB800002EBC000C1709DF8C5
:1092100050105498C0EB001000EB800002EBC0002F
:1092200001715498C0EB001002E03DE047E1C7E057
:1092300000EB8000114601EBC00104910521049868
:10924000F0F776FD0022CDE910021098C2B25498D2
:10925000C0EB001000EB8000244901EBC00042711C
:10926000DDE91020010641EA1220C2B25498C0EB99
:10927000001000EB80001D4901EBC0008271032249
:109280005498C0EB001000EB800001EBC000C271ED
:10929000FA225498C0EB001000EB800001EBC000F4
:1092A000027209200F907BE19DF854005030C1B24A
:1092B0005498C0EB001000EB80000C4A02F830100C
:1092C000549800EB8000064901EB4021C0315598CD
:1092D00000EB800202EB401001EB8000407807E0D9
:1092E000C0450020343F002000410020D4720020FF
:1092F00040F030015498C0EB001000EB8000FE4AB3
:1093000002EBC000417065215498C0EB001000EBE7
:10931000800002EBC000817001215498C0EB001066
:1093200000EB800002EBC000C1709DF8500040F0DF
:1093300010015498C0EB001000EB800002EBC0005D
:1093400001715498C0EB001000EB8000114601EB56
:10935000C001049105210498F0F7EAFC0022CDE950
:1093600010021098C2B25498C0EB001000EB8000BD
:10937000E14901EBC0004271DDE91001000A40EA59
:109380000160C2B25498C0EB001000EB8000DA49D3
:1093900001EBC000827103225498C0EB001000EB77
:1093A000800001EBC000C271FA225498C0EB00109B
:1093B00000EB800001EBC000027209200F90EFE08B
:1093C0009DF854005030C1B25498C0EB001000EB2F
:1093D0008000C94A02F83010549800EB8000C74959
:1093E00001EB4021C031559800EB800202EB4010A8
:1093F00001EB8000407840F030015498C0EB001041
:1094000000EB8000BC4A02EBC0004170012154987F
:10941000C0EB001000EB800002EBC000817054989C
:10942000C0EB001000EB800002EBC000C170052112
:109430005498C0EB001000EB800002EBC0000171FB
:109440005498C0EB001000EB8000114601EBC00106
:10945000049105210498F0F76BFC0022CDE910027D
:109460001098C2B25498C0EB001000EB8000A249E3
:1094700001EBC0004271DDE91001000A40EA016021
:10948000C1B25498C0EB001000EB80009A4A02EB86
:10949000C000817103215498C0EB001000EB8000E4
:1094A00002EBC000C171FA215498C0EB001000EB30
:1094B000800002EBC000017209210F9170E0549806
:1094C00000EB80008D4901EB4020C030559901EB45
:1094D000810202EB411100EB81008078B1282DD090
:1094E000549800EB8000854901EB4021C03155982C
:1094F00000EB800202EB401001EB80008278549870
:1095000000EB80007D4901EB4021C031559800EB14
:10951000800303EB401001EB80004271B1225498AC
:1095200000EB8000754901EB4020C030559901EBFC
:10953000810303EB411100EB810082709DF8540020
:109540005030C1B25498C0EB001000EB80006A4A62
:1095500002F83010549800EB8000684901EB40217C
:10956000C031559800EB800202EB401001EB800007
:10957000407840F0C0015498C0EB001000EB800030
:109580005D4A02EBC0004170FA215498C0EB001014
:1095900000EB800002EBC000817003210F9100BF3F
:1095A00000BF76E45649549801EB0011BDF86800FD
:1095B000014404910878401CC1B204980170549889
:1095C00000EB400101EB00104E4901EB0010007B65
:1095D00020B1012846D0022843D1B3E05698312863
:1095E00002D045283CD11DE000201A9013E008A9C4
:1095F000BDF86800095C5498C0EB001000EB8000D7
:109600003D4A02EBC002BDF868001154BDF8680085
:10961000401C81B21A91BDF868000728E7DB0720DB
:109620000F901DE000201A9013E006A9BDF8680015
:10963000095C5498C0EB001000EB80002E4A02EB4E
:10964000C002BDF868001154BDF86800401C81B22A
:109650001A91BDF868000728E7DB07200F9000BFCC
:1096600000BFD4E05598401CC1B215919DF854102C
:109670005498C0EB001000EB80001F4A02F8301035
:1096800003215498C0EB001000EB800002EBC000F7
:10969000417000215498C0EB001000EB800002EBF9
:1096A000C000817002215498C0EB001000EB8000D4
:1096B00002EBC000C17000215498C0EB001000EB19
:1096C000800002EBC000017109215498C0EB00102A
:1096D00000EB800002EBC00041715498C0EB001019
:1096E00000EB8000114601EBC001049106210498B3
:1096F000F0F7D4F8002207E0D4720020C045002023
:10970000343F002000410020CDE91002DDE91010B7
:10971000020642EA1120C1B25498C0EB001000EBDF
:109720008000FE4A02EBC000C1711098C1B254988B
:10973000C0EB001000EB800002EBC000817108213B
:109740000F9164E05598401CC1B215919DF85410DA
:109750005498C0EB001000EB8000F04A02F8301083
:1097600003215498C0EB001000EB800002EBC00016
:10977000417000215498C0EB001000EB800002EB18
:10978000C00081705498C0EB001000EB800002EB29
:10979000C000C1705498C0EB001000EB800002EBD9
:1097A000C000017102215498C0EB001000EB800052
:1097B00002EBC00041715498C0EB001000EB800038
:1097C000114601EBC001049106210498F0F766F8F8
:1097D0000022CDE91002DDE91020010641EA122045
:1097E000C2B25498C0EB001000EB8000CB4901EBF3
:1097F000C000C2711098C2B25498C0EB001000EBC8
:10980000800001EBC000827108200F9000BF00BFF4
:10981000C7E6C349549801EB00115598085C401CF9
:10982000C1B2BF4A549802EB001255981154549893
:1098300000EB400101EB0010BA4901EB001130319F
:10984000559801EB001041781591549800EB800079
:10985000B54901EB4020C030559901EB810202EB84
:10986000411100EB810090F87700002850DD0020C6
:109870001A901FE0549800EB8000AB4901EB4021A7
:10988000C031BDF86800559A104400EB800202EB2D
:10989000401011F82010549800EB8000A24A02EB0F
:1098A00040200079814200D018E0BDF86800401CDB
:1098B00081B21A91549800EB80009B4901EB402142
:1098C000C031559800EB800202EB401001EB8000A4
:1098D00090F87710BDF868008142CBDC00BF549847
:1098E00000EB8000904901EB4021C031559800EB1E
:1098F000800202EB401001EB800090F87710BDF879
:109900006800814204D15698052801D0062056905F
:109910005698F2287DD006DC05287BD0062809D091
:10992000F12878D1DBE3F32876D0F42875D0F62837
:10993000F7D1FCE3549800EB80007B4901EB402019
:10994000C030559901EB810202EB411100EB81001F
:1099500090F87700002875DD549800EB800072497C
:1099600001EB4021C031559800EB800202EB401022
:1099700001EB800090F879109DF8540081423BD0B3
:10998000549800EB8000684901EB4021C0315598A4
:1099900000EB800202EB401001EB800090F87A109F
:1099A0009DF85400814227D0549800EB80005E4916
:1099B00001EB4021C031559800EB800202EB4010D2
:1099C00001EB800090F87B109DF85400814213D089
:1099D000549800EB8000544901EB4021C031559868
:1099E00000EB800202EB401001EB800090F87C104D
:1099F0009DF85400814225D1549800EB80004A49DB
:109A000001EB4021C031559800EB800202EB401081
:109A100004E0C0E3FEE361E3FDE3FDE301EB80006E
:109A200090F87710491E549800EB80003E4A02EBF4
:109A3000402080780844C1B2549800EB800002EBCB
:109A400040208170F5215498C0EB001000EB80009D
:109A5000324A02F830109DF854105498C0EB0010B0
:109A600000EB800002EBC000417000215498C0EB75
:109A7000001000EB800002EBC00081705498C0EB36
:109A8000001000EB800002EBC000C170062154986A
:109A9000C0EB001000EB800002EBC000017105215B
:109AA0000F9100210B91B4E2549800EB80001E4905
:109AB00001EB4021C031BDF82C205598104400EB3B
:109AC000800202EB401001EB80004079F12804D0C5
:109AD000F2284ED0F3284BD1D1E1549800EB40014D
:109AE00001EB00100F4901EB00113031BDF82C00E3
:109AF000559A104401EB001041785498C0EB0010C7
:109B000000EB8000054A02EBC002BDF83C00115496
:109B1000BDF83C00401C81B20F9107E0D4720020D8
:109B2000343F002000410020C0450020549800EB45
:109B30008000FE4901EB4021C031BDF82C00559A50
:109B4000104400EB800202EB401001EB80004179F1
:109B50005498C0EB001000EB8000F54A02EBC00205
:109B6000BDF83C001154BDF83C00401C81B20F917F
:109B700049E2549800EB400101EB0010ED4901EB84
:109B800000113031BDF82C00559A104401EB001043
:109B900041785498C0EB001000EB8000E44A02EBDF
:109BA000C002BDF83C001154BDF83C00401C81B21D
:109BB0000F91549800EB8000DC4901EB4021C0314B
:109BC000BDF82C00559A104400EB800202EB4010C7
:109BD00001EB800041795498C0EB001000EB80004D
:109BE000D34A02EBC002BDF83C001154BDF83C0062
:109BF000401C81B20F91549800EB8000CB4901EBDF
